:0700000C322E362E312E3298
:1000000AD7F2F8DA1E13F9D419252908E32301E6F1
:1000000A0407E929160508EE1319F11B1FF4FDFA76
:1000000AFEFC05FE03FE45392BF64B3E482D054501
:1000000A30340917191A161B16161A1E191B17232C
:1000000A252622272222262A25222C2B322D322D62
:1000000A2D3135302D36363D383D38383C403B3879
:1000000A5B3D5F306655583E6363415B5F448D815B
:0500000A733E74636603
:020000040800F2
:40800000C0EC0020D5BD0008E7BD0008C5DB0308EBBD0008EDBD0008EFBD00080000000000000000000000000000000021830008F3BD000800000000E583000859840008B4
:40804000F9BD0008F9BD0008F9BD0008F9BD0008F9BD0008F9BD0008F9BD0008F9BD0008F9BD0008F9BD0008F9BD0008F9BD0008F9BD0008F9BD0008F9BD0008F9BD000820
:40808000F9BD0008F9BD0008D14303082F490308434A0308F9BD0008F9BD0008F9BD00085BAC030867AC030873AC0308EBAB03080DAC03081BAC030827AC03083D740308A5
:4080C0004D7403085D74030867740308F9BD0008717D03086D5403087754030881540308F9BD0008F9BD0008F9BD00087FAC03088BAC030897AC03084FAC0308F9BD0008F5
:40810000F9BD0008F9BD000831AC0308F9BD0008F9BD0008F9BD00083DAC030847AC0308F9BD0008F9BD0008F9BD0008F9BD0008F9BD0008F9BD0008F9BD0008E949030840
:40814000B74A03082D4B0308F9BD0008F9BD0008F9BD0008F9BD0008F9BD00089F5403087174030881740308F9BD0008F9BD0008F9BD0008F9BD0008F9BD00080000000016
:40818000F9BD0008F9BD0008A9540308B3540308F9BD0008F9BD00087B7D0308F9BD00080000000000000000F9BD000800F002F800F073F80AA090E8000C82448344AAF193
:4081C0000107DA4501D100F068F8AFF2090EBAE80F0013F0010F18BFFB1A43F001031847E0DB030000DC03000A444FF0000C10F8013B13F0070408BF10F8014B1D1108BFA0
:4082000010F8015B641E05D010F8016B641E01F8016BF9D113F0080F1EBF10F8014BAD1C0C1B09D16D1E58BF01F801CBFAD505E014F8016B01F8016B6D1EF9D59142D6D37C
:40824000704700000023002400250026103A28BF78C1FBD8520728BF30C148BF0B607047632935F05083732935F05583002070471FB53AF04CF89DE8030035F0DAFA35F042
:408280005EF935F028FC04000020002139F070F9401C60601FBD10B510BD35F0F7FB1146FFF7E6FF11F0A7FE35F028FC03B4FFF7F2FF03BC35F058FC80F309887047EFF312
:4082C00009807047684680F3098804480078C00714BF0220032080F314887047084D0408DFF818C0EFF305831B0618BF6047EFF31483DB0708BF604700DF7047F7060408A2
:40830000DFF818C0EFF305831B0618BF6047EFF31483DB0708BF604700DF7047FD080408EFF30980816911F8021C01B142E010B590E80F10E047BDE81040EFF3098C254B66
:4083400093E80600914232D041B91EF0100F16D12149086820F00100086010E00CB41EF0100F06BF2CED108A0323012381F826302CE9F00FC1F82CC038F056FE0CBC1A6061
:40838000D2F82CC0BCE8F00F92F8263013F0020F1ABFBCEC108A6FF0120E6FF0020E8CF3098813F0010F08BF704792F82500CCF80000704710B5094A1268914209D8084C02
:4083C00054F8214090E80F10A047EFF3098C8CE80F0010BD9C07002034EF00E0B4DB0308B4DB030810B538F0D3FCBDE81040194B93E80600914208BF70470CB4EFF3098C73
:408400001EF0100F06BF2CED108A0223002381F826302CE9F00FC1F82CC038F005FE0CBC1A60D2F82CC0BCE8F00F92F8263013F0020F1ABFBCEC108A6FF0120E6FF0020E04
:408440008CF3098813F0010F1CBF92F82530CCF8003070479C07002010B538F0B5FEC4E710B538F047F938F0AFFEBEE70B49D1F800C04A685CF8043B1068184442F8040B80
:408480008C4528BFA1F1DC0C8A4228BFA1F1DC02C1F800C04A6020F000407047B8E600200146F948B0F8AA0000EE100AB8EE400A81ED080AF44890ED800A81ED010A90EDF4
:4084C000810A81ED020A90ED820A81ED030A90F8AF0000EE100AB8EE400A81ED050AEA4890F8AE000877E84890ED7D0A81ED000A90F8B00000EE100AB8EE400A81ED060A06
:40850000B7EE000A81ED040A012070474FF6FF76DFF878C300DF074639460120DFF870C300DF0421DB4880F8D01100BF002231460120DFF864C300DF0446012C17D100BFA2
:40854000D44890F8D10140F00101D24880F8D111B0F8DC014FF6FF71884207DACD48B0F8DC01401C81B2CB48A0F8DC11DEE7022CDCD1DFF828C300DF054605F0010000288F
:40858000D4D0C748FFF78CFFD0E7C54880ED0C0ADFEDC40AC0ED0D0ADFEDC20AC0ED0F0ADFEDC00AC0ED0E0A80ED0A0A704710B52DED0C8BB0EE409AB0EE608AF0EE419AC2
:4085C0009FEDB80AF0EE408A2022B549243101F1200035F054F89FEDB40AC9EE000AB048C0ED090AB5EEC08AF1EE10FA04D1B0EE480AFFF7CAFF10E1B5EEC08AF1EE10FA89
:4086000007DDA74890ED120AB5EEC00AF1EE10FA0CD9B5EEC08AF1EE10FA0FD2A04890ED120AB5EEC00AF1EE10FA07DBB0EE480AFFF7ABFF2FF05FFC99498866984A92EDE8
:40864000080ABCEEC00A10EE101A906E2FF059FC50BBB5EEC08AF1EE10FA0ADD9FED930A8F4880ED0A0A9FED8F0A914880ED000A11E09FED900A8A4880ED0A0AD0ED050AE6
:40868000B7EE001A81EE200AF0EE000A80EE201A874880ED001A824890ED0A0A80ED0C0A012085490870B8E09FED800AB4EEC08AF1EE10FA07DB9FED810A794880ED0A0A79
:4086C000F0EE488A80E09FED7B0AB4EEC08AF1EE10FA07D89FED7A0A714880ED0A0AF0EE488A71E0724890ED000A30EE290A80ED000A6B4890ED050ADFED720A20EE200A92
:408700006B48D0ED000A20EE200A10EE101A084639F08CFD41EC1D0BB0EE4D0AF0EE6D0A37F01EF8B0EE40BAF0EE60BA5C4890ED060A10EE101A084639F078FD41EC1C0B5A
:4087400053EC1B2B39F07CFA41EC1A0B38F032FF08EE900AF5EEC08AF1EE10FA05DD504890ED060AF0EE408A06E04D4890ED060AB1EE400AF0EE408A38EE880AF0EE408ADC
:40878000B5EEC08AF1EE10FA09DDF5EEC08AF1EE10FA04D89FED4C0AF0EE408A0DE0B5EEC08AF1EE10FA08D2F5EEC08AF1EE10FA03DB9FED460AF0EE408A394890ED000A64
:4087C00020EE280A80ED0A0A3B48007870B13448C0ED0C8A90ED0A0AD0ED090A30EE600A80ED0D0A00203449087016E09FED2D0A2B49243101F1200014F098FE2849343157
:40880000A1F1300014F026FDF0EE408A244890ED0C0A30EE280A80ED0C0A214890ED0A0AB5EEC00AF1EE10FA0BDD90ED0C0AB5EEC00AF1EE10FA04D29FED1A0A80ED0C0AAB
:4088400054E0174890ED0A0AB5EEC00AF1EE10FA0BD290ED0C0AB5EEC00AF1EE10FA04DD9FED100A80ED0C0A40E00D4890ED0C0ADFED0E0AB4EEE00AF1EE10FA28DD9FEDBC
:408880000B0A80ED0C0A31E0301F0020A11404086108040850410020C108040809080408041500200000000000007A440000C842540300200000C8C2500300206666264020
:4088C000666626C0DB0FC9400AD7233C0AD723BCF64890ED0C0A5FED090AB4EEE00AF1EE10FA03D21FED0D0A80ED0C0AEF4890ED0C0ABDEC0C8B10BD01B500BF0122694695
:40890000EB480068B03011F031FE20B99DF80000E84981F8B00000BFE748D0F8CC110120DFF898C300DF08BD10B52DED020B00BF04226946DE48006800F5FA7011F016FEB8
:4089400020B99DED000ADB4880ED7D0A00BFDA48D0F8CC110120DFF864C300DF1CBD01B500BF01226946D2480068AE3011F0FEFD20B99DF80000CF4981F8AE0000BFCE48F1
:40898000D0F8CC110120DFF834C300DF08BD01B500BF01226946C6480068AF3011F0E6FD20B99DF80000C34981F8AF0000BFC248D0F8CC110120DFF804C300DF08BD10B5C7
:4089C0002DED020B00BF04226946B948006800F5027011F0CBFD20B99DED000AB54880ED820A00BFB448D0F8CC110120DFF8CCC200DF1CBD10B52DED020B00BF04226946A2
:408A0000AB48006800F5017011F0B0FD20B99DED000AA84880ED810A00BFA748D0F8CC110120DFF898C200DF1CBD10B52DED020B00BF042269469E48006800F5007011F0E1
:408A400095FD20B99DED000A9A4880ED800A00BF9948D0F8CC110120DFF860C200DF1CBD01B500BF0222694691480068AA3011F07DFD20B9BDF800008E49A1F8AA0000BFC2
:408A80008D48D0F8CC110120DFF830C200DF2F2004F0ACFC08BD10B58AB00446022C1FD1B2EE040A8DED090A9FED850A8DED020A1FED840A8DED030A9FED810A8DED040AC0
:408AC0009FED800A8DED060A01208DF820009FED7E0A8DED010AB1EE080A8DED070AA6E0042C1FD1B3EE080A8DED090A1FED910A8DED020A1FED950A8DED030A1FED950A4B
:408B00008DED040A1FED970A8DED060A01208DF820009FED6E0A8DED010AB1EE040A8DED070A84E0052C1FD1B2EE060A8DED090A9FED670A8DED020A1FEDA60A8DED030A67
:408B40009FED630A8DED040A1FEDA80A8DED060A01208DF820009FED5F0A8DED010AB2EE020A8DED070A62E00E2C1FD1B2EE040A8DED090A9FED520A8DED020A1FEDB70AD3
:408B80008DED030A9FED520A8DED040A9FED4D0A8DED060A01208DF820009FED4E0A8DED010AB2EE040A8DED070A40E0152C1FD1B2EE040A8DED090A9FED470A8DED020AFA
:408BC0001FEDC80A8DED030A9FED430A8DED040A9FED3C0A8DED060A01208DF820009FED3A0A8DED010AB1EE080A8DED070A1EE01FEDD40A8DED090A1FEDD60A8DED020A15
:408C00001FEDD80A8DED030A1FEDDA0A8DED040A1FEDDC0A8DED060A00208DF820001FEDDF0A8DED010A1FEDE10A8DED070A9DED090ABDEEC00A10EE101A08B2FFF710FF11
:408C4000DDED020AB0EE600AFFF7EFFEDDED030AB0EE600AFFF7CEFEDDED040AB0EE600AFFF7ADFE9DED060ABCEEC00A10EE101AC8B2FFF78CFE9DF82000FFF770FEDDEDFE
:408C8000010AB0EE600AFFF74FFE9DED070ABCEEC00A10EE101AC8B2FFF72EFE2F2004F0A5FB542004F0A2FB0AB010BD04150020B4030020301F0020504100206108040877
:408CC000000048420000A042F3FDD43CA69B443C0000484396438B3C0000F042204890ED0A0ABDEEC00A10EE100A00B270471C4890ED090ABDEEC00A10EE100A00B2704711
:408D000080220270164A92ED010ADFED160A20EE200ABCEEC00A10EE102A91B241700A0A82700F4A92ED020ADFED0E0A20EE200ABCEEC00A10EE102A91B2C1700A0A0271C4
:408D4000074A92ED030ADFED070A20EE200ABCEEC00A10EE102A91B241710A0A82717047041500200000C84270B5054601249048DFF840C200DF204670BD8F4909780170DD
:408D80008E49416001218160002181764176704700B5A1B06846FFF7F0FF01208DF8180006219DF81920501CC0B28DF819000DF14B00815400208DF81900684601992EF0A8
:408DC0006BFD002021B000BD00B5A1B06846FFF7D4FF02208DF8180005219DF81920501CC0B28DF819000DF14B00815400208DF81900684601992EF04FFD9DF81800401E18
:408E00000DF11B01085C21B000BD2DE9F74F814615464FF000081FFA89F7E8191FFA80FBBBF5005F02DD4FF0080854E02D2D02DD4FF040084FE04FF47A615D48DFF880C1F8
:408E400000DF012802D14FF0100844E0842034F011FA044654B3FFF79BFFFFF7B5FF82462046FFF78AFFE81C20760221627E501C607604F14B008154390A627E501C607638
:408E800004F14B008154627E501C607604F14B008754627E014650182A46019934F0AAFB00206076204661682EF0F6FC94F8800001280BD1FFF788FF06460AF0020010B132
:408EC00006F0020020B14FF0800801E04FF02008204634F00AFA3648DFF8E8C000DFB8F1000F05D03848007840EA0800364908704046BDE8FE8F2DE9F043A1B080460F4615
:408F000014460026BDB260191FFA80F9B9F5005F01DD082642E02D2C01DD40263EE06846FFF72BFFE01CC0B28DF8180003219DF81920501CC0B28DF819000DF14B008154DC
:408F4000290A9DF81920501CC0B28DF819000DF14B0081549DF81920501CC0B28DF819000DF14B0085549DF81920014650185522214602F05BFF00208DF81900684601993D
:408F80002EF08AFC9DF88000012806D122460DF11E01404634F02EFB00E0202626B10A480078304308490870304621B0BDE8F0839C440020350C0408D20600200038004081
:408FC000290D0408450C0408B103002088B0016807914168069181680591C1680491016903914169029181690191C169009108B07047704770477047FFFFFFFFFFFFFFFF4A
:40900000FE4890ED0A0A704710B52DED048BB0EE408A0446F94890ED720ADFEDF90A80EE201AB0EE419AF74890F8AE0058B1FFF7E7FFF0EE409A9FEDF41AF0EE480AFFF786
:40904000B6FAB0EE408AEF4890F89C00012803D1B1EE480AB0EE408A9FEDEC0AB4EEC08AF1EE10FA04D29FEDE90AB0EE408A0AE09FEDE70AB4EEC08AF1EE10FA03DD9FED6B
:40908000E40AB0EE408A20460E2C12D008DCA0F10200052863D2DFE800F00F110E104800122843D013280AD0152803D0182856D106E000BF00BF00BF00BF00BF00BF00BFCA
:4090C000B5EEC08AF1EE10FA0ED2B1EE480AB0EE408A0021CF4800782CF092FB0121CE4800782CF08DFB19E0B5EEC08AF1EE10FA0ADD0121C74800782CF082FB0021C6488D
:4091000000782CF07DFB09E00021C24800782CF077FB0021C04800782CF072FBB0EE480ABE48007830F032FF1AE000BFF0EE000A89EE200A9FEDB61AC8EE010A60EE890AE0
:40914000B1EE001AC0EE811A70EE218ADFEDB40AB0EE680AB34800782CF0CCFB00E000BF00BFBDEC048B10BD70B52DED048B04460D46AD48007848B1012020700121AB48FA
:4091800080F829102EF0B7FEA8490862207830B1012845D0022857D003287ED168E0A34890F8290001280ED1A048016A28462EF0D9FEFA2807D2012020709C4890ED090A8C
:4091C00084ED010A2BE0994890F8350001280ED19648C16A28462EF0C5FEFA2807D202202070924890ED0C0A84ED010A17E08F4890F8410001280ED18C48816B28462EF069
:40920000B1FEFA2807D203202070884890ED0F0A84ED010A03E09FED860A84ED010A3FE0824890F8290030B18048016A28462EF099FEFA2802D90020207004E07B4890EDD2
:40924000090A84ED010A2BE0784890F8350030B17648C16A28462EF085FEFA2802D90020207004E0714890ED0C0A84ED010A17E06E4890F8410030B16C48816B28462EF022
:4092800071FEFA2803D90020207005E005E0674890ED0F0A84ED010A02E00020207000BF00BF94ED020A84ED030A2078F0B394ED050AB5EEC00AF1EE10FA5AD094ED010A14
:4092C00010EE101A084638F0B1FF41EC190BB0EE490AF0EE690A35F083FBB0EE408AF0EE608A9FED540B53EC102B51EC180B38F06BFC3ED894ED010AB5EEC00AF1EE10FA6E
:4093000004D19FED4B0A84ED020A36E094ED010AD4ED050A30EE600AD4ED020AB4EEE00AF1EE10FA0ADD94ED020A00E02EE0D4ED050A30EE200A84ED020A1EE094ED010A3D
:40934000D4ED050A30EE200AD4ED020AB4EEE00AF1EE10FA08D294ED020AD4ED050A30EE600A84ED020A08E094ED010A84ED020A03E094ED010A84ED020A94ED020A84ED7C
:40938000040A0120294981F8480013E09FED280A84ED020A9FED260A84ED010A9FED240A84ED030A9FED220A84ED040A00201F4981F8480094ED040A1C4880ED110ABDEC09
:4093C000048B70BD10B52DED088B044603F074FFB0EE408A94ED090AD4ED0B0A30EE200AF0EE000A80EE201AF0EE418A94ED080AD4ED0A0A30EE200A20E0000080080020E4
:4094000000007A44301F00206F12833A0000C8C20000C842C5060020C60600202307002003005841EB0600202D000020D4070020000000000000000000005940F0EE000A96
:4094400080EE201AB0EE419A94ED020AB4EEE80AF1EE10FA2BDD94F8440002281DD1B2EE040A03F021F8A0B994ED120A38EE400AF0EE040AB4EEE00AF1EE10FA09D24FF432
:409480007A71E06C2EF03DFD30B101215020015502E000215020015508E0022084F8440084ED128A2EF027FDE06400BF56E094ED020AB4EEC90AF1EE10FA2BD294F8440081
:4094C00001281DD1B2EE040A02F0AAFFA0B994ED120A38EE400AF8EE040AB4EEE00AF1EE10FA09DD4FF47A71E06C2EF00AFD30B101215020015502E000215020015508E03E
:40950000012084F8440084ED128A2EF0F4FCE06400BF23E0002084F8440094ED120A30EE480A10EE101A084638F080FE41EC1B0BB0EE4B0AF0EE6B0A35F052FAB0EE40AA8E
:40954000F0EE60AA9FEDF70B53EC102B51EC1A0B38F074FC02D2002150200155BDEC088B10BD70B52DED0C8B04460D4694ED0A0AF2EE040AB4EEE00AF1EE10FA0CD294ED73
:409580000A0AFAEE040AB4EEE00AF1EE10FA03DD1FED590A84ED0A0A94ED0A0A5FED680AC0EE208A95ED020AD5ED080AB4EEE00AF1EE10FA18D895ED0C0AD5ED020A20EE72
:4095C000200A1FED6D1AC0EE010A94ED780A20EE800A1FED751AC0EE010A95ED0D0A30EEC00A84ED620A25E095ED020AD5ED090AB4EEE00AF1EE10FA18DB95ED0C0AD5ED7E
:40960000020A60EE200A1FED7E1A80EE810AD4ED780A60EE200A1FED861A80EE810AD5ED0D0A30EE200A84ED620A03E01FED800A84ED620A95ED020AB5EEC00AF1EE10FA71
:4096400002D11FED918A18E094ED620A10EE101A084638F0EBFD41EC1B0BB0EE4B0AF0EE6B0A35F0BDF9B0EE40AAF0EE60AA51EC1A0B37F09FFF08EE100A94ED620A10EE7F
:40968000101A084638F0D2FD41EC1D0BB0EE4D0AF0EE6D0A35F0A4F9B0EE40BAF0EE60BA18EE900A38F0C2FD41EC1D0BB0EE4D0AF0EE6D0A35F094F9B0EE40CAF0EE60CAC2
:4096C00053EC1B2B51EC1C0B38F0C6FC41EC1A0B37F070FF09EE100A89EE080AB0EE409A1E219248B0EE490A1CF0C0FCBDEC0C8B70BD2DE9F0412DED028B04460D468C48FF
:4097000090F8BD010A287DD14FF432700159001D0151001FD4F8C41201518648007830F090FBC4F8C4024FF432700059D4F8C412081A00EE100AB8EEC00ADFED7F0A80EEF2
:40974000201A84EDB41A94EDB40AB2EE041AC0EE010A9FED7A0A20EE800A84EDC40A95ED020AD5ED080AB4EEE00AF1EE10FA23D895ED0E0AD5ED020A20EE200A1FEDDC1A5F
:40978000C0EE010A94ED780A20EE800A1FEDE41AC0EE010A95ED0F0A30EEC00A84EDDA0A94EDDA0AB5EEC00AF1EE10FA37DD1FEDE00A84EDDA0A32E095ED020AD5ED090A2B
:4097C000B4EEE00AF1EE10FA25DB95ED0E0AD5ED020A20EE200A1FEDF21AC0EE010A94ED780A20EE800A1FEDFA1AC0EE010A95ED0F0A30EE800A84EDDA0A94EDDA0AB5EE6F
:40980000C00A00E07DE0F1EE10FA08D21FEDF80A84EDDA0A03E01FEDFA0A84EDDA0A444890F830000A2803D132274FF0480802E032274FF04108D4EDC40AB0EE600A3946A8
:4098400004F53E701CF012FCD4EDDA0AB0EE600A414604F554701CF009FC94EDD40AD4EDBE0A30EE600AF2EE040A20EE208A9FED340AB4EEC08AF1EE10FA04DD9FED300AC9
:40988000B0EE408A0AE09FED2F0AB4EEC08AF1EE10FA03D29FED2B0AB0EE408A012104F53970B0EE480A1CF0E1FB94EDD40A84EDDD0A94EDBE0A84EDC70A04261AE0711E2D
:4098C00004F55D7000EB810090ED000A04F55D7000EB860080ED000A04F5477000EB810090ED000A04F5477000EB860080ED000A701EC6B2002EE2DC94EDB90A124880EDC9
:40990000150ABDEC028BBDE8F081094991F84A10062904D0064991F84A10122916D1012015E00000000000000000F83FC0070020301F0020E80600208DED244800606A4788
:4099400000007A4400007AC4D40700200020704710B52DED020B00BF04226946FE48006800F5587010F002FE20B99DED000AFB4880EDD80A00BF1CBD10B52DED020B00BFEC
:4099800004226946F448006800F5577010F0EEFD20B99DED000AF14880EDD70A00BF1CBD10B52DED020B00BF04226946EA48006800F5567010F0DAFD20B99DED000AE748B3
:4099C00080EDD60A00BF1CBD10B52DED020B00BF04226946E048006800F5557010F0C6FD20B99DED000ADD4880EDD50A00BF1CBDDA4991F84A10032901D1012000E000205A
:409A0000704710B52DED020B00BF04226946D248006800F55C7010F0A9FD20B99DED000ACE4880EDDC0A00BF1CBD10B52DED020B00BF04226946C848006800F55B7010F0E0
:409A400095FD20B99DED000AC44880EDDB0A00BF1CBD10B52DED020B00BF04226946BE48006800F55A7010F081FD20B99DED000ABA4880EDDA0A00BF1CBD10B52DED020B82
:409A800000BF04226946B448006800F5597010F06DFD20B99DED000AB04880EDD90A00BF1CBDAE4991F84A1004291DD0AB4991F84A10022918D0A94991F84A10052913D075
:409AC000A64991F84A100E290ED0A44991F84A10152909D0A14991F84A10132904D09F4991F84A10182901D1012000E00020704710B52DED028B84B00446FFF779FF10B1EC
:409B0000B2EE048A01E0B7EE008A944890ED280A20EE080A84ED000AB0F8A80000EE100AB8EE400A84ED020A9FED8D0A84ED010A8A4890F89C0084F82C00884890F8421015
:409B40006C3000EB810090ED000A84ED030A834890F84210743000EB810090ED000A84ED040A7E4890F842107C3000EB810090ED000A84ED050A794890F84210843000EB24
:409B8000810090ED000A84ED060A744890ED700A84ED070A90ED710A84ED080A90ED720A84ED090A90ED730A84ED0A0A2BF0FEFD002876D0FFF7A9FE78B3012169480078D9
:409BC0002BF01EFE0021684800782BF019FE0021664800782BF014FEB2EE040AFFF7F4FE9FED630AFFF7DCFEB7EE000AFFF7C4FE9FED5B0AFFF7ACFE9FED5E0AFFF73DFFC2
:409C00009FED5D0AFFF725FF9FED5C0AFFF70DFF1FEDB50AFFF7F5FE95E0FFE7FFF741FFF0B35748009094ED020AF0EE400A9FED550A01231A465449544800782FF008FE12
:409C40000021484800782BF0DBFD0121464800782BF0D6FD0121454800782BF0D1FD9FED4C0AFFF7B1FE9FED440AFFF799FE9FED430AFFF781FE1FEDCE0AFFF769FE9FED99
:409C8000450AFFF7FAFE9FED3C0AFFF7E2FE9FED3B0AFFF7CAFE1FEDD60AFFF7B2FE52E000E041E0FFF7A4FE70B33548009094ED020AF0EE400A9FED330A01231A46324926
:409CC000324800782FF0C4FD0021264800782BF097FD0121244800782BF092FD0121234800782BF08DFD9FED2A0AFFF76DFE9FED220AFFF755FE9FED210AFFF73DFE1FED6C
:409D0000F00AFFF725FE1EE00021164800782BF077FD0121144800782BF072FD0121134800782BF06DFD0EE01548009094ED020AF0EE400A9FED130A012300221649134859
:409D400000782FF085FD94F82C0038BB0020009001900290034622E0B4030020301F0020000000000007002021070020200700206F12833A00401C45000048420000FA435F
:409D8000C8D80020A037A04B001800402307002000004845008054450000014011E00322FE49039055202BF002FE002000900190029003460322FA49039056202BF0F7FD7C
:409DC00015E0002000900190029003460322F449039055202BF0EBFD002000900190029003460322ED49039056202BF0E0FD012004B0BDEC028B10BD2DED028B5421E94848
:409E000033F091FC4FF46771E74833F08CFC5821E64833F088FCE348E5490860E3484830E4490860E048E449086000F5F070E3490860A0F5DC70E249086000F5B070E149DD
:409E4000086000F59E70E04908604C30DF490860D6485430DE490860DE48DF490860D1481430DE4908609FEDDE0A143880ED030A9FEDDB0ACD4880ED130A9FEDDA0A80EDE0
:409E8000140AFFF7B5FD40B1DFF85CC300DF06460A2202212EF039F90AE02BF087FC38B1DFF844C300DF0646012202212EF02DF9DFF834C300DF064602212EF055F9DFF8C8
:409EC00028C300DF064631460120DFF820C300DF0321C74880F8541000BF00224FF6FF710320DFF810C300DF044604F001000028F3D104F002000028EFD0DFF8FCC200DF4E
:409F0000054605F0010030B1A6481430FFF7F0FD182025F0AFFD05F002000028DDD0B748007818F0E1F9A04880ED780AD0ED780AB0EE600A142100F5E4701CF097F82BF07A
:409F40001DFC78B1AE48007818F08BFB964880ED0A0AD0ED0A0AB0EE600A1E2110301CF085F887E02BF022FC002823D0FFF7CDFC08B3A448007818F074FB8B4880ED8E0A7B
:409F8000A148007818F0B0F9874880EDA40AD0EDA40AB0EE600A142100F51E701CF066F88148D0ED8E0AB0EE600A142100F508701CF05CF85EE09248007818F052FB7A4841
:409FC00080ED0A0AD0ED0A0AB0EE600A1E2110301CF04CF8744890ED0A0AD0ED040A30EE600A20EE000AB0EE408A1E212030B0EE480A1CF03BF88548007818F032FB6A482E
:40A0000080ED200AD0ED200AB0EE600A1E2168301CF02CF8644890ED200AD0ED1A0A30EE600A20EE000AB0EE408A1E217830B0EE480A1CF01BF85948007818F012FB5A4891
:40A0400080ED360AD0ED360AB0EE600A1E21C0301CF00CF85248007818F003FB524880ED4C0AD0ED4C0AB0EE600A1E2100F58C701BF0FCFF4B494C48FFF73BFB49494A48B1
:40A08000FFF76FFA4748FFF79DF92DF034FF064631464448FFF768F84248007818B1434890F84800F0BB2BF069FB90B11FEDD40A3C4880ED020A00203B49087000215448E0
:40A0C00000782BF09DFB0021524800782BF098FBB2E02BF06BFB002827D01FEDDF0A314880ED020A0020304908700021494800782BF086FB0021464800782BF081FB002185
:40A10000454800782BF07CFB0021444800782BF077FB0021424800782BF072FB00214148007800E002E02BF06BFB85E01F4890F84800012830D11C48007868BB2BF01EFBCD
:40A1400068B10120184908700121324800782BF057FB01212E4800782BF052FB6CE02BF025FBC8B10120104908700121294800782BF046FB0121264800782BF041FB0121F9
:40A18000254800782BF03CFB0121244800782BF037FB0121224847E04EE0000035070020360700202C08002080080020D40700200000002004000020080000200C000020EC
:40A1C000100000201400002018000020200000201C000020E80B002024000020280000200000C8420000C8C2A11404086108040850410020C108040809080408A306002072
:40A20000F4060020EC060020F1060020F70600200507002006070020040700201C070020240700200707002000782BF0E9FA0121FD4800782BF0E4FAFC4991F84A00FC49D3
:40A24000D1ED020AB0EE600AFEF7DEFE45E601B50DF0CAFA70B900BF01226946F54800689C3010F083F920B99DF80000EF4981F89C0000BFF048016D0120DFF8C0C300DF78
:40A28000132003F0B3F808BD10B52DED020B00249DED000AF2EE040AB4EEE00AF1EE10FA05DDB2EE040A8DED000A02240BE09DED000AB5EEC00AF1EE10FA04D29FEDE00AA6
:40A2C0008DED000A032400BF04226946D9480068A03010F04BF920B99DED000AD34880ED280A00BFD448016D0120DFF850C300DF182003F07BF820461CBD01B500BF0222B2
:40A300006946CC480068A83010F030F920B9BDF80000C649A1F8A80000BFC748016D0120DFF818C300DF08BD10B5FFF761FB58B144F62060FFF7E1FFB6EE000AFFF7A4FF69
:40A340000020FFF784FF1BE0FFF7DFFA50B12820FFF7D3FF9FEDBA0AFFF796FF0020FFF776FF0DE0FFF79DFB50B144F62060FFF7C4FF9FEDB30AFFF787FF0020FFF767FFD3
:40A38000AA4991F84A00FEF786FB012010BD70B52DED028BB0EE408A04460D460026012C04D0022C03D0032C4AD101E000BF00BFA44890ED140AB4EEC80AF1EE10FA05DD0B
:40A3C00090ED140AB0EE408A03260CE09D4890ED130AB4EEC80AF1EE10FA04D290ED130AB0EE408A022610219648DFF85CC200DF012823D004EB44019248143000EB8100AC
:40A4000080ED018A2DF077FD04EB44028D49143141F82200012104EB44028A48143000EB8200017204EB44018648143000EB810045728448DFF814C200DF00E0062601E0ED
:40A44000062600BF00BF3046BDEC028B70BD7D4890ED110A7047764890F85000012800D170470020FCE7774890ED150A70470020744991F84810012904D1754909780129C3
:40A4800000D10120704701B500BF01226946694800684A3010F06AF820B99DF80000634981F84A0000BFFFF73FFF6348016D0120DFF888C100DF262002F098FF08BD64486E
:40A4C00090ED780A7047624890ED8E0A7047604890ED040A70475E4890ED1A0A70475C4890ED080A70475A4890ED300A7047584890ED460A704700B5FFF77AFA30B155488D
:40A50000007808B1012000BD0020FCE70020FAE7002070474F480078022804D14E48007D012800D170470020FCE710B5FFF7EDF930B14A4800782BF065FD08B1012010BDAC
:40A540000020FCE7394890F84A00182801D1012070470020FCE700B50121FFF7F3FF00B900E00021084600BD70B52DED068B0024FFF77DFF80B32BF035F968B3FFF7EBFF37
:40A5800050B3FFF78EFA38B3284890EDD50A10EE101A084637F04AFE41EC180BFEF730FD10EE105A284637F041FE41EC1A0BB0EE4A0AF0EE6A0A34F013FAB0EE409AF0EEB3
:40A5C000609A53EC182B51EC190B37F037FC01D2012000E0002004462046BDEC068B70BD0020134991ED020A104991F84220743101EB8201D1ED000AB4EEE00AF1EE10FA7E
:40A6000010DB0B4991ED020A084991F84220843101EB8201D1ED000AB4EEE00AF1EE10FA00D801207047000007070020301F00202C080020B4030020504100206108040816
:40A6400000000000D4070020290D0408450C0408800800202C000020A0290020280700200020FE4991ED020AFD4991F842206C3101EB8201D1ED000AB4EEE00AF1EE10FAA9
:40A6800010D8F64991ED020AF54991F842207C3101EB8201D1ED000AB4EEE00AF1EE10FA00DB0120704700B50023FFF7D9FF10B9FFF796FF00B10123184600BD70B52DED8B
:40A6C000068B0024FFF7D3FE88B32BF08BF870B3FFF7E9FF58B3FFF73EFF40B3FFF7E1F928B3DF4890EDD60A10EE101A084637F09DFD41EC180BFEF783FC10EE105A2846D3
:40A7000037F094FD41EC1A0BB0EE4A0AF0EE6A0A34F066F9B0EE409AF0EE609A53EC182B51EC190B37F050FA02D2012001E001E0002004462046BDEC068B70BD70B52DED77
:40A74000068B0024FFF793FE80BB2BF04BF868B3FFF701FF50B3FFF7A4F938B3C04890EDD70A10EE101A084637F060FD41EC180BFEF746FC10EE105A284637F057FD41EC0D
:40A780001A0BB0EE4A0AF0EE6A0A34F029F9B0EE409AF0EE609A53EC182B51EC190B37F04DFB01D2012000E0002004462046BDEC068B70BD70B52DED068B0024FFF771F9E9
:40A7C00080B3FFF754FE68B32BF00CF850B3FFF7C2FE38B3A24890EDD50A10EE101A084637F024FD41EC180BFFF77DFE10EE105A284637F01BFD41EC1A0BB0EE4A0AF0EE04
:40A800006A0A34F0EDF8B0EE409AF0EE609A53EC182B51EC190B37F011FB01D2012000E0002004462046BDEC068B70BD70B52DED068B0024FFF735F988B3FFF718FE70B3A8
:40A84000FFF70EFF58B32AF0CDFF40B3FFF783FE28B3834890EDD60A10EE101A084637F0E5FC41EC180BFFF73EFE10EE105A284637F0DCFC41EC1A0BB0EE4A0AF0EE6A0A0C
:40A8800034F0AEF8B0EE409AF0EE609A53EC182B51EC190B37F098F902D2012001E001E0002004462046BDEC068B70BD70B52DED068B0024FFF7F5F880B3FFF7D8FD68BBFD
:40A8C0002AF090FF50B3FFF746FE38B3644890EDD70A10EE101A084637F0A8FC41EC180BFFF701FE10EE105A284637F09FFC41EC1A0BB0EE4A0AF0EE6A0A34F071F8B0EE9E
:40A90000409AF0EE609A53EC182B51EC190B37F095FA01D2012000E0002004462046BDEC068B70BD70B52DED068B0024FFF7B9F880B3FFF79CFD68B32AF054FF50B3FFF7E3
:40A940000AFE38B3464890EDD50A10EE101A084637F06CFC41EC180BFFF7C9FD10EE105A284637F063FC41EC1A0BB0EE4A0AF0EE6A0A34F035F8B0EE409AF0EE609A53EC17
:40A98000182B51EC190B37F059FA01D2012000E0002004462046BDEC068B70BD70B52DED068B0024FFF77DF888B3FFF760FD70B3FFF716FE58B32AF015FF40B3FFF7CBFD6A
:40A9C00028B3274890EDD60A10EE101A084637F02DFC41EC180BFFF78AFD10EE105A284637F024FC41EC1A0BB0EE4A0AF0EE6A0A33F0F6FFB0EE409AF0EE609A53EC182B80
:40AA000051EC190B37F0E0F802D2012001E001E0002004462046BDEC068B70BD70B52DED068B0024FFF73DF898B3FFF720FD80BB2AF0D8FE68B3FFF78EFD50B3084890EDB4
:40AA4000D70A10EE101A084637F0F0FB41EC180BFFF74DFD10EE105A284603E02C080020301F002037F0E2FB41EC1A0BB0EE4A0AF0EE6A0A33F0B4FFB0EE409AF0EE609AA1
:40AA800053EC182B51EC190B37F0D8F902D2012001E001E0002004462046BDEC068B70BD70B52DED088B0024FEF7FBFFB8B32AF099FEA0B3FFF74FFD88B3FFF714FDF0EE17
:40AAC000400AFFF714FD30EE800AB0EE408AF44890EDD80A10EE101A084637F0A7FB41EC190BFFF7F4FC30EE480A10EE105A284637F09CFB41EC1B0BB0EE4B0AF0EE6B0A47
:40AB000033F06EFFB0EE40AAF0EE60AA53EC192B51EC1A0B37F092F902D2012001E002E00020044600BF2046BDEC088B70BDDD4890ED030A704710B50124D94890F84A008B
:40AB40000E2816D0D64890F84A00022811D0D44890F84A0015280CD0D14890F84A00032802D12AF023FE20B9CD4890F84A00182800D100240CB1012010BD0020FCE710B52B
:40AB80000024FFF774FCB0B12AF02CFE98B1FFF7D2FF80B1FFF7DFFC68B1FFF7C8FFC048D0EDD90AB4EEE00AF1EE10FA01DD012000E000200446204610BD10B50024FFF706
:40ABC00056FCB0B12AF00EFE98B1FFF7B4FF80B1FFF7ADFFB248D0EDDA0AB4EEE00AF1EE10FA04D2FFF7B7FC08B1012000E000200446204610BD10B50024FFF738FCB0B955
:40AC00002AF0F0FD98B1FFF796FF80B1FFF78FFFA348D0EDDB0AB4EEE00AF1EE10FA04DDFFF799FC08B1012000E000200446204610BD9D4890ED030A704710B50024FFF7BA
:40AC400016FCB0B12AF0CEFD98B1FFF774FF80B1FFF781FC68B1FFF7ECFF9148D0EDD90AB4EEE00AF1EE10FA01DD012000E000200446204610BD10B50024FFF7F8FBB0B18F
:40AC80002AF0B0FD98B1FFF756FF80B1FFF763FC68B1FFF7CEFF8248D0EDDA0AB4EEE00AF1EE10FA01D2012000E000200446204610BD10B50024FFF7DAFBB0B92AF092FDC0
:40ACC00098B1FFF738FF80B1FFF745FC68B1FFF7B0FF7348D0EDDB0AB4EEE00AF1EE10FA01DD012000E000200446204610BD70B52DED068B00242AF075FD88B3FFF71BFF9F
:40AD000070B3FFF728FC58B3654890EDDC0A10EE101A084637F08AFA41EC180BFFF707FFF0EE400AFFF785FF30EEC00A10EE105A284637F07BFA41EC1A0BB0EE4A0AF0EE30
:40AD40006A0A33F04DFEB0EE409AF0EE609A53EC182B51EC190B37F071F802D2012001E001E0002004462046BDEC068B70BD10B52DED028B9FED4D0AB0EE408A2AF0FEFC75
:40AD800028B14B4890ED030AB0EE408A11E02AF00DFD70B1FFF7CBFEB0EE408AB3EE040AB4EEC08AF1EE10FA03D89FED400AB0EE408AB0EE480ABDEC028B10BD3D4890ED46
:40ADC000A40A704710B52DED068BFEF79EFD20B1FFF7ADFEB0EE408A0CE0314890F84A00032803D1344890ED038A03E0FFF76FFBB0EE408A18EE100A37F018FA41EC1A0B02
:40AE0000B0EE4A0AF0EE6A0A33F0EAFDB0EE409AF0EE609A9FED290B53EC102B51EC190B36F0D2FE03D89FED210AB0EE408AB0EE480ABDEC068B10BD00B50022FFF717FB13
:40AE400090B1FEF762FD78B1FFF7B8FFF0EE400AFFF735FB9FED1B1A20EE010AF4EEC00AF1EE10FA00DD0122104600BD00B50022FFF7FDFA90B1FEF748FD78B1FFF79EFF9C
:40AE8000F0EE400AFFF71BFB9FED0F1A20EE010AF4EEC00AF1EE10FA00D20122104600BD301F00201C0C0020740C002000000000CC0C002080080020240D002000000000AB
:40AEC000000034406666663FCDCCCC3D10B501F088FF282002F08AFA292002F087FA00F043FE70B1DFF8D0C300DF044604212DF03BF9DFF8C4C300DF044602212DF034F9C5
:40AF00000DE0DFF8B4C300DF044604212DF049F9DFF8A4C300DF044602212DF042F910BD10B5E648C16B01202DF058F9E348C16B0120DFF88CC300DF10BD10B52DED0C8B0C
:40AF4000B0EE408ADF4890ED630AB0EE409AB4EEC98AF1EE10FA02DD01F02DFF38B9B4EEC98AF1EE10FA2CD201F025FF48BBD54890ED6A0A10EE101A084637F057F941ECF9
:40AF80001B0B38EE490A10EE101A084637F04EF941EC1D0BB0EE4D0AF0EE6D0A33F020FDB0EE40CAF0EE60CA53EC1B2B51EC1C0B36F046FE41EC1A0B36F0FCFA08EE900A2E
:40AFC0003BE0B4EEC98AF1EE10FA02DD01F0F3FE38B1B4EEC98AF1EE10FA2CD201F0EBFE48B3B84890ED6B0A10EE101A084637F01DF941EC1B0B38EE490A10EE101A084616
:40B0000037F014F941EC1D0BB0EE4D0AF0EE6D0A33F0E6FCB0EE40CAF0EE60CA53EC1B2B51EC1C0B36F00CFE41EC1A0B36F0C2FA08EE900A01E0DFEDA48A9FEDA40AF4EEB4
:40B04000C08AF1EE10FA03DD9FEDA00AF0EE408A9FED9F0AF4EEC08AF1EE10FA03D29FED9C0AF0EE408AB0EE680ABDEC0C8B10BD10B52DED028B2CF03EFF9649086000209D
:40B0800001F0A1F9B0EE408AFFF757FF914880ED030A01F07FFBBDEC028B10BD28218D4832F041FB0121854880F82012DFF808C200DF0646012204212DF027F8DFF8F8C19B
:40B0C00000DF0646192202212DF01FF8DFF8E8C100DF064631460120DFF8E4C100DF0321764880F8201200BF00224FF6FF710720DFF8E4C100DF85B2012DF5D0022DF3D134
:40B10000DFF8D8C100DF044604F0040008B101F02FFC04F0020018B1FFF7AAFFFFF700FF04F001000028DFD0FFF7D0FEDCE710B504466248D0F81C122046DFF884C100DFF3
:40B1400010BD10B52DED088B5E4890ED630AD0ED610A30EE600ADFED5E0A80EE801A11EE104A204637F062F841EC1B0BB0EE4B0AF0EE6B0A33F034FCB0EE40AAF0EE60AA78
:40B1800051EC1A0B36F00AFA41EC190B36F012FA08EE900A4B4890ED620AD0ED630A30EE600ADFED4A0A80EE801A11EE104A204637F03CF841EC1A0BB0EE4A0AF0EE6A0AEA
:40B1C00033F00EFCB0EE409AF0EE609A51EC190B36F0F0F908EE100A002001F0C1FA394890F830000A280CD1364890F8B201032807D19FED3B0AB0EE408AB1EE480AF0EE7A
:40B20000408AB0EE680A01F021FBB0EE480A01F031FBBDEC088B10BD70B505460C4601F048FA284600F0ECFE204600F001FFFFF788FF642016F024F80120FFF778FF70BDA0
:40B240002448D0ED030AB0EE600A7047214890F82400032801D0012070470020FCE70220704710B52DED088BB0EE408A18EE100A36F0DCFF41EC190BFFF7E2FF10EE104A99
:40B28000204636F0D3FF41EC1B0BB0EE4B0AF0EE6B0A33F0A5FBB0EE40AAF0EE60AA53EC192B51EC1A0B36F08FFC03D20120BDEC088B10BD0020FAE7A1140408504100205C
:40B2C00061080408301F0020000000000000C8420000C8C2EC1A0020C108040809080408D051863910B5044600BF28222146FD4800680FF03BF920B928222146FA4832F091
:40B3000079F900BF10BD10B504462822F649204632F070F910BD01B500BF04226946F148006828300FF022F918B99DF80000EE49886200BFED48C16B0220DFF8B4C300DF66
:40B3400008BD01B500BF04226946E64800682C300FF00CF918B99DF80000E349C86200BF08BD01B500BF04226946DE48006830300FF0FCF810B9DC490098086300BF08BDE8
:40B3800010B52DED020B00BF04226946D54800683C300FF0EBF820B99DED000AD24880ED0F0A00BF10F0E8F9D048C16B0220DFF840C300DF022002F019F84F2002F016F8DA
:40B3C0001CBD01B500BF01226946C648006848300FF0CCF820B99DF80000C34981F8480000BF08BD08B5002000902AF0DFF9A0B10021C04800782AF003FABF4800782AF0BC
:40B4000001FE28B10220FFF7DCFF0120009004E00120FFF7D6FF0220009000BF01226946B048006849300FF0A1F820B99DF80000AD4981F8490000BFAC48016D0120DFF8CD
:40B44000B0C200DF08BD01B500BF04226946A548006844300FF08AF810B9A3490098486400BF08BD01B5A04890F841009DF80010884215D000BF012269469A48006841309E
:40B480000FF074F820B99DF80000974981F8410000BF25F018FD13F007FF1E2001F0A6FF08BD01B500BF012269468E48006842300FF05CF820B99DF800008B4981F8420047
:40B4C00000BF25F000FD252001F090FF8748C16B0220DFF81CC200DF13F0E6FE08BD01B500BF0422694685480068AC300FF03EF818B97D480099C0F89C1400BF08BD8048E6
:40B50000006870477E490860704770B52DED028B04460D4616462AF031F9F8B17249E0314A5D891C495D501800EBD071491000EE101AB8EEC00AB0EE408ABCEEC80A10EE3F
:40B54000101AC8B2294613F0E8FABCEEC80A10EE101AC8B2294613F013FB0EE02AF026F958B16149E031485D294613F0D6FA5E49E231485D294613F003FB624800EB84007B
:40B58000D0ED000AB0EE600A2946204613F0B9F95C490831085D2A46214613F004FA59490A31085D2A46214613F03BFA55490C31085D2A46214613F072FA46B1182024F0FD
:40B5C00059FA4A48016D0120DFF824C100DFBDEC028B70BD70B500240CE0002506E0002229462046FFF791FF681CC5B2022DF6DB601CC4B2022CF0DB182024F03BFA3B4832
:40B60000016D0120DFF8E8C000DF70BD70B52DED028B04460D462AF0B1F800B33248D03000EB840090ED000AB1EE400A2E48D83000EB8400D0ED000A30EE200AF0EE000AD4
:40B6400080EE201AB0EE418A2046B1EE480A13F093FB2046B0EE480A13F0E9FB18E02AF0A5F8A8B12048D03000EB8400D0ED000AB0EE600A204613F07FFB1B48D83000EBAD
:40B680008400D0ED000AB0EE600A204613F0CFFB1548C03000EB8400D0ED000AB0EE600A204613F0B5FA1048C83000EB8400D0ED000AB0EE600A204613F005FB75B1142010
:40B6C00024F0D8F9182024F0D5F9142024F0D2F90648016D0120DFF818C000DFBDEC028B70BD0000B4030020301F002050410020610804080707002027070020B8030020A7
:40B70000A00300201421002010B5002405E000212046FFF77BFF601CC4B2022CF7DB142024F0A8F9182024F0A5F9142024F0A2F9F948016D0120DFF8E4C300DF10BD70B565
:40B7400005460C4600212046FFF760FF002221462846FFF7DAFE70BD70B52DED028B05460024B5E0EE4890F84900C0EB001105F1380000EB81000E3030F9140000EE900A2E
:40B78000F8EEE00AB0EE600A204613F015FCE44890F84900C0EB001105F1380000EB8100123030F9140000EE900AF8EEE00AB0EE600A204613F034FCD94890F84900C0EBCF
:40B7C000001105F1380000EB8100163030F9140000EE900AF8EEE00AB0EE600A204613F043FCCF4890F84900C0EB001105F1380000EB81001A3030F9140000EE900AF8EEE0
:40B80000E00AB0EE600A204613F053FCC44991F84910C1EB011205F1380101EB82010931085D214613F06AFCBD4991F84910C1EB011205F1380101EB82010B31085D214656
:40B8400013F07BFCB64890F84900C0EB001105F1380000EB8100401C005D00EE100AB8EE400ADFEDB00A80EE201AB0EE418A2046B0EE480A13F080FCA94991F84910C1EB8C
:40B88000011205F1380101EB8201C91C085D214613F08BFCA24991F84910C1EB011205F1380101EB8201491D085D214613F091FC9B4991F84910C1EB011205F1380101EB10
:40B8C0008201C91D085D214613F097FC601CC4B2022CFFF647AF924890F84900C0EB001105F1380000EB8100D0ED080AB0EE600A13F026FBBDEC028B70BD894890F8280092
:40B9000008B9012070470020FCE710B5012026F071FB0146844880F83910002026F06AFB81494874012026F065FB0446214601201DF075FE002026F05DFB044621460020C6
:40B940001DF06DFE10BD01460020282901D1012200E00022402901D1012300E000231A43492901D1012300E000231A434A2901D1012300E000231A434B2901D1012300E039
:40B9800000231A4302B10120704701460020562901D0782900D10120704701460020592900D10120704701460020712900D10120704710B500245A4890F830000A2803D1F6
:40B9C00029F0F4FE00B10124204610BD544890F82810082905D0092903D00A2901D00E2901D1012070470020FCE74D4890F828100A2901D1012070470020FCE7484890F897
:40BA00002810082901D1012070470020FCE7444890F82810092901D1012070470020FCE73F4890F828100E2901D1012070470020FCE710B5044629F0B9FE70B129F0C9FEBA
:40BA400000B92CB901213948007829F0D9FE04E000213648007829F0D3FE10BD304890F8300000EB401101EB8010314901EB8000408E70470246012109E001EB01102D4B50
:40BA800013F81000904201D1C8B27047491C1A29F3DB0020F9E7224890ED0F0A7047204890F84900022801D1012070470020FCE71B4890F84900012800D170470020FCE771
:40BAC000174890F8490008B9012070470020FCE710B50024FFF7F4FF08B1012419E029F065FEB0B1FFF7E4FF20B1134800782AF089FA68B9FFF7D3FF58B1FEF7B8FC38B94E
:40BB0000FEF7B5FC28B90C4800782AF07BFA00B90124204610BD00005041002061080408301F00200000C84200CE00200207002044350408D031040827070020524890F85A
:40BB4000970020B1504890F89700012801D1012070470020FCE74C4890F82800072801D1012070470020FCE7474890F89700022804D0454890F89700032801D10120704783
:40BB80000020FCE7404890F89700032801D1012070470020FCE73C4890F89700022801D1012070470020FCE7374890F8970008B9012070470020FCE7334890F8970001288C
:40BBC00000D170470020FCE72F4890F89700042801D1012070470020FCE72B4890F89700042801D1012070470020FCE701B500BF012269462548006897300EF0B7FC20B973
:40BC00009DF80000204981F8970000BF08BD01B500BF012269461D48006800F285300EF0A5FC20B99DF80000174981F8850300BF08BD10B50024144890F8300028281DD08B
:40BC4000114890F83000402818D00F4890F83000492813D00C4890F830004A280ED00A4890F830004B2809D0074890F83000592804D0054890F830005C2800D1012420460D
:40BC8000FFF7C5FF204610BD301F0020B40300203EB504460020029064200223464AD421009020462BF0C4F864200223434AD421009020462BF0BCF864200223404AD4214F
:40BCC000009020462BF0B4F8642002233D4AD421009020462BF0ACF8642002233A4AD421009020462BF0A4F864200223374AD421009020462BF09CF80420012102AB0F22F6
:40BD0000CDE90010D42120462BF09AFA9DF80800D72801D101203EBD0020FCE72DE9FF4107460C4615461E464FF000080420062102ABA822CDE90010D42138462BF080FA1B
:40BD40000E2836D19DF808009DF8091040EA012000B200EE100AB8EEC00ADFED1D0A20EE200A84ED000A9DF80A009DF80B1040EA012000B200EE100AB8EEC00ADFED140A72
:40BD800020EE200A85ED000A9DF80C009DF80D1040EA012000B200EE100AB8EEC00ADFED0C0A20EE200A86ED000A012004B0BDE8F0814046FAE70000480500204A05002042
:40BDC0004C0500204E0500205005002052050020F9FFF43B0C48016841F4700101600B4880470B480047FEE7FEE7FEE7FEE7FEE7FEE7FEE7FEE7FEE7FEE700000548064946
:40BE0000064A074B7047000088ED00E035C90308AD810008C0E60020C0EC0020C0E80020C0E80020004870477CE5002002F0FF0343EA032242EA024231F055BC000000008B
:40BE40000000000000000000000000000000000000000000000000000000000000000000000000000000000000000000526176656E20496E647573747269657320496E6342
:40BE80000000000000000000000000004175672D31382D323031380000000000322E362E312E320000000000000000005374656572696E6720436F6E74726F6C20556E69F4
:40BEC0007400000000000000000000003037373031373135323100000000000000000000000000000000000000000000FFFFFFFFFFFFFFFFFFFFFFFFFFFFFFFFFFFFFFFFE3
:40BF0000FFFFFFFFFFFFFFFFFFFFFFFFFFFFFFFFFFFFFFFFFFFFFFFFFFFFFFFFFFFFFFFFFFFFFFFFFFFFFFFFFFFFFFFFFFFFFFFFFFFFFFFFFFFFFFFFFFFFFFFFFFFFFFFF41
:40BF4000FFFFFFFFFFFFFFFFFFFFFFFFFFFFFFFFFFFFFFFFFFFFFFFFFFFFFFFFFFFFFFFFFFFFFFFFFFFFFFFFFFFFFFFFFFFFFFFFFFFFFFFFFFFFFFFFFFFFFFFFFFFFFFFF01
:40BF8000FFFFFFFFFFFFFFFFFFFFFFFFFFFFFFFFFFFFFFFFFFFFFFFFFFFFFFFFFFFFFFFFFFFFFFFFFFFFFFFFFFFFFFFFFFFFFFFFFFFFFFFFFFFFFFFFFFFFFFFFFFFFFFFFC1
:40BFC000FFFFFFFFFFFFFFFFFFFFFFFFFFFFFFFFFFFFFFFFFFFFFFFFFFFFFFFFFFFFFFFFFFFFFFFFFFFFFFFFFFFFFFFF00C00008FFFF030800800008FBBF0008BDAEA6162B
:40C0000001B500BF01226946F848006800F5D9700EF0ACFA20B99DF80000F54981F8B20100BF022014F04DFF0120FFF780F808BD01B500BF01226946EC48006800F2B3103A
:40C040000EF094FA20B99DF80000E94981F8B30100BF022014F035FF0120FFF768F808BD70B52DED028B05460E460024012D07D1DF4890ED610ABDEEC00A10EE104A12E0AF
:40C08000032D07D1DA4890ED630ABDEEC00A10EE104A08E0022D06D1D54890ED620ABDEEC00A10EE104AD24890F8B201032809D1D048844202DC4042844201DA00244BE056
:40C0C000012449E0CA4890F8B20108280AD142F21070844202DC4042844201DA00243BE0012439E0C24890F8B201092819D100EE104AB8EEC00AF1EE020AB4EEE00AF1EE34
:40C1000010FA0ADC00EE104AB8EEC00AF6EE000AB4EEE00AF1EE10FA01D200241CE001241AE0204635F025FD41EC180B9FEDB20B53EC102B35F082FE0BD3204635F019FDFE
:40C1400041EC180B9FEDAE0B53EC102B35F03CFD01D2002400E001241CB10120BDEC028B70BD0020FAE701460420704731B52DED020B044600BF042269469C48006800F5B6
:40C18000C2700EF0F3F920B99DED000A984880ED610A00BFFFF7E8FC10B1FEF7D2FF08E0FFF71BFD10B119F01DF802E0012014F0BBFF1C2023F05EFC01203EBD31B52DEDC3
:40C1C000020B2DED088B044694B300209FED8E0A13F0B0FD10EE105A284636F027F841EC1B0BB0EE4B0AF0EE6B0A32F0F9FBB0EE40AAF0EE60AA51EC1A0B35F0DBF908EE75
:40C20000100A7B4890EDE20A30EE480AF0EE408A90EDE20A30EE080AB0EE409A9DED080AB4EEC90AF1EE10FA03DD8DED089A09E009E09DED080AB4EEE80AF1EE10FA01D2DB
:40C24000CDED088A0FE000BF042208A96748006800F562700EF08AF920B99DED080A644880EDE20A00BF00BF042208A95F48006800F5C6700EF07AF920B99DED080A5C48FB
:40C2800080ED630A00BFFFF76FFC10B1FEF759FF08E0FFF7A2FC10B118F0A4FF02E0022014F042FF1C2023F0E5FB0120BDEC088B3EBD31B52DED020B044600BF04226946D3
:40C2C0004A48006800F5C4700EF050F920B99DED000A474880ED620A00BFFFF745FC10B1FEF72FFF08E0FFF778FC10B118F07AFF02E0032014F018FF1C2023F0BBFB01204B
:40C300003EBD014600200A292CD2DFE801F02B2021051E1F2B2B131D9FED3C1AC0EE010A9FED3B1A70EE810AFCEEE00A10EE902A90B219E0DFED360A70EE200AFCEEE00AEA
:40C3400010EE902A90B20FE000BF00BF00BF00BFDFED300A60EE200AFCEEE00A10EE902A90B201E0002000BF00BF7047014600200A2924D2DFE801F0231819051617232342
:40C380000F15DFED220A80EE201AFDEEC10A10EE902A10B215E0FCEEC00A10EE902A10B20FE000BF00BF00BF00BFDFED1A0A60EE200AFDEEE00A10EE902A10B201E00020C3
:40C3C00000BF00BF7047DFED140AB0EE600A28B91249D1ED360AB0EE600A06E0012804D10E49D1ED590AB0EE600A7047B4030020301F0020001A0B009A9999999999134064
:40C400009A9999999999B93F35FA0E3D0000AF4300401C4500007A44000000007C0D002070B52DED0A8BB0EE408A9FEDF80AC8EE000A10EE905AF64890ED610AF0EE408AB9
:40C4400090ED630AB0EE409A0020FFF7BCFFF0EE409A284635F0EAFE41EC1A0B38EEE90A78EEC90A80EE201A11EE106A304635F0DDFE41EC1C0BB0EE4C0AF0EE6C0A32F05D
:40C48000AFFAB0EE40BAF0EE60BA53EC1A2B51EC1B0B35F099FB01D2012000E0002004462046BDEC0A8B70BD70B52DED0A8BB0EE408A9FEDD60AC8EE000A10EE905AD44828
:40C4C00090ED620AF0EE408A90ED630AB0EE409A0020FFF778FFF0EE409A284635F0A6FE41EC1A0B38EEE90A78EEC90A80EE201A11EE106A304635F099FE41EC1C0BB0EEE4
:40C500004C0AF0EE6C0A32F06BFAB0EE40BAF0EE60BA53EC1A2B51EC1B0B35F055FB01D2012000E0002004462046BDEC0A8B70BD70B52DED0C8BF0EE408A9FEDB40AC8EE51
:40C54000800A10EE904AB24890ED620AF0EE409A90ED610AB0EE40AA90ED630AB0EE408A0020FFF730FFB0EE409A204635F05EFE41EC1B0B39EE480A7AEE480A80EE201A2A
:40C5800011EE106A304635F051FE41EC1D0BB0EE4D0AF0EE6D0A32F023FAB0EE40CAF0EE60CA53EC1B2B51EC1C0B35F00DFB24D2204635F03BFE41EC1B0B39EE480A79EE87
:40C5C000C80A80EE201A11EE106A304635F02EFE41EC1D0BB0EE4D0AF0EE6D0A32F000FAB0EE40CAF0EE60CA53EC1B2B51EC1C0B35F0EAFA01D2012000E000200546284677
:40C60000BDEC0C8B70BD834890F85000032801D0012070470020FCE710B50124FFF7F3FF28B97C49C86A64212BF06BFC00B10024204610BD774890F82800032801D00120CE
:40C6400070470020FCE710B50124FFF7F3FF28B97049486864212BF054FC00B10024204610BD10B5FFF7EFFF10B1FFF7D5FF08B9022411E0664890ED6A0AB5EEC00AF1EEF5
:40C6800010FA08D090ED6B0AB5EEC00AF1EE10FA01D0012400E00024204610BD18B95D4991ED080A04E0012802D15A4991ED120A704710B50021584800782DF055FC0021BB
:40C6C000564800782DF050FC514890F8B201032804D0082812D0092830D11FE000209FED500AFFF743FD00201FEDB50AFFF766FD00209FED4C0AFFF7DCFD2FE000209FED99
:40C700004A0AFFF733FD00201FEDBD0AFFF756FD00209FED460AFFF7CCFD1FE00020B6EE000AFFF723FD0020B0EE040AFFF746FD0020B1EE020AFFF7BCFD0FE00020B7EE72
:40C74000000AFFF713FD0020B0EE040AFFF736FD0020B1EE000AFFF7ACFD00BF00BF10BD01B52B4890F8410001280FD000BF012269462F48006800F2B5100DF0F7FE20B915
:40C780009DF80000224981F8B50100BF1C2023F071F908BD10B52DED028B044694ED030AD4ED040A30EE600A84ED060A94ED030A84ED040A2BF09FFB2060D4E90001401A97
:40C7C000A06094ED020AB8EE400A5FEDEE0A80EE201AB0EE418A20686060B5EEC08AF1EE10FA30DD94ED060AC0EE080AC4ED050AFFF7ECF8F0B1D4ED050AB0EE600AC821EF
:40C8000004F11C0019F032FC1DE000000000C842301F00207C0D0020E8060020E706002090ED24C990ED244900803BC500803B45B4030020D4ED050AB0EE600A042104F1D9
:40C840001C0019F013FCBDEC028B10BD10B52DED020B00BF04226946FE48006800F5D4700DF084FE20B99DED000AFB4880ED6A0A00BF1CBD10B52DED020B00BF04226946F2
:40C88000F448006800F5D6700DF070FE20B99DED000AF14880ED6B0A00BF1CBD10B52DED020B00BF04226946EA48006800F5CE700DF05CFE20B99DED000AE74880ED670AF0
:40C8C00000BF1CBD10B52DED020B00BF04226946E048006800F5D2700DF048FE20B99DED000ADD4880ED690A00BF1CBDDB4981F850007047D94981F82800704710B52DED0F
:40C90000088BB0EE408A9FEDD60AF0EE408AB3EE040AB0EE40BA18EE100A35F087FC41EC1A0BB0EE4A0AF0EE6A0A32F059F8B0EE409AF0EE609A9FEDCB0B53EC102B51EC67
:40C94000190B35F07BFA0AD21FED500AC8EE000A9FEDC60A20EE800AF0EE408A03E09FEDC00AF0EE408AB0EE680ABDEC088B10BD10B52DED028BB94890F86D01012815D0F0
:40C98000B54890F84B00B54981F86C01084690F86C11543019F05AFBB04890F86C11E03019F054FB0120AD4981F86D01AA4890F8B2010A287DD2DFE800F0FC053365FBFA38
:40C9C000F9F86681AA48007829F0E0F800EE100AB8EE400ADFEDA70A20EE200A9F4880ED040A90ED040AF6EE000AB4EEE00AF1EE10FA03D20020FFF77DFF10E0974890ED54
:40CA0000040ADFED9D0AB4EEE00AF1EE10FA03DD0120FFF76FFF02E00320FFF76BFFEDE09348007829F0B2F800EE100AB8EE400ADFED900A20EE200ADFED900A80EE201AAF
:40CA4000864880ED041A90ED040ADFED8D0AB4EEE00AF1EE10FA03D20020FFF74BFF10E07E4890ED040ADFED870AB4EEE00AF1EE10FA03DD0120FFF73DFF02E00320FFF784
:40CA800039FFBBE000BF7A4800782DF0DAF900EE100AB8EEC00A7148D0ED000A30EE200A80ED040AFDF727FD20B10020FFF722FF03E098E00320FFF71DFF9FE00AF094FE44
:40CAC00010B90AF052FB18B311F00EFFB0EE408AFFF714FF6C4880ED000A6C4800682BF032FA00EE100AB8EE400ADFED690A80EE201A684880ED001A634890ED000A654859
:40CB0000D0ED000A20EE200A634880ED000A1EE0574800782DF095F900EE100AB8EEC00A5E48D0ED000A30EE600ADFED590A80EE201A594880ED001A4D4800782DF081F904
:40CB400000EE100AB8EEC00A544880ED000A2BF0D2F94E490860414890ED040A4E48D0ED000A30EE200AF6EE000AB4EEE00AF1EE10FA19DD394890ED040A4748D0ED000AD1
:40CB800030EE200AF1EE020AB4EEE00AF1EE10FA0AD2324890ED040A3F48D0ED000A30EE200A2E4880ED040A04E01EE017E00DE00BE019E0FDF79FFC18B10020FFF79AFEB5
:40CBC00002E00320FFF796FE18E000BF9FED240A224880ED040A0020FFF78CFE0EE00320FFF788FE0AE000BF00BF9FED1D0A1B4880ED040A0020FFF77DFE00BF00BF1748BC
:40CC000090F86C11D0ED040AB0EE600A543019F0C9F91248001DFFF7BDFD0F4890F8B3010A287CD2DFE800F0AC055D9B9192A79E9C9D1B48007828F0A9FF00EE100AB8EE49
:40CC4000400ADFED0C0A20EE200A044880ED0E0A28E00000B4030020301F00207C0D0020000000000000000000003440713DAA3FE80600203333533A666646400CAC233F10
:40CC8000CDCCCC3C33339F40400000205000002000007A444C0000204800002044000020E706002090ED0E0AF6EE000AB4EEE00AF1EE10FA03D20020FFF718FE10E0FB488F
:40CCC00090ED0E0A5FED140AB4EEE00AF1EE10FA03DD0120FFF70AFE02E00320FFF706FE57E0F348007828F051FF00EE100AB8EE400A5FED200A20EE200A5FED200A80EEE6
:40CD0000201AEA4880ED0E1A90ED0E0A5FED240AB4EEE00AF1EE10FA05D2002000E02EE0FFF7E4FD10E0E14890ED0E0A5FED2B0AB4EEE00AF1EE10FA03DD0120FFF7D6FD44
:40CD400002E00320FFF7D2FD23E000BF1FED3C0AD64880ED0E0A0020FFF7C8FD19E000BF00BF00BF1FED420AD04880ED0E0A0320FFF7BCFD0DE00320FFF7B8FD09E000BFF7
:40CD80001FED490AC94880ED0E0A0020FFF7AEFD00BF00BFC54890F86C11D0ED0E0AB0EE600AE03019F0FEF8C0482C30FFF7F2FCBDEC028B10BDBF4890ED610AD0ED630ADD
:40CDC00030EE600AB5EEC00AF1EE10FA01DD012070470020FCE7B0EE040AB44880ED040A704730B589B028F0F4FC40B10021084614F087F90121002014F083F92AE0AD48F7
:40CE000090F8B201032804D0AA4890F8B201082808D10021032014F074F90121032014F070F917E0A34890F8B20109280AD10021032014F066F90121032014F062F9FFF7B1
:40CE4000CAFF07E00021032014F05BF90121002014F057F9974890F8B25190F8B3410A2D7ED2DFE805F08A0517298C8D5E8B2A2B0020009001900290034603228E490390D6
:40CE80000846007828F093FD03218B48007829F03CF987E0002000900190029003460322854903900846007828F081FD00218248007829F02AF975E000BF00BF00200090C0
:40CEC00001900290034602227B4903900846007828F06DFD02217848007829F016F928F04DFC68B175485FEDA20A9FED750A0423002274490090704800782CF0A9FC0FE0D0
:40CF000028F054FC60B16D485FEDAB0A9FED6C0A0423002219070090674800782CF098FC40E0002000900190029003460222624903900846007828F03AFD06215E480078F8
:40CF400029F0E3F8002000900190022314220121029004A82CF094FD04A85FEDBF0A00E00BE09FED590A032300224FF080410090514800782CF06CFC14E000BF00BF00BFFB
:40CF80000020009001900290034603224A4903900846007828F00BFD01214748007829F0B4F800BF00BF0A2C7ED2DFE804F09C0517299E9F5E9D2A2B002000900190029036
:40CFC000034603223A4903900846007828F0EFFC03213748007829F098F899E0002000900190029003460322314903900846007828F0DDFC00212E48007829F086F887E095
:40D0000000BF00BF002000900190029003460222274903900846007828F0C9FC02212448007829F072F828F0A9FB68B123485FEDF40A9FED230A04230122224900901C4816
:40D0400000782CF005FC0FE028F0B0FB60B11B485FEDFD0A9FED1A0A0423012291070090134800782CF0F4FB52E00020009001900290034602220E4903900846007828F068
:40D0800096FC06210A48007829F03FF8002000900190034614220121029004A82CF0F0FC04A8DFED0A0A13E01DE000007C0D0020E7060020301F0020E8060020C8D8002006
:40D0C000809FD54A00040140A037A04C000000001FED050A0223012291070090B34800782CF0B6FB14E000BF00BF00BF002000900190029003460322AC490390084600785F
:40D1000028F055FC0121A948007828F0FEFF00BF00BF09B030BD10B5A54988684FF496712AF0EFFE10BDA34890ED000A7047A24991F84110012901D1012007E09E4991F89F
:40D14000B51109B1012100E000210846704710B52DED068BB0EE408A9848007838B91FED250A974880ED000A012094490870FFF7DEFF00286AD00AF037FB002866D0FFF72A
:40D18000D2FF10EE104A204635F050F841EC1A0BB0EE4A0AF0EE6A0A31F022FCB0EE409AF0EE609A9FED870B53EC102B51EC190B34F00AFD4AD2FFF7AEFFE0BB21F009FFB7
:40D1C000DFED820AB4EEE00AF1EE10FA3EDBFFF748FA01283AD1784890F830000A2835D0754890F8B2010A2829D2DFE800F02811120513142828060700BF00BF704890EDCB
:40D20000000ADFED730A08EE200A80ED000A1CE000BF00BF00BF6848D0ED630A9FED6C1A48EE410AB0EE600A0120FEF7C7FF1FED590A634800E009E080ED000A05E01FED2F
:40D240005D0A5F4880ED000A00BF00BFBDEC068B10BD5B4890F8280008B9012070470020FCE7574890F82800012800D170470020FCE7534890F8500008B901207047002086
:40D28000FCE74F4890F85000012800D170470020FCE700B50021FFF7DCFF08B13D2103E0FFF7DFFF00B13C21084600BD10B513F0CFFF0446204610BD10B52DED028BFEF766
:40D2C00053FC20B1FDF7BCFFB0EE408A16E013F0B6FE3948D0ED640A30EE600ADFED3D0A20EE200AD0ED650A90ED641A70EEC10A80EE201A9FED380A31EE008AB0EE480A6C
:40D30000BDEC028B10BD01B59DF80000202801DD2020009000BF01226946304800684B300DF024F920B99DF80000234981F84B0000BF0020224981F86D0108BD10B54FF407
:40D34000B8711F4830F0EFF910BD25490870704723480078704710B52DED028BB0EE408A2048007830B9134800210160416001201C49087021F029FEF0EE408AF0EE680AC8
:40D38000B0EE480A13F02BFD174880ED000A28210848154A92ED000A18F068FEBDEC028B10BD114890ED000A70470000E7060020402A002038000020301F00205400002021
:40D3C0007C0D0020000000A046DF813F2FDDE43E0AD7A33B000048430000C8C2B403002030000020550000203400002010B50446204623F035FE10BD07B586B000200490DF
:40D40000002108980170069800786D2881F08E82DFE810F06D006F00EB000B0139018C0AAF003C07470752076701CD013302A802FD0252039F03F403590449048000A904B2
:40D440001B058905CF051E069C06FC08B6065D078A096907AF07BE07FC070A0818085908650875087F088F088C0A8C0A8C0A9F08B008D208750781078B07A30797078C0AB5
:40D480008C0A8C0A8C0A8C0A8C0A8C0A8C0A8C0A8C0A8C0AC0048C0A8C0A8C0A0009280945096D098C0A8C0A8C0A8C0A8C0A8C0A8C0A8C0A8C0A8C0A8C0A8C0A8C0A8C0AD8
:40D4C0008C0A8C0A8C0A8C0A8C0A9A09CB09FC098C0A8C0A8C0A0E0A560A8C0A8C0A8C0A8C0A200A320A8C0A440A680A7A0A01F021BAFE4890F841000390069890ED010A5C
:40D50000BCEEC00A10EE100AC0B20290039913F0F8FDECE70698007A032803D006210898017025E0069890ED010AF7EE000AB4EE600AF1EE10FA02D117F0B4F818E006987B
:40D5400090ED010AF0EE000AB4EE600AF1EE10FA02D117F06CF80BE0069890ED010AF0EE080AB4EE600AF1EE10FA01D116F0BDFEBDE70698007A032809D1069890ED010A98
:40D580008DED030A9DED030A0EF0CCFF2AE00698007A012811D1D548B0F8BE110A22079802FB001000EE100AB8EEC00A8DED030A9DED030A0EF0B6FF14E00698007A02286C
:40D5C00010D1CA48B0F8BE110A22079802FB101000EE100AB8EEC00A8DED030A9DED030A0EF0A0FF0120049081E70AF0FDF8C0B90698007A032811D1069890ED010A8DED5C
:40D60000030A9DED030AFDF7BBFEB948D0F81801014603908020DFF8DCC200DF0120049002E001210898017061E716F0E1F930BB0698007A03281ED1069890ED010ABCEE0A
:40D64000C00A10EE100A80B20390FDF78AFE0AF02AFE80B90821A848DFF8A0C200DF012809D0A748406840F00101A5484160A248DFF890C200DF132022F0FCF902E0012172
:40D680000898017033E716F0B3F930BB0AF00BFE18B30698007A03281BD1069890ED010ABCEEC00A10EE100AC0B20390FDF733FE08219148DFF844C200DF012809D0904831
:40D6C000406840F001008E4948608B48DFF834C200DF132022F0CEF902E001210898017005E70698007A032817D1804890F8420003907E4890F841000290069890ED010AAF
:40D70000BCEEC00A10EE100AC0B20190DDE9021211F049F90899087046E00698007A01281FD1724890F841105C3000EB41006F4991F84210415C0122079802FB0010C0B211
:40D7400001906A4890F842000390684890F8410002900146039A019811F025F90899087022E00698007A02281ED1604890F841105C3000EB41005D4991F84210415C01229C
:40D78000079802FB1010C0B20190584890F842000390564890F8410002900146039A019811F001F908990870012004909FE60698007A032817D14D4890F8420003904B4839
:40D7C00090F841000290069890ED010ABCEEC00A10EE100AC0B20190DDE9021211F021F90899087046E00698007A01281FD13F4890F84110603000EB4101603890F8420035
:40D80000095C0122079802FB0010C0B20190374890F842000390354890F8410002900146039A019811F0FDF80899087022E00698007A02281ED12D4890F84110603000EB75
:40D8400041002A4991F84210415C0122079802FB1010C0B20190254890F842000390234890F8410002900146039A019811F0D9F8089908700120049039E60698007A03288B
:40D8800017D11A4890F842000390184890F841000290069890ED010ABCEEC00A10EE100AC0B20190DDE9021211F0F9F80899087055E00698007A01282ED10C4890F84110CA
:40D8C000643000EB4100094991F84210415C0122079802FB0010C0B20190044890F842000390024890F8410002900DE0301F0020504100206108040834310020290D040835
:40D9000044310020450C04080146039A019811F0C6F80899087022E00698007A02281ED1FE4890F84110643000EB4100FB4991F84210415C0122079802FB1010C0B20190F0
:40D94000F64890F842000390F44890F8410002900146039A019811F0A2F80899087001200490C4E50698007A032810D1EB4890F842000390069890ED010A8DED020A0398EB
:40D980009DED020A11F0F8F9089908703CE00698007A01281AD1E14890F842107C3000EB8100D0ED000A9DED070AB8EEC00A30EEC00A8DED020AD94890F8420003909DED1B
:40D9C000020A11F0D9F9089908701DE00698007A022819D1D14890F842107C3000EB8100D0ED000A9DED070AB8EEC00A30EE800A8DED020AC94890F8420003909DED020AF7
:40DA000011F0BAF908990870012004906FE50698007A032810D1C14890F842000390069890ED010A8DED020A03989DED020A11F0EFF8089908703CE00698007A01281AD160
:40DA4000B64890F842106C3000EB8100D0ED000A9DED070AB8EEC00A30EEC00A8DED020AAE4890F8420003909DED020A11F0D0F8089908701DE00698007A022819D1A748A3
:40DA800090F842106C3000EB8100D0ED000A9DED070AB8EEC00A30EE800A8DED020A9F4890F8420003909DED020A11F0B1F808990870012004901AE50698007A032812D10D
:40DAC000964890F842000390069890ED010ABCEEC00A10EE100AC0B20290039911F01DF80899087032E00698007A012815D18B4890F842106830415C0122079802FB001080
:40DB0000C0B20290854890F8420001460390029811F003F80899087018E00698007A022814D17E4890F842106830415C0122079802FB1010C0B20290784890F84200014619
:40DB40000390029810F0E9FF0899087001200490CDE40698007A032810D1704890F842000390069890ED010A8DED020A03989DED020A11F05CF9089908703CE00698007A58
:40DB800001281AD1654890F84210843000EB8100D0ED000A9DED070AB8EEC00A30EE800A8DED020A5D4890F8420003909DED020A11F03DF9089908701DE00698007A022883
:40DBC00019D1564890F84210843000EB8100D0ED000A9DED070AB8EEC00A30EEC00A8DED020A4E4890F8420003909DED020A11F01EF9089908700120049078E40698007A80
:40DC0000032810D1454890F842000390069890ED010A8DED020A03989DED020A11F053F8089908703CE00698007A01281AD13B4890F84210743000EB8100D0ED000A9DEDA6
:40DC4000070AB8EEC00A30EE800A8DED020A334890F8420003909DED020A11F034F8089908701DE00698007A022819D12B4890F84210743000EB8100D0ED000A9DED070A59
:40DC8000B8EEC00A30EEC00A8DED020A234890F8420003909DED020A11F015F8089908700120049023E40698007A03280AD1069890ED010ABCEEC00A10EE100AC0B2039070
:40DCC000FCF7C5FA13E40698007A032812D1134890F842000390069890ED010ABCEEC00A10EE100AC0B20290039910F049FF0899087035E00698007A012818D1074890F8D4
:40DD000042106A30415C0122079802FB0010C0B20290024890F84200014601E0301F00200390029810F02CFF0899087018E00698007A022814D1FB4890F842106A30415CF8
:40DD40000122079802FB1010C0B20290F54890F8420001460390029810F012FF089908700120049004E40698007A032803D00621089801700DE0069890ED010A8DED030A96
:40DD80009DED030A0A2009F0B9F910B901210898017029E40698007A032814D1069890ED010ABCEEC00A10EE100A80B200EE100AB8EE400A8DED030A9DED030A0EF0B2FB21
:40DDC000089908703EE00698007A01281BD10FF03AF9F0EE400AD348B0F8BE0100EE100AB8EE401A9DED070AF8EE401AB0EE410A00EEA10A8DED030A9DED030A0EF092FBD5
:40DE0000089908701EE00698007A02281AD10FF01AF9F0EE400AC348B0F8BE0100EE100AB8EE401A9DED070AF8EE401AB0EE410A00EEE10A8DED030A9DED030A0EF072FBC4
:40DE400008990870012004901CE40698007A032815D1B44890F842000390B24890F841000290069890ED010A8DED010ADDE902019DED010A10F045FD0899087050E00698CB
:40DE8000007A012824D1A74890F842000290A54890F84100019002990FF0C2F9DDED070AF8EE600A9FEDA01A01EE200A8DED030A9C4890F8420002909A4890F84100019056
:40DEC00002999DED030A10F01CFD0899087027E00698007A022823D1924890F842000290904890F84100019002990FF099F9DDED070AF8EE600A9FED8C1A01EE600A8DEDBD
:40DF0000030A884890F842000290864890F84100019002999DED030A10F0F3FC089908700120049042E40698007A03280BD1069890ED010A8DED030A9DED030A11F000F80F
:40DF40000899087032E00698007A012815D17548D0ED7E0A9DED070AB8EE401ADFED731AB0EE600A01EE810A8DED030A9DED030A10F0E6FF0899087018E00698007A022881
:40DF800014D16848D0ED7E0A9DED070AB8EE401ADFED661AB0EE600A01EEC10A8DED030A9DED030A10F0CCFF089908700120049062E40698007A032814D1069890ED010A93
:40DFC000BCEEC00A10EE100A80B200EE100AB8EE400A8DED030A9DED030AFCF755F90899087032E00698007A012815D14D48D0ED280A079800EB8000400000EE100AB8EE3E
:40E00000C00A30EE800A8DED030A9DED030AFCF73BF90899087018E00698007A022814D14048D0ED280A079800EB8000400000EE100AB8EEC00A30EEC00A8DED030A9DEDBF
:40E04000030AFCF721F9089908700120049039E20698007A03282DD1069890ED010ADFED340AB4EEE00AF1EE10FA06DD022108980170642006F022F962E0069890ED010AA3
:40E08000F2EE040AB4EEE00AF1EE10FA06D20321089801700A2006F011F951E0069890ED010ABCEEC00A10EE100AC0B2039006F005F945E00698007A01281BD1194890F8AF
:40E0C000401007984000C0F1650081420BDA154890F840100222079802FB0010C0B2039006F0ECF82CE0022108980170642006F0E5F825E00698007A022821D1094890F8A6
:40E100004010079840000930814213DD054890F840100222079802FB1010C0B2039006F0CDF80DE0301F00200AD7233CCDCCCC3D0000C8420321089801700A2006F0BEF8AC
:40E140001920FFF753F901200490F3E30698007A032803D006210898017010E0069890ED010ABCEEC00A10EE100AC0B21FED100A039008F0C3FF10B9012108980170D9E30C
:40E180000698007A032803D00621089801707CE0069890ED010AF8EE000AB4EE600AF1EE10FA13D1FE4890F842107C3000EB810090ED000A8DED030A9DED030A082008F0C9
:40E1C0009DFF00BB0121089801705EE0069890ED010AFFEE000AB4EE600AF1EE10FA13D1EF4890F842106C3000EB810090ED000A8DED030A9DED030A082008F07FFF10B93C
:40E2000001210898017040E0069890ED010AF7EE000AB4EE600AF1EE10FA13D1E04890F84210743000EB810090ED000A8DED030A9DED030A082008F061FF00BB01210898E9
:40E24000017022E0069890ED010AF0EE000AB4EE600AF1EE10FA13D1D14890F84210843000EB810090ED000A8DED030A9DED030A082008F043FF10B901210898017004E04A
:40E280009FEDC80A002008F039FF53E30020FEF79AF88DED030A00209DED030AFDF766FF48E30020FEF78FF88DED030A00209DED030AFDF783FF3DE30020FEF784F88DED96
:40E2C000030A00209DED030AFDF7F3FF32E3069890ED010ABCEEC00A10EE100AC0B203900EF004FD26E3069890ED010ABCEEC00A10EE100AC0B20390FEF732FA1AE306982D
:40E3000090ED010ABCEEC00A10EE100AC0B2039010F087FF0EE3069890ED010A8DED030A9DED030A10F093FF04E3069890ED010ABCEEC00A10EE100AC0B2039011F0D0FC0C
:40E34000F8E2069890ED010ABCEEC00A10EE100A80B2039011F0ADFAECE2069890ED010ABCEEC00A10EE100A80B2039011F0B6FAE0E2069890ED010ABCEEC00A10EE100A3A
:40E38000C0B203900FF0A0FC2020FFF72FF8D1E20698007A032803D006210898017034E0069890ED010AF7EE000AB4EE600AF1EE10FA0ED1FDF70AFB28B1B7EE000A1120B0
:40E3C00008F09CFE21E0B7EE000A072008F096FE1BE0069890ED010AF0EE000AB4EE600AF1EE10FA05D19FED6F0A002008F086FE0BE0069890ED010AF0EE080AB4EE600AA6
:40E40000F1EE10FA01D100F07BFC93E2069890ED010ABCEEC00A10EE100A80B201460390022012F06EFC85E2069890ED010ABCEEC00A10EE100A80B201460390012012F0B1
:40E4400060FC77E20698007A03283BD1069890ED010AB5EEC00AF1EE10FA0BD1504890F8420003904E4890F8410002900399FDF766F927E0069890ED010AF7EE000AB4EEAD
:40E48000600AF1EE10FA07D1454890F8420001210390FDF7BBF815E0069890ED010AF0EE080AB4EE600AF1EE10FA0BD13C4890F8420003903A4890F8410001220290039925
:40E4C000FDF723F836E2069890ED010ABCEEC00A10EE100AC0B20390FCF7E3FF2AE20698007A03280AD1069890ED010ABCEEC00A10EE100AC0B20390FBF7C5FF1AE215F0D1
:40E5000077FA28B90698007A032801D1FCF76AFF10E20698007A03280AD1069890ED010ABCEEC00A10EE100AC0B20390FDF768FD00E20698007A03280AD1069890ED010AD2
:40E54000BCEEC00A10EE100AC0B20390FDF770FDF0E10698007A03280BD1069890ED010ABCEEC00A10EE100AC0B20121039011F0CAF9DFE10698007A03281CD1069890ED11
:40E58000010ADFED090AB4EE600AF1EE10FA12D10CF076FF01200CF051FE0020034907E0301F00200000000000007E43443100200872FE490870BDE10698007A03280BD1AE
:40E5C000069890ED010ABDEEC00A10EE100A00B20390FAF745FA18E00698007A012808D1F348B0F8AA00401C00B20390FAF738FA0BE00698007A022807D1ED48B0F8AA0004
:40E60000401E00B20390FAF72BFA93E11B20FEF7EDFE8FE10698007A03281AD1E44890F842106C3000EB810090ED000A8DED050A9DED050AB5EEC00AF1EE10FA03D19FED87
:40E64000DD0A8DED050A9DED050A082008F056FD07E00698007A20B91FED2E0A082008F04DFD67E10698007A03280FD1D04890F842107C3000EB810090ED000A8DED030A15
:40E680009DED030A082008F039FD07E00698007A20B91FED3C0A082008F030FD4AE10698007A03281AD1C24890F84210743000EB810090ED000A8DED050A9DED050AB5EE5D
:40E6C000C00AF1EE10FA03D19FEDBB0A8DED050A9DED050A082008F011FD07E00698007A20B91FED500A082008F008FD22E10698007A03280FD1AE4890F84210843000EBFA
:40E70000810090ED000A8DED030A9DED030A082008F0F4FC07E00698007A20B91FED5F0A082008F0EBFC05E10698007A03280AD1069890ED010ABCEEC00A10EE100AC0B227
:40E740000390FCF78FFEF5E00698007A03280ED1069890ED010ABCEEC00A10EE100A80B20121039016F0BDFD089908701CE00698007A01280AD116F031FD401C80B2012121
:40E78000039016F0AEFD089908700DE00698007A022809D116F022FD401E80B20121039016F09FFD08990870C4E00698007A03280ED1069890ED010ABCEEC00A10EE100A56
:40E7C00080B20121039016F0A4FD089908701CE00698007A01280AD116F0FCFC401C80B20121039016F095FD089908700DE00698007A022809D116F0EDFC401E80B20121BE
:40E80000039016F086FD0899087093E00698007A03280CD1069890ED010ABCEEC00A10EE100A80B2039016F08CFD0899087081E00698007A03280CD1069890ED010ABCEEA0
:40E84000C00A10EE100A80B2039016F091FD089908706FE00698007A03280CD1069890ED010ABCEEC00A10EE100A80B2039016F09AFD089908705DE00698007A03280CD14B
:40E88000069890ED010ABCEEC00A10EE100A80B2039016F0A3FD089908704BE00698007A03280CD1069890ED010ABCEEC00A10EE100AC0B2039012F0E3FC0899087039E00D
:40E8C0000698007A03280CD1069890ED010ABCEEC00A10EE100A80B2039016F0AFFD0899087027E00698007A03280CD1069890ED010ABDEEC00A10EE100A00B2039016F091
:40E90000CFFD0899087015E00698007A03280CD1069890ED010ABDEEC00A10EE100A00B2039016F0A6FD0899087003E007210898017000BF00BF049809B000BD86B04FF6FC
:40E94000FF7438211D48DFF878C000DF02211D4880F808110C2284211B4831F02BFE002877D10321174880F8081100BF224605A91248DFF858C000DF01286CD000208DF854
:40E9800000008DF80D0001208DF80C0000208DF80E000598007800284CD004AA01210598FEF72AFD05469DF8100011E0E8040020301F0020CDCCCCBDCDCCCC3D840F0020AB
:40E9C000E909040850410020000F0020790B040868B100250599087822F094FE06460598837A427A9DF81010304622F091FE08F0FBFE08B1002504E00598007A032800D175
:40EA000000250DB39DF80D00F0B90598007AD8B1059A07CA8DE8070001208DF80D008DF80C004FF47A649DF80E00401CC0B28DF80E0009E008F099FB30B15F48D0F890114B
:40EA40000120DFF878C100DF5D480599F9F758FC8CE748E0FFE79DF80000002886DD9DF80E0000283CDD9DF80E00032803D102208DF80C000EE09DF80E00052803D106206D
:40EA80008DF80C0006E09DF80E00072802D110208DF80C009DF80E00FF2805DA9DF80E00401CC0B28DF80E009DF80C1004AA6846FEF7A2FC9DF8100078B100208DF80E00AB
:40EAC0000599087822F01EFE06460598837A427A9DF81010304622F01BFE4FF4FA6445E74FF6FF7442E70521334880F808110020DFF8D0C000DF00BFFEE72DE9F0472DED81
:40EB0000028B0546B0EE408A0E46174698464FF001092D48DFF8B4C000DFD0B900BF264890F8090140F00201234880F80911B0F814014FF6FF71884207DA1F48B0F8140165
:40EB4000401C81B21C48A0F8141100BF4FF000092CE01B48F9F7C4FB04466CB1257084ED018A2672677284F80A800A2221461648DFF85CC000DF19E000BF0F4890F80901ED
:40EB800040F004010C4880F80911B0F814014FF6FF71884207DA0848B0F81401401C81B20548A0F8141100BF4FF000094846BDEC028BBDE8F087000050410020610804086A
:40EBC000000F0020E5120408840F0020E1090408D50A040831B52DED020B0446FE4890EDD40ADDED000AB4EEE00AF1EE10FA00D3ACB100BF04226946F848006800F55470E9
:40EC00000BF0B4FC20B99DED000AF34880EDD40A00BFF348C16B0220DFF8C8C300DF3EBD31B52DED020B0446EB4890EDD30ADDED000AB4EEE00AF1EE10FA00DCACB100BF8D
:40EC400004226946E548006800F553700BF08EFC20B99DED000AE04880EDD30A00BFE048C16B0220DFF87CC300DF3EBD31B52DED020B0446D84890ED2F0ADDED000AB4EE46
:40EC8000E00AF1EE10FA00D3A4B100BF04226946D2480068BC300BF069FC20B99DED000ACD4880ED2F0A00BFCD48C16B0220DFF834C300DF3EBD31B52DED020B0446C648A0
:40ECC00090ED2E0ADDED000AB4EEE00AF1EE10FA00DCA4B100BF04226946C0480068B8300BF044FC20B99DED000ABB4880ED2E0A00BFBB48C16B0220DFF8E8C200DF3EBD3E
:40ED000010B54FF4C871B8482EF00DFDB24890F82800B54981F88C0129F0EDF8B2498860012081F88801002081F889019FEDAF0A084680ED3B0A002006F01FFF01209FED6F
:40ED4000AB0AFFF7B8FF01209FEDA80AFFF78EFF01209FEDA60AFFF763FF01209FEDA30AFFF738FF10BD10B5002426F007FD40B39F4800680078012800D128E09C4800683B
:40ED80000078022801D1142421E0994800680078052801D128241AE0954800680078032801D13C2413E0924800680078062801D150240CE08E4800680078082807D1642433
:40EDC00005E026F0F3FC10B1874890F88D41204610BD10B5844890F8890186490978884203D0FFF7C0FF8449087010BD70B52DED028B044614F0FCFD00287DD1002596E095
:40EE00007548C03000EB8400D0ED000AB0EE600A284610F0D1F87048C03000EB8400D0ED000AB0EE600A28460FF0F2FE6A48C83000EB8400D0ED000AB0EE600A284610F017
:40EE4000EFF86548C83000EB8400D0ED000AB0EE600A28460FF037FF5F48D03000EB8400D0ED000AB0EE600A284610F0FDF85A48D03000EB8400D0ED000AB0EE600A28468F
:40EE80000FF07AFF5448D83000EB8400D0ED000AB0EE600A284610F00CF94F48D83000EB8400D0ED000AB0EE600A28460FF0BFFF4949E031085D294610F020F94649E2314B
:40EEC000085D294610F039F926F058FC08B34249E0310A5D891C095D501800EBD071491000EE101AB8EEC00AB0EE408ABCEEC80A10EE101AC8B200E01DE021460FF00DFE90
:40EF0000BCEEC80A10EE101AC8B221460FF038FE0BE03149E031085D21460FF0FEFD2E49E231085D21460FF02BFE681CC5B2022DFFF666AFA3E02848C03000EB8400D0ED1A
:40EF4000000AB0EE600A204610F036F82248C03000EB8400D0ED000AB0EE600A20460FF057FE1D48C83000EB8400D0ED000AB0EE600A204610F054F81748C83000EB840086
:40EF8000D0ED000AB0EE600A20460FF09CFE1248D03000EB8400D0ED000AB0EE600A204610F062F80C48D03000EB8400D0ED000AB0EE600A20460FF0DFFE0748D83000EB15
:40EFC0008400D0ED000AB0EE600A204610F071F80148D83012E00000301F0020B40300205041002061080408C00F002000000000180300203F0300203E03002000EB8400E4
:40F00000D0ED000AB0EE600A20460FF010FFFE49085D214610F072F8FB49891C085D214610F08BF826F0AAFBF0B1F7490A5D891C095D501800EBD071491000EE101AB8EE1F
:40F04000C00AB0EE408ABCEEC80A10EE101AC8B221460FF062FDBCEEC80A10EE101AC8B221460FF08DFD0AE0E749085D21460FF054FDE549891C085D21460FF081FDBDEC72
:40F08000028B70BD01B500BF01226946DF48006800F5E9700BF06AFA28B99DF80000DA49E03981F8D20100BF08BD10B5032006F064FD1FED320A002008F020F80120FFF7C3
:40F0C000E1FFD149E03991F84200FFF78FFE172020F0D0FC10BD01B5B8B000203590349033903290319030902F902E901FED410A389880ED530A1FED430A389880ED560A9E
:40F100001FED460A389880ED540A1FED480A389880ED580A1FED4B0A389880ED550A1FED4D0A389880ED590A01203790FEE3379832F036FD9FEDB60B53EC102BCDE926014A
:40F140009DED260B51EC100B32F022FBCDE92C0137983690389890ED6A0B8DED200B9DED2C0B53EC102B9DED200B51EC100B32F067FDCDE92401389890ED680B8DED1A0B56
:40F180009DED2C0B53EC102B9DED1A0B51EC100B32F056FDCDE91C019DED2C0B53EC102B9DED1C0B51EC100B32F04AFDCDE92001389890ED660B8DED140B9DED2C0B53ECEA
:40F1C000102B9DED140B51EC100B32F039FDCDE916019DED2C0B53EC102B9DED160B51EC100B32F02DFDCDE918019DED2C0B53EC102B9DED180B51EC100B32F021FDCDE91F
:40F200001C01389890ED640B8DED0E0B9DED2C0B53EC102B9DED0E0B51EC100B32F010FDCDE910019DED2C0B53EC102B9DED100B51EC100B32F004FDCDE912019DED2C0B51
:40F2400053EC102B9DED120B51EC100B32F0F8FCCDE914019DED2C0B53EC102B9DED140B51EC100B32F0ECFCCDE91801389890ED620B8DED080B9DED2C0B53EC102B9DED13
:40F28000080B51EC100B32F0DBFCCDE90A019DED2C0B53EC102B9DED0A0B51EC100B32F0CFFCCDE90C019DED2C0B53EC102B9DED0C0B51EC100B32F0C3FCCDE90E019DEDE3
:40F2C0002C0B53EC102B9DED0E0B51EC100B32F0B7FCCDE910019DED2C0B53EC102B9DED100B51EC100B32F0ABFCCDE91401389890ED600B8DED020B9DED2C0B53EC102B80
:40F300009DED020B51EC100B32F09AFCCDE904019DED2C0B53EC102B9DED040B51EC100B32F08EFCCDE906019DED2C0B53EC102B9DED060B51EC100B32F082FCCDE9080149
:40F340009DED2C0B53EC102B9DED080B51EC100B32F076FCCDE90A019DED2C0B53EC102B9DED0A0B51EC100B32F06AFCCDE90C019DED2C0B53EC102B9DED0C0B51EC100B57
:40F3800032F05EFCCDE91001389890ED5E0B8DED000B9DED2C0B53EC102B9DED000B51EC100B32F04DFCCDE902019DED2C0B53EC102B9DED020B51EC100B32F041FCCDE944
:40F3C00004019DED2C0B53EC102B9DED040B51EC100B32F035FCCDE906019DED2C0B53EC102B9DED060B51EC100B32F029FCCDE908019DED2C0B53EC102B9DED080B51EC83
:40F40000100B32F01DFC07E010200020B40300200000000000002440CDE90A019DED2C0B53EC102B9DED0A0B51EC100B32F008FCCDE90C019DED2C0B53EC102B9DED0C0B4C
:40F4400051EC100B32F0FCFBCDE90E019DED100B53EC102B9DED0E0B51EC100B32F0DCF8CDE912019DED140B53EC102B9DED120B51EC100B32F0D0F8CDE916019DED180BF7
:40F4800053EC102B9DED160B51EC100B32F0C4F8CDE91A019DED1C0B53EC102B9DED1A0B51EC100B32F0B8F8CDE91E019DED200B53EC102B9DED1E0B51EC100B32F0ACF847
:40F4C000CDE922019DED240B53EC102B9DED220B51EC100B32F0A0F8CDE92601389890ED6C0B8DED240B9DED240B53EC102B9DED260B51EC100B32F08FF8CDE92A0138984D
:40F5000090ED7A0B8DED200B9DED2C0B53EC102B9DED200B51EC100B32F092FBCDE92401389890ED780B8DED1A0B9DED2C0B53EC102B9DED1A0B51EC100B32F081FBCDE94D
:40F540001C019DED2C0B53EC102B9DED1C0B51EC100B32F075FBCDE92001389890ED760B8DED140B9DED2C0B53EC102B9DED140B51EC100B32F064FBCDE916019DED2C0B0F
:40F5800053EC102B9DED160B51EC100B32F058FBCDE918019DED2C0B53EC102B9DED180B51EC100B32F04CFBCDE91C01389890ED740B8DED0E0B9DED2C0B53EC102B9DEDEA
:40F5C0000E0B51EC100B32F03BFBCDE910019DED2C0B53EC102B9DED100B51EC100B32F02FFBCDE912019DED2C0B53EC102B9DED120B51EC100B32F023FBCDE914019DED5F
:40F600002C0B53EC102B9DED140B51EC100B32F017FBCDE91801389890ED720B8DED080B9DED2C0B53EC102B9DED080B51EC100B32F006FBCDE90A019DED2C0B53EC102B6F
:40F640009DED0A0B51EC100B32F0FAFACDE90C019DED2C0B53EC102B9DED0C0B51EC100B32F0EEFACDE90E019DED2C0B53EC102B9DED0E0B51EC100B32F0E2FACDE91001BC
:40F680009DED2C0B53EC102B9DED100B51EC100B32F0D6FACDE91401389890ED700B8DED020B9DED2C0B53EC102B9DED020B51EC100B32F0C5FACDE904019DED2C0B53EC40
:40F6C000102B9DED040B51EC100B32F0B9FACDE906019DED2C0B53EC102B9DED060B51EC100B32F0ADFACDE908019DED2C0B53EC102B9DED080B51EC100B32F0A1FACDE9F3
:40F700000A019DED2C0B53EC102B9DED0A0B51EC100B32F095FACDE90C019DED2C0B53EC102B9DED0C0B51EC100B32F089FACDE91001389890ED6E0B8DED000B9DED2C0B6C
:40F7400053EC102B9DED000B51EC100B32F078FACDE902019DED2C0B53EC102B9DED020B51EC100B32F06CFACDE904019DED2C0B53EC102B9DED040B51EC100B32F060FAC0
:40F78000CDE906019DED2C0B53EC102B9DED060B51EC100B32F054FACDE908019DED2C0B53EC102B9DED080B51EC100B32F048FACDE90A019DED2C0B53EC102B9DED0A0B00
:40F7C00051EC100B32F03CFACDE90C019DED2C0B53EC102B9DED0C0B51EC100B32F030FACDE90E019DED100B53EC102B9DED0E0B51EC100B31F010FFCDE912019DED140B95
:40F8000053EC102B9DED120B51EC100B31F004FFCDE916019DED180B53EC102B9DED160B51EC100B31F0F8FECDE91A019DED1C0B53EC102B9DED1A0B51EC100B31F0ECFE0F
:40F84000CDE91E019DED200B53EC102B9DED1E0B51EC100B31F0E0FECDE922019DED240B53EC102B9DED220B51EC100B31F0D4FECDE92601389890ED7C0B8DED240B9DED88
:40F88000240B53EC102B9DED260B51EC100B31F0C3FECDE928016421369890FBF1F201FB120008BB9DED2A0B51EC100B31F082FE01466422369890FBF2F2521E389800F542
:40F8C000027040F822109DED280B51EC100B31F071FE01466422369890FBF2F2521E389800F50C7040F82210389890ED000AB1EE400A8DED250A259832F098FCCDE9260129
:40F900009DED2A0B53EC102B9DED260B51EC100B32F094FA2AD23598401C80B235909DED350AB8EE400ADFEDFE0A00E028E2B4EEE00AF1EE10FA1BDD389890ED530AB5EE7E
:40F94000C00AF1EE10FA13D19DED2C0B51EC100B31F030FE00EE100AB1EE400AF3EE040A30EE200A389880ED530A01E000203590389890ED000AB1EE400A8DED250A25985A
:40F9800032F054FCCDE926019DED2A0B53EC102B9DED260B51EC100B32F050FA26D23498401C80B234909DED340AB8EE400ADFEDDC0AB4EEE00AF1EE10FA19DD9DED2C0B94
:40F9C00051EC100B31F0F6FD00EE100AF1EE400A9DED340AB8EE400AB2EE041AC0EE011A30EEA10A389880ED520A01E000203490389890ED010AB1EE400A8DED250A25985D
:40FA000032F014FCCDE926019DED2A0B53EC102B9DED260B51EC100B32F010FA28D23198401C80B231909DED310AB8EE400AF1EE040AB4EEE00AF1EE10FA1BDD389890EDD1
:40FA4000540AB5EEC00AF1EE10FA13D19DED2C0B51EC100B31F0AEFD00EE100AB1EE400AF6EE000A30EE200A389880ED540A01E000203190389890ED030AB1EE400A8DEDC8
:40FA8000250A259832F0D2FBCDE926019DED2A0B53EC102B9DED260B51EC100B32F0CEF928D22F98401C80B22F909DED2F0AB8EE400AF1EE040AB4EEE00AF1EE10FA1BDD3E
:40FAC000389890ED550AB5EEC00AF1EE10FA13D19DED2C0B51EC100B31F06CFD00EE100AB1EE400AF6EE000A30EE200A389880ED550A01E000202F9038980068259032F0EB
:40FB000095FBCDE926019DED280B53EC102B9DED260B51EC100B32F057F826D23398401C80B233909DED330AB8EE400ADFED7C0AB4EEE00AF1EE10FA19DD389890ED560A68
:40FB4000B5EEC00AF1EE10FA11D19DED2C0B51EC100B31F02FFD00EE100AF3EE040A30EE600A389880ED560A01E00020339038980068259032F05AFBCDE926019DED280B09
:40FB800053EC102B9DED260B51EC100B32F01CF824D23298401C80B232909DED320AB8EE400ADFED5F0AB4EEE00AF1EE10FA17DD9DED2C0B51EC100B31F0FCFC00EE900A64
:40FBC0009DED320AB8EE400AB2EE041AC0EE011A30EEE10A389880ED570A01E00020329038984068259032F021FBCDE926019DED280B53EC102B9DED260B51EC100B31F0AB
:40FC0000E3FF26D23098401C80B230909DED300AB8EE400AF1EE040AB4EEE00AF1EE10FA19DD389890ED580AB5EEC00AF1EE10FA11D19DED2C0B51EC100B31F0BBFC00EE02
:40FC4000100AF6EE000A30EE600A389880ED580A01E0002030903898C068259032F0E6FACDE926019DED280B53EC102B9DED260B51EC100B31F0A8FF26D22E98401C80B2AA
:40FC80002E909DED2E0AB8EE400AF1EE040AB4EEE00AF1EE10FA19DD389890ED590AB5EEC00AF1EE10FA11D19DED2C0B51EC100B31F080FC00EE100AF6EE000A30EE600A60
:40FCC000389880ED590A01E000202E90389890ED5C0AB1EE400A8DED250A259832F0A6FACDE926019DED2A0B53EC102B9DED260B51EC100B32F0A2F819D29DED2A0B51EC15
:40FD0000100B31F057FC3899C1F870019DED2C0B51EC100B31F04EFC00EE100A02E0000000004843B1EE400A389880ED5A0A3898D0F87401259032F079FACDE926019DEDF8
:40FD4000280B53EC102B9DED260B51EC100B31F03BFF11D29DED280B51EC100B31F02AFC3899C1F874019DED2C0B51EC100B31F021FC3899C1F86C013798401C80B23790B8
:40FD80003798B0F57A7F7FF7D2A9389890ED540AB5EEC00AF1EE10FA0BD0389890ED540A80ED5A0A389890ED010AB1EE400A80ED5C0A389890ED580AB5EEC00AF1EE10FA74
:40FDC00009D0389890ED580A80ED5B0A389890ED010A80ED5D0A389890ED530AB5EEC00AF1EE10FA61D0389890ED560AB5EEC00AF1EE10FA59D0389890ED5A0AD0ED530A55
:40FE0000B7EE001A70EEC10AB4EEE00AF1EE10FA4BDC389890ED5B0AD0ED560AB7EE001A70EE810AB4EEE00AF1EE10FA3DD3389890ED530AD0ED520A30EE600A8DED230A50
:40FE4000239832F0F3F9CDE924019DED240B2EF0C7FD8DED260B9FEDFD0B53EC102B9DED260B51EC100B31F0E9FF1ED3389890ED560AD0ED570A30EE600A8DED230A2398C8
:40FE800032F0D4F9CDE924019DED240B2EF0A8FD8DED260B9FEDED0B53EC102B9DED260B51EC100B31F0CAFF03D22320E94981F88601389890ED550AB5EEC00AF1EE10FA0A
:40FEC00004D19FEDE50A389880ED550A389890ED590AB5EEC00AF1EE10FA04D19FEDDF0A389880ED590A39B000BD70B52DED088B064600246FE09FEDDA0BB0EE408AF0EE38
:40FF0000608A9FEDD70BB0EE409AF0EE609A002551E006F1400000EB850090ED000A10EE101A084632F082F941EC1B0B04EB440000EBC400CC4901EBC00000EBC50090ED5F
:40FF4000001BB0EE410AF0EE610A53EC102B51EC1B0B31F075FE53EC182B31F05DFB41EC180B06F16C0000EB850090ED000A10EE101A084632F05AF941EC1B0B04EB4400AD
:40FF800000EBC400B84901EBC00000EBC50090ED001BB0EE410AF0EE610A53EC102B51EC1B0B31F04DFE53EC192B31F035FB41EC190B681CC5B20B2DABDB06F5BC7000EB32
:40FFC000C40080ED008B06F5DC7000EBC40080ED009B601CC4B2082C8DDBBDEC088B70BDA24A92F82810022914D19FEDA10A80ED000A9FEDA00A80ED010A9FED9F0A80ED94
:020000040801F1
:40000000020A9FED9E0A80ED030A9FED9D0A80ED040A6FE00D2914D19FED950A80ED000A9FED940A80ED010A9FED930A80ED020A9FED920A80ED030A9FED910A80ED040AC4
:4000400058E00C2914D19FED8A0A80ED000A9FED890A80ED010A9FED880A80ED020A9FED870A80ED030A9FED860A80ED040A41E0032914D19FED7E0A80ED000A9FED7D0A6B
:4000800080ED010A9FED7C0A80ED020A9FED7B0A80ED030A9FED7A0A80ED040A2AE0012914D19FED730A80ED000A9FED720A80ED010A9FED710A80ED020A9FED720A80ED19
:4000C000030A9FED710A80ED040A13E09FED680A80ED000A9FED670A80ED010A9FED660A80ED020A9FED670A80ED030A9FED660A80ED040A704770B52DED028B04466348B9
:40010000FFF76EFF6148FFF7F0FE6048FEF7E3FF5E48D0ED550AB0EE600A20460EF02CFE5A48D0ED550AB0EE600A20460EF09CFF5648D0ED590AB0EE600A20460EF077FE94
:400140005248D0ED590AB0EE600A20460EF0B1FF4E4890ED000AFFEE000A20EE200AB0EE408A90ED5A0AD0ED530A30EE600AD0ED5C0A70EEC80A80EE801A80ED7E1AD0ED55
:400180007E0A90ED531AB0EE480A00EEC10A80ED7F0A90ED000AB0EE408A90ED5B0AD0ED560A30EE600AD0ED5D0A70EEC80A80EE801A80ED801AD0ED800A90ED561AB0EE83
:4001C000480A00EEC10A80ED810A90ED040AD0ED7E0A80EE201AB0EE418A9FED200A28EE000AB0EE408A9FED2A0AB4EEC08AF1EE10FA04DD9FED260AB0EE408A0AE0B7EEB4
:40020000000AB4EEC08AF1EE10FA03D2B7EE000AB0EE408AB6EE000A38EE000ABCEEC00A10EE100AC5B2214628460EF076FC214628460EF063FF154890ED040AD0ED800A69
:4002400080EE201AB0EE418A24E00000000000000000F03FC00F00200000C8C20000C842000000000000000058000020301F002035FA0E3DC2B8323E00000000C2B8B23E02
:400280008FDAA53B920A063F88C3643B5011002000007F431FED0F0A28EE000AB0EE408A1FED050AB4EEC08AF1EE10FA04DD1FED080AB0EE408A0AE0B7EE000AB4EEC08A5E
:4002C000F1EE10FA03D2B7EE000AB0EE408AB6EE000A38EE000ABCEEC00A10EE100AC5B2214628460EF04CFC214628460EF025FFBDEC028B70BD70B502460C4600201FEDE8
:40030000222AF0EE420A1FED242AB0EE421A1FED262AB0EE420A1FED282AF0EE421A64B902F1400102F16C031FED2C2AB0EE420A9FEDF92AF0EE421A1CE0012C0CD102F134
:40034000980102F1C403B0EE002AB0EE420AB7EE002AF0EE421A0DE0022C0BD102F1F00102F58E73B3EE042AB0EE420AB2EE042AF0EE421AB5EEC00AF1EE10FA7EDD1FED1E
:40038000422A81ED002A1FED442A83ED002A1FED462A82ED052A012082E002EE100AB8EE422AF2EE042A22EE222A02F1140505EB800585ED002A451ED84E06EB850595ED5F
:4003C000002AB5EEC02AF1EE10FA06DD1FED562A01EB800585ED002A09E0451ECF4E06EB850595ED002A01EB800585ED002A451ECA4E2C3606EB850595ED002AB5EEC02AB3
:40040000F1EE10FA06D21FED642A03EB800585ED002A0AE0451EC14E2C3606EB850595ED002A03EB800585ED002A01EB800595ED002A451E01EB8505D5ED002A32EE622AD0
:40044000F0EE420A03EB800595ED002A451E03EB8505D5ED002A32EE622AB0EE421AB1EE402AF4EEC20AF1EE10FA12D3F4EEE10AF1EE10FA0DDCB4EEC01A00E013E0F1EE74
:4004800010FA06DCB1EE612AB4EEC21AF1EE10FA04D22325A14E2C3E86F88651451CE8B20B28FFF67AAF70BD10B500219C48FFF722FF01219A48FFF71EFF02219848FFF789
:4004C0001AFF10BD10B52DED028B964890F828400E2C2AD2DFE804F0290B080712292929191A1B220A0900BF00BF00BF00BF9FED8E0A8A482C3880ED3B0A1DE09FED8B0A72
:4005000086482C3880ED3B0A16E000BF00BF9FED860A82482C3880ED3B0A0DE0B3EE040A7E482C3880ED3B0A06E01FEDAD0A7B482C3880ED3B0A00BF00BFFBF756FA70B18C
:4005400014F0BEFEB0EE408A14F040FE00EE100AB8EE400AB4EEC08AF1EE10FA10DCFBF735FA30B1FAF76CFEB5EEC00AF1EE10FA06DC10F00EFDB5EEC00AF1EE10FA09DD7C
:4005800066482C3890ED3B0AFFEE000A20EE200A80ED3B0ABDEC028B10BD73B52DED020B04460D460A2C21D200BF05EB85026049096801F5177101EBC20101EB840004225B
:4005C000694609F0D3FF50B99DED000A05EB8501584800EBC10000EB840080ED000A00BF5548C16B0220DFF854C100DF7FBD10B5FAF7E8FB10BD73B52DED020B04460D4639
:400600000A2C21D200BF05EB85024949096801F59A7101EBC20101EB84000422694609F0A5FF50B99DED000A05EB8501444800EBC10000EB840080ED000A00BF3E48C16B24
:400640000220DFF8F8C000DF7FBD73B52DED020B04460D460A2C22D200BF05EB85023449096801F5037101EBC20101EB84000422694609F07BFF58B99DED000A05EB850188
:400680002C48503800EBC10000EB840080ED000A00BF2948C16B0220DFF8A0C000DF7FBD10B5FAF78FFB10BD73B52DED020B04460D460A2C21D200BF05EB85021C490968AE
:4006C000E43101EBC20101EB84000422694609F04DFF58B99DED000A05EB85011848503800EBC10000EB840080ED000A00BF1248C16B0220DFF844C000DF7FBD094A92F8DD
:40070000281004292DD01DDC012924D002291FD003292CD11BE00000920A863EEC0F002050110020301F002000008C4200004842B40300208C210020504100206108040875
:40074000642000200C2905D00D2910D101E000BF00BF00BF00BF1FED0C0AFE4A82ED3B0A0BE01FED0E0AFB4A82ED3B0A05E09FEDFA0AF84A82ED3B0A00BF00BF032808D1C4
:40078000F44A92ED3B0AFFEE000A20EE200A82ED3B0A7047F14A92F82810062905D19FEDF00AEC4A82ED3B0A0CE0042905D11FED210AE84A82ED3B0A04E01FED250AE54AD1
:4007C00082ED3B0A062808D1E24A92ED3B0AFFEE000A20EE200A82ED3B0A7047B5EEC00AF1EE10FA01D2012070470020FCE7B5EEC00AF1EE10FA01DD012070470020FCE7A1
:400800002DE9F04106460C4615460427D34890F828802868A0B927F06EFB28600020D14908709FEDD10A10F0E3FC20B1BFEE000ACE4880ED000A10F0ACFBCD4880ED000AD1
:40084000B8F1040F1FD009DCB8F1010F11D0B8F1020F0BD0B8F1030F1FD106E0B8F10C0F06D0B8F10D0F18D101E000BF00BF00BF00BFBE4890ED000A5FED550A20EE200A93
:4008800084ED000A13E0B94890ED000A5FED590A20EE200A84ED000A09E0B44890ED000ADFEDAD0A20EE200A84ED000A00BF00BF41F28831286827F024FB20B1212030705C
:4008C0000127002595E040F6C411286827F019FBE0B1A4480078C8B99FEDA60A10F088FC20B99FEDA40A10F028FC78B101209D4908709E4890ED000AFFEE000A20EE200ABF
:4009000080ED000A27F0F7FA286072E0D4ED000AB0EE600AFFF76BFF68B110F03AFB9448D0ED000A30EE600ADFED920AB4EEE00AF1EE10FA14DCD4ED000AB0EE600AFFF71C
:400940004DFFA8B110F025FB8948D0ED000A30EE600ADFED890AB4EEE00AF1EE10FA07D203279FED7D0A84ED000A0020286040E0D4ED000AB0EE600AFFF739FF68B110F04B
:4009800008FB7B48D0ED000A30EE600ADFED7A0AB4EEE00AF1EE10FA14D3D4ED000AB0EE600AFFF71BFF20B310F0F3FA7048D0ED000A30EE600ADFED6F0AB4EEE00AF1EE1C
:4009C00010FA16DD654890F89C0018B90120F9F73EFC07E0614890F89C00012802D10020F9F735FC03279FED5C0A84ED000A002028603846BDE8F08110B52DED048B0424B3
:400A0000544890F888010A287DD2DFE800F00506FE477CFD487CFCFB00BF4E4890F8890120B1102821D0112835D110E01120494981F8890110F0ADFA464880ED080AB6EE9F
:400A4000000A80ED3B0A00204249086024E0414A02F1EC0101F19A00FFF7D2FE032803D110203C4981F8890116E00620394981F88801022081F889010A2081F88F01002017
:400A8000086010F086FA334880ED080AB6EE000A80ED3B0A00E000BF00BF1EE300BF2D4890F88901801E0B286AD2DFE800F00669B7FD76DF6969696990002648006870B9E0
:400AC00027F019FA23490860084690F88D010A2805DD084690F88D01C01F81F88D011D4991F88801FFF756FE1A4908684FF47A6127F007FAB0B110F04CFA1648D0ED080A97
:400B000030EEC00A00E0F9E3B0EEC00ADFED1B0AB4EEE00AF1EE10FA04D221200D4981F8860139E09FED130A10F062FB20B1094890F88801032809D09FED0E0A10F0FDFAE5
:400B400050B3044890F88801062825D1B6EE000A004816E0C00F002000000000301F00200000204241030020C2B8323E4403002048030020C2B8B23DC2B8B2BD35FA0E3D59
:400B8000A9E280ED3B0A0620FE4981F889010C2081F88B01002008609EE2B6EE000AF94880ED3B0A006818B927F0A5F9F5490860F4490868C82127F0A4F938B1F14890F826
:400BC0008B01F04981F889010020086084E2ED4991F88801FFF792FDEA48006818B927F08AF9E8490860E74908684FF4FA7127F088F990B1B6EE000AE24880ED3B0A0620FD
:400C0000E04903E0E1E3E7E368E268E281F8890100200860042081F88B015DE210F0B9F9F0EE409A4FF6FF71D74815F01FFAD548006818B927F05FF9D2490860D149086865
:400C40004FF4FA7127F05DF978B1CE4890ED530A80ED080A0720CB4981F889010020086001F580700021C164016535E2C548006818B927F040F9C3490860C24890F88F0126
:400C800000EB8000400000EE100AB8EEC00ABD4880ED3B0A90F8880103280AD1B94890ED3B0AFFEE000A00E044E020EE200A80ED3B0A1FED500A10F09BFA20B1B14890F84E
:400CC0008801062809D01FED550A10F036FAB0B1AC4890F88801032811D10220A94981F8890101F580700021C164016510F051F9A44880ED080A0020A249086019E0A149A2
:400D000008684FF4FA7127F0FCF890B1B6EE000A9C4880ED3B0A06209A4981F88901086827F011F99749C86100200860052081F88B01D1E110F02DF9F0EE409A4FF6FF7168
:400D4000914815F093F98F48006818B927F0D3F88C4908608B4908684FF4FA7127F0D1F800287DD0874890ED530AD0ED080A30EE608AB0EEC80AF0EE409A10F0DEF920B143
:400D8000804890F8880103281FD01FED860A10F0D4F920B17B4890F88801032815D0B0EEC80AF0EE409A10F023FA20B1754890F88801062809D01FED910A10F019FA98B134
:400DC000704890F8880106280ED102206D4981F88901084690ED530A80ED080A00F580700021C16401650DE00720664981F88901084690ED530A80ED080A00F58070002197
:400E0000C16401655F4890F88F01401E5D4981F88F01084690F8880103285AD1084690ED070AF8EE400A9FED591A80EE810AC8EE000A90F88F112C3000EB8100C0ED000A3B
:400E4000534A92F842104F4A92F88F0192F88F312C3202EB8302D2ED000AB0EE600A00E038E1FFF721FC474890F88F112C3000EB8100D0ED000AB0EE600A0020FDF71BFFD3
:400E8000FFF70EFC3F4890F88F11843000EB810080ED000A3E4A92F842103A4A92F88F0192F88F31843202EB8302D2ED000AB0EE600AFFF7CAFB334890F88F11843000EBAA
:400EC0008100D0ED000AB0EE600A0020FDF7A8FE57E02C4890ED070AF8EE400A9FED2B1A80EE810AC8EE000A90F88F11583000EB8100C0ED000A264A92F84210214A92F8E1
:400F00008F0192F88F31583202EB8302D2ED000AB0EE600AFFF76FFB1A4890F88F11583000EB8100D0ED000AB0EE600A0020FDF79DFEFFF75CFB134890F88F11B03000EB13
:400F4000810080ED000A124A92F842100D4A92F88F0192F88F31B03202EB8302D2ED000AB0EE600AFFF719FB064890F88F11B03000EB8100D0ED000AB0EE600A0020FDF7B2
:400F80004FFE07E0C00F00200C11002000007A44301F0020FD4890F88F01002813D1FB4890F8880106280FD10320F84981F88801022081F88901B6EE000A084680ED3B0AA0
:400FC0000A2081F88F0182E0B7EE000AEF4880ED390A0920EE49087026E0EC485830EC4991F9001000EB810090ED000ADFEDE90AB4EEE00AF1EE10FA10D2E54890F900009E
:4010000000EE100AB8EEC00AF2EE040A20EE200ADE4880ED390AFF20DD490870DC480078401E40B2DA490870D94890F900000028D3DAB7EE000AD54880ED380A0920D449B8
:40104000087026E0D1482C30D14991F9001000EB810090ED000ADFEDD00AB4EEE00AF1EE10FA10DDCA4890F9000000EE100AB8EEC00AFAEE040A20EE200AC44880ED380AD2
:40108000FF20C3490870C2480078401E40B2C0490870BF4890F900000028D3DABB4890ED390A80ED3A0A0520B84981F888010D2081F88901B6EE000A084680ED3B0A00203B
:4010C00081F88F019FEDB50A084680ED370A0020AE49086000E000BF00BF9BE100BFAB4890F8890106281CD00D2802D00E287DD131E0FFF7E7F99FEDA70A10F04EF878B14B
:40110000B6EE000AA14880ED3B0A06209F4981F889010E2081F88B0126F0EDFE9B49086051E1B6EE000A994880ED3B0A014608684FF4FA7126F0E5FE60B1944890F88B0103
:40114000924981F88901002008600FF022FF8F4880ED080A37E18D4890F88801052807D10FF017FF8948D0ED080A70EE608A06E00FF00FFF8548D0ED080A70EEC08A834891
:40118000006818B926F0B7FE804908609FED840AF4EEC08AF1EE10FA7EDD7C4890ED370AD0ED3B0A30EE200A80ED370A90F88F01401C764981F88F01B6EE000A084680ED51
:4011C0003B0A0D2081F88901086826F0BCFE00EE100AB8EE400A5FED930A80EE209A6B4890F88801052818D1684800E0EAE090ED3A0A30EE090AF1EE040A30EE600A80ED29
:401200003A0A90ED3A0AB5EEC00AF1EE10FA1AD29FED620A80ED3A0A15E05C4890ED3A0A30EE490AF1EE040A30EE200A80ED3A0A90ED3A0AB5EEC00AF1EE10FA03DD9FED8A
:40124000570A80ED3A0A514890F88F01032839DB4E48D0ED370A90F88F0100EE100AB8EE400A80EE801A494880ED371A90F88801052828D14B4991F842004449D1ED370A4F
:40128000B0EE600A0DF0CCFE9FED440A3F4880ED370AB6EE000A00E031E080ED3B0A00203A4981F88F01022081F888010D2081F8890126F020FE35490860084690ED380AD8
:4012C00080ED3A0A7DE0374991F842002F49D1ED370AB0EE600A0DF06FFE9FED300A2B4880ED370AB6EE000A80ED3B0A0820274981F888010F2081F8890162E089E0234883
:4013000090ED3B0AB0EEC00ADFED270AB4EEE00AF1EE10FA07DA0146086826F014FE4EF66021884207D92120184981F88601092081F8880145E0154890F88801022817D170
:401340001249086826F0FFFD00EE100AB8EE400AFFEE000A60EE200A1FEDF41A80EE810A0A48D0ED3A0A30EE200A80ED3B0A28E00649086826F0E7FD00EE100AB8EE400A10
:40138000F7EE000A60EE200A10E00000C00F00204003002035FA0E3D35FA0EBD0000000035FA8E3C301F002000008C429FEDFE1A80EE810AFD48D0ED3A0A30EE200A80ED42
:4013C0003B0A00E000BF00BF24E002241FED0D0AF64880ED3B0A1DE0FFF766F8F34890F8860120B10920F14981F8880110E0F04991F84200FEF77FFE1020EC4981F889016E
:4014000003241FED1A0A084680ED3B0AFDF74DFE00E000BF00BFE54890F88A01E34991F88911884214D0E14890F88D01401CDF4981F88D01084690F88D01642802DD64205E
:4014400081F88D01D94890F88901D84981F88A01D64890ED3B0AB5EEC00AF1EE10FA08D0D0ED3B0AB0EE600A01210846F8F78FFF08E0CE48D0ED3B0AB0EE600A00210120BE
:40148000F8F785FF2046BDEC048B10BD10B52DED088BB0EE408AFAF7A8FA18B313F096FE00EE100AB8EE400A38EE400A10EE104A204630F0BBFE41EC1B0BB0EE4B0AF0EE5C
:4014C0006B0A2DF08DFAB0EE40AAF0EE60AA9FEDB90B53EC102B51EC1A0B30F059F941EC100B0BE018EE100A30F0A0FE41EC1A0BB0EE4A0AF0EE6A0A2DF072FAB0EE409A1D
:40150000F0EE609A51EC190B30F054F800EE100ABDEC088B10BD2DE9F0412DED068B0426FAF763FA08B1A54800E0A5480446FAF75CFA08B1A34800E0A34807469B4890F860
:4015400088010A2872D2DFE800F00506497171487171FDFC00BF954890F8890110B1102810D000BF1020914981F88901A0478F4880ED090AB6EE000A80ED3B0A00208B4977
:40158000086028E00520894981F88801A047B0EE40AAFFF77BFF854880ED0A0A0D20834981F88901B6EE000A084680ED3B0A002081F88F0126F09FFC7C4908601FED890A45
:4015C000084680ED370A1FED8B0A80ED3A0A002081F88D0100BF00BF4FE200BF734890F8890106284FD00D2802D00E2870D163E0FEF768FFA047B0EE40AAFFF747FFB0EE88
:40160000409AB0EE000AB84788B1B6EE000A674880ED3B0A0620654981F889010E2081F88B0126F068FC614908602BE024E2FAF7DCF908B1052000E00A2000EE100AB8EEDE
:40164000C00A5A48D0ED0A0A79EE600AB4EEE00AF1EE10FA07D21E20544981F88601092081F888010EE05149086826F06CFC44F62061884206D921204C4981F8860109202F
:4016800081F8880198E1B6EE000A484880ED3B0A014608684FF4FA7126F033FC58B1434890F88B01414981F8890100200860A0473E4880ED090A7FE13C4890F88801052849
:4016C00007D1A0473948D0ED090A70EE608A06E071E1A0473548D0ED090A70EEC08A3348006818B926F007FC30490860FAF77DF910B1B3EE090A01E0B1EE040AB4EEE80AD2
:40170000F1EE10FA76D2294890F88F01002808DD264890ED370AD0ED3B0A30EE200A80ED370A224890F88F01401C204981F88F01B6EE000A084680ED3B0AA047B0EE40AA51
:4017400001E03BE141E1FFF7A1FE184880ED0A0A0D20164981F88901086826F0F4FB00EE100AB8EE400ADFED100A80EE208A0F4890F88F01012804D1B1EE040A28EE000AA0
:4017800003E0B6EE000A28EE000AB0EE408A26F0B2FB06490860084690F8880105282AD1084690ED3A0A11E000007A44C00F0020301F00200000000000005940C15202083D
:4017C00041B20008CF54020863B2000830EE080AF2EE040A30EE600A80ED3A0A90ED3A0AB5EEC00AF1EE10FA1BD29FEDFA0A80ED3A0A16E07BE0F84890ED3A0A30EE480A46
:40180000F2EE040A30EE200A80ED3A0A90ED3A0AB5EEC00AF1EE10FA03DD9FEDEE0A80ED3A0AED4890F88F01032844DDEA48D0ED370A90F88F0100EE100AB8EE400AB7EE17
:40184000001A30EE410A80EE801AE34880ED371A90F8880105282FD1E04991F84200DE49D1ED370AB0EE600A0DF0DAFB9FEDD90AD94880ED370AB6EE000A80ED3B0A002004
:40188000D54981F88F01A047B0EE40AAFFF7FEFDD14880ED0A0A0220CF4981F888010D2081F8890126F027FBCB4908609FEDC90A084680ED3A0A7DE0C84991F84200C64941
:4018C000D1ED370AB0EE600A0DF076FB9FEDC10AC14880ED370AB6EE000A80ED3B0A0820BD4981F888010F2081F8890162E0FAF77CF810B19FEDBA0A01E0BAEE040AB4EEB2
:40190000E80AF1EE10FA07DD1E20B34981F88601092081F888014DE0AF4890ED3B0AB0EEC00ADFEDB00AB4EEE00AF1EE10FA07DA0146086826F007FB4EF66021884207D91B
:401940002120A54981F88601092081F8880131E0A14890F88F0110B9B1EE040A01E0B6EE000AF0EE409A9C49086826F0ECFA00EE100AB8EE400A20EE290A5FED750A80EE7B
:40198000201A954880ED3B1A90F88801022808D1914890ED3B0AFFEE000A20EE200A80ED3B0A8D4890ED3B0AD0ED3A0A30EE200A80ED3B0A00E000BF00BF5EE002269FEDDC
:4019C000850A854880ED3B0A57E0834890F8860120B10920804981F888014CE06425A8467E4991F84200694200EE101AB8EEC00A0DF0C2F9794991F84200694200EE101A93
:401A0000B8EEC00A0DF030FB744991F8420000EE105AB8EE400A0DF00AFA704991F8420000EE105AB8EE400A0DF043FB6B4890F8421040460DF071F8684890F842104046AD
:401A40000DF05CFB654890F8421040460DF098F8624890F8421040460DF06FFB10205E4981F8890103269FED5B0A084680ED3B0AFDF71BFB00BF00E000BF00BF564890F8C6
:401A80008A01554991F88911884214D0524890F88D01001D504981F88D01084690F88D01642802DD642081F88D014B4890F88901494981F88A01484890ED3B0AB5EEC00A6B
:401AC000F1EE10FA08D0D0ED3B0AB0EE600A01210846F8F75CFC08E03F48D0ED3B0AB0EE600A00210120F8F752FC3046BDEC068BBDE8F081002070479FED360A364880ED18
:401B00005D0A9FED340A80ED5F0A9FED320A80ED570A9FED300A80ED550A9FED2E0A80ED5B0A9FED2C0A80ED590A704770B52DED048B0446F0EE408AB0EE609AF0EE419A86
:401B40000D46264890F8300070280CD1F7EE000A80EEA80A5FEDEC0A89EE201A20EE010A20EE298A6EE01D4890F830000A280CD1F0EE000A80EEA80A5FEDF50A89EE201A1D
:401B800020EE010A20EE298A5CE0A81E0C284BD2DFE800F03B4A064A132E4A4A4A4A3D3CF0EE080A80EEA80ADFED0F0A89EE201A20EE010A20EE298A43E0DFED0C0A80EE97
:401BC000A80ADFED090A89EE201A20EE010A20EE298A36E000000000C00F0020301F00200000FAC30000A04200007A44CDCC4C40DFEDFD0A80EEA80A5FED050A89EE201AD4
:401C000020EE010A20EE298A1BE000BF00BFDFEDF70A80EEA80A5FED0C0A89EE201A20EE010A20EE298A0CE0DFEDF10A80EEA80A5FED130A89EE201A20EE010A20EE298AB0
:401C400000BF00BFB2EE040AB4EEC08AF1EE10FA04D2B2EE040AB0EE408A0AE09FEDE50AB4EEC08AF1EE10FA03DD9FEDE20AB0EE408A012C0AD1E04A92F84210BCEEC80AF3
:401C800010EE102AD0B20DF039FA09E0DA4A92F84210BCEEC80A10EE102AD0B20DF04DFABDEC048B70BD00B52DED028B95B0D34890ED3B0A8DED140A26F01DF90E9004206E
:401CC0000C900FF0E3F8CD4880ED3D0AC068CB494861084600698861C948007828F0B1F8C649C86026F007F9C4490861084680690B9026F028F94FF47A71B1FBF0F00F90B1
:401D0000BE48C068BD494969401A00EE100AB8EEC00AF7EE000A20EE200A9FEDBA1AC0EE010A9DED0F0AB8EEC00A20EE800A8DED130A0521B4489DED130A14F097F90521E6
:401D4000B14808309DED140A14F090F91DF03DF98DED0B0A1E21AC4818389DED0B0A14F085F9AA4890ED000A8DED0B0A1E21A64820389DED0B0A14F079F9A44890ED000A72
:401D80009E4880ED3C0AA248007810F0ADFA8DED0B0A05219C4808389DED0B0A14F066F99C48007810F05DFC8DED050A059830F03DFACDE906019DED060B2CF011FE8DED77
:401DC000080B9DED080B51EC100B2FF0F3FB05210B908D4810389DED0B0A14F047F98648B0F8BE014FF4967190FBF1F000EE100AB8EEC00A8DED0D0A7F4890F82800062874
:401E000031D07D4890F8280007282CD07B4890F88801042804D0794890F88801072822D1764890ED5F0ADFED7C0AB4EEE00AF1EE10FA19DD90ED5D1A9DED0D0AF2EE040A55
:401E4000F1EE041A41EEC00AB4EEE01AF1EE10FA79D20920694981F88801242081F88601002081F889016EE0644890ED5F0ADFED6B0AB4EEE00AF1EE10FA19D290ED5D1AE3
:401E80009DED0D0AFAEE040AF1EE041A41EE800AB4EEE01AF1EE10FA55DD0920574981F88801242081F88601002081F889014AE05248D0F87C01079030F0B8F9CDE90801BC
:401EC0009DED080B2CF08CFD8DED0A0B9FED540B53EC102B9DED0A0B51EC100B2FF0B0FD31D1DDED0D0AB1EE040AB1EE041A01EE200A8DED070A079830F098F9CDE90A01E7
:401F00003E48D0F87401059030F090F9CDE906019DED060B2CF064FD8DED080B9DED0A0B53EC102B9DED080B51EC100B2FF086FF09D20920314981F88801242081F88601C8
:401F4000002081F889012D4890F88901062813D12A48806801460B900E9826F003F827494968884241F2C983244890F88B01234981F8890101F0C1BB204890F888010A2841
:401F800081F0B983DFE810F050000A0060003504B70B39022807B70BAD0B980B174890F8870180B1154890F88701144981F88801062081F88901002081F88B0119204860D6
:401FC0000E9888600EE000200C4981F88801062081F88901002081F88B014FF47A7048600E98886001F088BB6666A6408FC2753E9A99193F00007F43301F0020C00F0020A8
:40200000E806002052EC2F4534110020402A0020A3060020F406002000004842000048C200000000000020400220FC4981F88801062081F88901002081F88B014FF47A7036
:4020400048600E988860CDE7F44890F88801F34981F88701084690F8890108287ED003DC38B105287BD13FE1092879D00B28F9D10BE00620E94981F889010B2081F88B01C0
:40208000192048600E988860B5E1E448806801460B900E9825F066FF41F28831884207D90920DE4981F88801262081F8860170E0DB4890F8280006280ED0D94890F82800D7
:4020C000072809D0D54890ED3D0ADFEDD60AB4EEE00AF1EE10FA13DCD14890F82800062804D0CF4890F8280007280FD1CB4890ED3D0ADFEDCD0AB4EEE00AF1EE10FA05DD75
:40210000BBEE0E0AC54880ED3B0A42E0C44890F8280006280ED0C24890F82800072809D0BE4890ED3D0ADFEDC10AB4EEE00AF1EE10FA17D3BA4890F82800062804D0B848FF
:4021400090F82800072813D1B44890ED3D0ADFEDB80AB4EEE00AF1EE10FA02E032E043E118E005D2B3EE0E0AAC4880ED3B0A10E00620AA4981F88901092081F88B014FF416
:402180007A7048600E9888609FEDAA0A084680ED3B0A30E10620A14981F88901082081F88B01192048600E988860BAEE000A084680ED3B0AA048007827F043FE9749C1F8FC
:4021C000340118E1964890F82800062804D0944890F82800072810D19048C0688F49D1F83411401A00EE100AB8EEC00ADFED930AB4EEE00AF1EE10FA31D3894890F8300062
:402200000A2800D010E08548C0688449D1F83411401A00EE100AB8EEC00ADFED890AB4EEE00AF1EE10FA1AD37D4890F82800062836D07B4890F82800072831D07748C06816
:402240007649D1F83411401A00EE100AB8EEC00ADFED7A0AB4EEE00AF1EE10FA20D2704890F842000B909DED140A0CF0A5FE06206A4981F88901052081F88B014FF47A7071
:4022800048600E9888609DED140A084680ED3B0A6948007827F0D5FD6049C1F8340122E05E4890ED3B0A5FEDA30AB4EEE00AF1EE10FA0BD89FED5F0A80ED3B0A092057496C
:4022C00081F88801272081F886010CE09DED140ADFED5C0A30EE600A8DED140A9DED140A4E4880ED3B0A86E04C48D0ED3B0A9FED561A80EE810A8DED010A01982FF096FFFC
:40230000CDE902019DED020B2CF06AFB8DED060B4248D0F86C0103902FF088FFCDE904019DED060B53EC102B9DED040B51EC100B2FF086FC9FED450B53EC102BCDE90801D2
:402340009DED080B51EC100B2FF022FACDE90A019DED0A0B51EC100B2FF02CF92F49C1F80401084690ED590ADFED3A0A80EE201A80ED451A2A4890F830000A2804D1B3EE77
:40238000090A8DED100A03E0B1EE040A8DED100A9DED100ADFED300A80EE201A9FED2F0A21EE000ABDEEC00AB8EEC00A1B4880ED490AB0F8840140F004001849A1F884013A
:4023C000052081F88801062081F88901002081F88B014FF47A7048600E9888609FED150A084680ED3B0A06E000200C49A1F8840181F8880100BF00BFF4E5084890F8880127
:40240000064981F88701084690F88901082879D026DC10B1052876D162E126E0C00F0020301F0020CDCCCC3CCDCC4C3DCDCCCCBCCDCC4CBD00000000E80600206CE7DBC50E
:402440007390EAC4CDCCCC3D0000C8420000000000408F4000007A44000070428DED244809287DD00B28D6D10BE00620F94981F889010B2081F88B01192048600E9888604D
:40248000B5E1F448806801460B900E9825F06AFD41F28831884207D90920EE4981F88801282081F8860170E0EB4890F8280006280ED0E94890F82800072809D0E54890ED4C
:4024C0003D0A5FED280AB4EEE00AF1EE10FA13DCE14890F82800062804D0DF4890F82800072811D1DB4890ED3D0A5FED310AB4EEE00AF1EE10FA07DDBBEE0E0AD54880EDDE
:402500003B0A42E05AE06BE1D34890F8280006280ED0D14890F82800072809D0CD4890ED3D0A5FED3E0AB4EEE00AF1EE10FA13D3C94890F82800062804D0C74890F82800BC
:40254000072811D1C34890ED3D0A5FED470AB4EEE00AF1EE10FA07D2B3EE0E0ABD4800E014E080ED3B0A10E00620BA4981F88901092081F88B014FF47A7048600E9888609F
:402580001FED540A084680ED3B0A30E10620B14981F88901082081F88B01192048600E988860B2EE000A084680ED3B0AAB48007827F047FCA749C1F8340118E1A64890F825
:4025C0002800062804D0A44890F82800072810D1A048C0689F49D1F83411401A00EE100AB8EEC00ADFED9E0AB4EEE00AF1EE10FA31DC994890F830000A2800D010E09548CF
:40260000C0689449D1F83411401A00EE100AB8EEC00ADFED940AB4EEE00AF1EE10FA1ADC8D4890F82800062836D08B4890F82800072831D08748C0688649D1F83411401A46
:4026400000EE100AB8EEC00ADFED850AB4EEE00AF1EE10FA20DD804890F842000B909DED140A0CF0DDFC06207A4981F88901052081F88B014FF47A7048600E9888609DED68
:40268000140A084680ED3B0A7448007827F0D9FB7049C1F8340122E06E4890ED3B0ADFED720AB4EEE00AF1EE10FA0BDB1FED9F0A80ED3B0A0920674981F88801292081F815
:4026C00086010CE09DED140A5FEDA20A30EE200A8DED140A9DED140A5E4880ED3B0A86E05C48D0ED3B0A1FEDA81A80EE810A8DED010A01982FF09AFDCDE902019DED020BF0
:402700002CF06EF98DED060B5248D0F86C0103902FF08CFDCDE904019DED060B53EC102B9DED040B51EC100B2FF08AFA1FEDB90B53EC102BCDE908019DED080B51EC100B1F
:402740002FF026F8CDE90A019DED0A0B51EC100B2EF030FF3F49C1F80C01084690ED590A5FEDC40A80EE201A80ED471A3A4890F830000A2804D1B3EE090A8DED100A03E09F
:40278000B1EE040A8DED100A9DED100A5FEDCE0A80EE201A1FEDCF0A21EE000ABDEEC00AB8EEC00A2B4880ED4B0AB0F8840140F020002849A1F88401032081F888010620F9
:4027C00081F88901002081F88B014FF47A7048600E9888601FEDE90A084680ED3B0A06E000201C49A1F8840181F8880100BF00BF29E4184890F88801164981F8870108461A
:4028000090F8890130B1052879D0072878D00A2877D10BE006200F4981F889010A2081F88B01192048600E988860D3E20948806801460B900E9825F095FB42F2107188429A
:4028400014D90920034981F88801262081F88601C8E00000C00F0020301F0020E80600206CE7DB457390EA4400004842FE4890F8280006280ED0FC4890F82800072809D06E
:40288000FA4890ED3D0ADFEDFA0AB4EEE00AF1EE10FA13DCF44890F82800062804D0F24890F8280007282DD1F04890ED3D0ADFEDF10AB4EEE00AF1EE10FA23DDEA4890F8E7
:4028C0002800062804D0E84890F8280007280BD100BFE54890ED300AF0EE040A30EE600AE24880ED3B0A7DE0DF4890ED300AF2EE0E0A30EE600ADD4880ED3B0A72E072E09A
:402900000BE260E2D84890F8280006280ED0D64890F82800072809D0D448D0ED3D0A9FEDD60AF4EEC00AF1EE10FA13D3CE4890F82800062804D0CC4890F8280007282AD1F9
:40294000CA4890ED3D0ADFEDCA0AB4EEE00AF1EE10FA20D2C44890F82800062804D0C24890F8280007280BD100BFBF4890ED320AF0EE040A30EE200ABC4880ED3B0A31E07D
:40298000B94890ED320AF2EE0E0A30EE200AB74880ED3B0A26E00620B44981F88901052081F88B0140F6B83048600E988860AE4890F8280007280AD1AB48D0ED320A9FED9A
:4029C000AF0A20EE800A084680ED3B0A04E09FEDAC0AA64880ED3B0A0020A449C1F83401C1F84001F6E1A148D0F83401D0BBA548007827F026FA9D49C1F83401084690ED48
:402A0000550A80ED4E0A90ED570A80ED4F0A062081F88901072081F88B01934890F82800072803D14FF47A70486003E04FF47A708E4948608D490E9888608B4890F82800A0
:402A4000062804D0884890F8280007280BD1864890ED300AF2EE0E0A30EE600A834880ED3B0A59E10AE0804890ED300A5FED820A30EE600A7D4880ED3B0A4DE17B48D0F814
:402A8000400100287DD17F48007827F0DAF97749C1F84001084690ED550A80ED510A90ED570A80ED520AD0F84001D1F83411401A0B9013F047FD00EE100AF8EE400A9FEDCC
:402AC000720A20EE800ADFED700A80EE201A674880ED4A1AD0F840016449D1F83411401A00EE100AB8EEC00ADFED680AB4EEE00AF1EE10FA7DD25C4890F82800062804D066
:402B0000594890F82800072804D19FED610A8DED130A04E0554890ED570A8DED130A524890F82800072839D1504890F88C010B904D4890ED0F0A8DED0A0A4C4890ED510ACC
:402B40008DED090A0B989DED0A1ADDED130A9DED090A0DF071FA454880ED400A90F88C010B90414890ED0F0A8DED0A0A3F4890ED4E0A8DED090A0B989DED0A1ADDED130AC9
:402B800000E0C9E09DED090A0DF056FA3748D0ED400A30EEC00A80ED400A38E0334890F88C010B90304890ED0F0A8DED0A0A2F4890ED510A8DED090A0B989DED0A1ADDEDA7
:402BC000130A9DED090A0DF037FA284880ED400A90F88C010B90244890ED0F0A8DED0A0A224890ED4E0A8DED090A0B989DED0A1A00E085E0DDED130A9DED090A0DF01CFA8D
:402C00001A48D0ED400A30EEC00A80ED400A174890F88C010B90154890ED420AB1EE400A8DED0A0A90ED400A8DED090A0B999DED0A1ADFED150A9DED090A0120FEF776FF27
:402C40000A4890ED400AF7EE000A80EE201A9FED0C0A31EE408A0F4800780FF045FBDFED0A0A80EE201A17E0301F0020C00F0020CDCCCC3DCDCC4C3ECDCC4C3D9A99193FBC
:402C800000000000E806002000007A44FF4680C639B40040A3060020FE4890ED420AB1EE400AC0EE010AFC4890ED300A9FEDFB1A10EE810AC8EE000AF648C0ED3E0AB0F856
:402CC000840140F00800F349A1F884010846B0F8840140F01000A1F88401062081F8880181F88901002081F88B014FF47A7048600E9888601FED1E0A084680ED3B0A0BE012
:402D00001FED210AE34880ED3B0A0920E14981F888012B2081F886015CE00620DD4981F88901052081F88B010A2048600E9888600846D0ED3B0A9FEDD91A80EE810A8DED88
:402D4000010A01982FF072FACDE902019DED020B2BF046FE8DED060BCE48D0F86C0103902FF064FACDE904019DED060B53EC102B9DED040B51EC100B2EF062FF9FEDC80BF0
:402D800053EC102BCDE908019DED080B51EC100B2EF0FEFCCDE90A019DED0A0B51EC100B2EF008FCBB49C1F80801084690ED590A5FED4B0A80EE201A80ED461ABAEE000A37
:402DC00080ED3B0A06E00020B249A1F8840181F8880100BF00BFFDE3AE4890F88801AD4981F88701084690F8890130B105287CD007287BD00A287AD10BE00620A54981F87B
:402E000089010A2081F88B01192048600E988860F3E3A048806801460B900E9825F0A2F842F21071884207D909209A4981F88801282081F88601BCE0974890F8280006287F
:402E40000ED0954890F82800072809D0914890ED3D0ADFED950AB4EEE00AF1EE10FA13D38D4890F82800062804D08B4890F8280007282AD1874890ED3D0ADFED8C0AB4EEB1
:402E8000E00AF1EE10FA20D2834890F82800062804D0814890F8280007280BD100BF7E4890ED320AF0EE040A30EE200A794880ED3B0A7EE0784890ED320AF2EE0E0A30EE7A
:402EC000200A744880ED3B0A73E0734890F82800062812D0704890F8280007280DD06D4890ED3D0ADFED720A02E063E086E3D5E3B4EEE00AF1EE10FA13DC674890F828002E
:402F0000062804D0644890F8280007282AD1614890ED3D0ADFED640AB4EEE00AF1EE10FA20DD5D4890F82800062804D05A4890F8280007280BD100BF574890ED300AF0EE49
:402F4000040A30EE600A534880ED3B0A31E0524890ED300AF2EE0E0A30EE600A4D4880ED3B0A26E006204B4981F88901052081F88B0140F6B83048600E988860464890F8EE
:402F8000280007280AD1444890ED300A5FEDC50A20EE200A084680ED3B0A04E01FEDC80A3C4880ED3B0A00203A49C1F83401C1F840017FE33748D0F83401D0BB3D48007860
:402FC00026F03FFF3349C1F83401084690ED550A80ED4E0A90ED570A80ED4F0A062081F88901072081F88B012B4890F82800072803D14FF47A70486003E04FF47A702549B2
:40300000486024490E988860234890F82800062804D0214890F8280007280BD11E4890ED320AF2EE0E0A30EE200A1A4880ED3B0AE3E20AE0184890ED320ADFED1F0A30EE5E
:40304000200A144880ED3B0AD7E21248D0F840010028EDD11748007826F0F3FE0D49C1F84001084690ED550A80ED510A90ED570A80ED520AD0F84001D1F83411401A0B9043
:4030800013F060FA4FF47A71B0FBF1F000EE100A14E00000C00F0020301F00200000C8420000000000408F40CDCCCCBDCDCC4CBECDCC4CBDE806002000004842B8EE400A97
:4030C000DFEDFE0A20EE200AFD4880ED4C0AD0F84001FB49D1F83411401A00EE100AB8EEC00ADFEDF80AB4EEE00AF1EE10FA7DDDF54890F82800062804D0F34890F8280018
:40310000072804D19FEDF10A8DED130A04E0EC4890ED570A8DED130AEB4890F82800072837D1E74890F88C010B90E74890ED0F0A8DED0A0AE24890ED510A8DED090A0B9862
:403140009DED0A1ADDED130A9DED090A0CF074FFDB4880ED400A90F88C010B90DA4890ED0F0A8DED0A0AD64890ED4E0A8DED090A0B989DED0A1ADDED130A9DED090A0CF08D
:403180005BFFCF48D0ED400A30EEC00A80ED400A38E0CB4890F88C010B90CB4890ED0F0A8DED0A0AC64890ED510A8DED090A0B989DED0A1ADDED130A9DED090A0CF03CFF67
:4031C000BF4880ED400A90F88C010B90BE4890ED0F0A8DED0A0ABA4890ED4E0A8DED090A0B989DED0A1ADDED130A00E0F9E19DED090A0CF021FFB248D0ED400A30EEC00A3F
:4032000080ED400AAE4890F88C010B90AC4890ED440A8DED0A0A90ED400A8DED090A0B999DED0A1ADFEDA50A9DED090A0220FEF77DFCA34890ED400AF7EE000A80EE201A4D
:403240009FEDA30A31EE408AA24800780FF04CF8DFED9A0A80EE201A994890ED440AC0EE010A994890ED320A1FED741A10EE810AC8EE000A9248C0ED3F0AB0F8840140F060
:4032800040008F49A1F884010846B0F8840140F08000A1F884010846D0ED410A90ED430A30EE800A80ED410A90ED410AF0EE000A80EE201A80ED411AD0ED420A90ED440A1B
:4032C00030EE800A80ED420A90ED420AF0EE000A80EE201A80ED421AD0ED450A90ED470A30EE800A80ED450A90ED450AF0EE000A80EE201A80ED451A90ED460AD0ED480A09
:4033000030EE200A80ED460A90ED460AF0EE000A80EE201A80ED461A90ED490AD0ED4B0A30EE200A80ED490A90ED490AF0EE000A80EE201A80ED491A90ED490ADFED660A38
:4033400020EE200A80ED490A90ED4A0AD0ED4C0A30EE200A80ED4A0A90ED4A0AF0EE000A80EE201A80ED4A1A90ED4A0ADFED5A0A20EE200A80ED4A0A90ED460AD0ED450A63
:4033800070EE600A90ED420A90ED411A30EE411A80EE810A8DED0B0A9DED0B0A09F083F9474890ED460A4848D0ED700A444890ED421A00EEC10A8DED0B0A9DED0B0A09F027
:4033C00058F93F4890ED4A0AD0ED490A70EE600A90ED420A90ED411A30EE411A80EE810A8DED0B0A9DED0B0A09F029F9344890ED4A0A3548D0ED720A314890ED421A00EEAD
:40340000C10A8DED0B0A9DED0B0A09F0FEF8314800780EF069FFDFED290A80EE201A2A4890ED700A21EE000AD0ED710AB2EE001A71EE600A80EE801A1FEDE80A21EE000A4A
:403440008DED130A90F82800062804D19FED230A8DED110A0DE01C4890F830000A2804D19FED1E0A8DED110A03E09FED1D0A8DED110A1348D0ED3E0A9DED110A80EE201A83
:40348000114890ED300A31EE400A8DED120A9DED130ADFED140AB4EEE00AF1EE10FA29DD9DED120ADFED0F0AB4EEE00AF1EE10FA20DD90F842009FED0C0A17E000007A44D3
:4034C000C00F0020FF468046301F002039B4004000000000A30600205F43BA393333B33F3333B33E0000C8420000C8C20B900BF0BBFD1DE09DED130ADDED120AB4EEE00A31
:40350000F1EE10FA0ADDF74890F842000B909DED120AB1EE400A0BF0A7FD09E0F14890F842000B909DED130AB1EE400A0BF09CFDED48D0ED3F0A9DED110A80EE201AE94885
:4035400090ED320A31EE000A8DED120A9DED130A5FED1C0AB4EEE00AF1EE10FA10DD9DED120A5FED200AB4EEE00AF1EE10FA07DD90F842001FED250A0B900BF09AFD19E0B8
:403580009DED130ADDED120AB4EEE00AF1EE10FA08DDD44890F842000B909DED120A0BF088FD07E0CF4890F842000B909DED130A0BF07FFD0820CC4981F88801062081F81E
:4035C0008901002081F88B014FF47A7048600E98886000E090E01FED420A084680ED3B0A0BE01FED450AC04880ED3B0A0920BE4981F888012B2081F886015BE00620BA4930
:4036000081F88901052081F88B010A2048600E9888600846D0ED3B0A1FED4E1A80EE810A8DED030A03982EF001FECDE904019DED040B2BF0D5F98DED080BAB48D0ED5B0A22
:403640001FED621A80EE810A8DED050A05982EF0EDFDCDE906019DED080B53EC102B9DED060B51EC100B2EF0EBFACDE90A019DED0A0B51EC100B2DF09DFF9B49C1F81001B2
:40368000084690ED590A5FED730A80EE201A80ED481AB2EE000A80ED3B0A0BE000209249A1F8840181F888011FED770A084680ED3B0A00BF00BF1FE002200C9006208A4979
:4036C00081F88901002081F88B01192048600E9888601FED810A084680ED3B0AFEF70CFA0AE003200C901FED860A7F4880ED3B0AFBF7DBFC00E000BF00BF7B4890ED3B0A37
:40370000B5EEC00AF1EE10FA0AD090ED3B0A8DED0B0A012108469DED0B0AF6F738FE0AE0714890ED3B0A8DED0B0A002101209DED0B0AF6F72CFE0C9815B0BDEC028B00BD8E
:4037400010B50124684890F8860170BB22F016F868B1644991F83000F8F725F918B1FDF7DAFE04461FE0FEF79EFA04461BE022F01DF8C0B15B4890F82800072803D1FEF736
:40378000B9F904460FE0F8F721F928B9554991F83000F8F708F918B1FDF7BDFE044602E0FDF72AF90446FBF714FB204602F0E5F94D4890F8860120B14B4991F8860102F0A6
:4037C000E5FE204610BD10B5474890F888010A284CD2DFE800F04C4D20054B21064B4B4E00BF0220404981F88901002008600DF0D0FB3D4880ED080A90F88F01401C3A497B
:4038000081F88F01084690F88F010A2802DD0A2081F88F0130E000BF0D20334981F8890124F069FB304908601FEDD70A084680ED370A002081F88F01F8F7C8F870B12A48AD
:4038400090F88D01322804DD3220274981F88D010BE00020244981F88D0106E0224890F88D01C01E204981F88D0105E000BF00BF00BFFBF745FA00BF00BF1C480021C16480
:4038800001650020184981F88601B6EE000A084680ED3B0A10BD10B521F070FF50B302F071FE2B2802D1FBF72BFA26E00E4890F887010D4981F88801062081F889010020B3
:4038C00081F88B014FF47A70486024F014FB064988609FED070A084680ED3B0A002081F886010AE0301F0020C00F0020C010002000000000FFE7FFF766FF10BDB7EE000AE2
:4039000070475B4890F88601704710B55948FCF767FB5848FCF7E9FA5648FBF7DCFB10BD10B55448FCF75CFB5248FCF7DEFA5148FBF7D1FB10BD4E4890F8880170474C48DC
:4039400090F88901704710B50424494890F88801012804D10620464981F8880186E04FF4FA714548008824F0CCFA00287ED024F0C2FA414908803E4890F88801801E07287B
:4039800072D2DFE800F0450571440471700000BF374890F88901801E0B2835D2DFE800F00634151F0B1A3434343410000620304981F8890129E00C202D4981F8890124E082
:4039C00004202B4981F889011FE00720284981F889011AE00520264981F8890115E0244890F88801062807D10320214981F88801022081F8890106E005201D4981F8880162
:403A00000D2081F8890100E000BF00BF2DE000BF174890F88901062804D00D2807D00E281ED109E00D20124981F8890119E00E200F4981F8890114E00D4890F8880105280B
:403A400009D102200A4981F88801062081F8890105E00BE008E00820054981F8880100E000BF00BF01E000E000BF00BF204610BDC00F0020501100204C03002010B50446DE
:403A800021F07CFE00287DD0092C7CD005DC4CB1032C31D0062C77D158E00B2C75D00C2CF9D1E5E00120FE490870FA208861FA21FB48C16124F01FFAF94948620121F848A4
:403AC00080F82810D0ED080AB0EE600AF548007826F05CFA0020F24948604FF47A71F0488160416A0161002101759FEDEF0AEF48007826F04BFAF5E00120E9490870FA20E7
:403B00004860FA21E648816024F0F5F9E44908610121E3480175D0ED030AB0EE600AE348007826F033FA0020DD4988614FF47A71DB48C16101694162002180F828109FED94
:403B4000DA0AD848007826F021FACBE00120D44908704FF47A7088610021D148C16124F0CAF9CF4948620121CD4880F82810D0ED080AB0EE600ACB48007826F007FA0020AC
:403B8000C74903E0AFE011E0ABE03AE048604FF47A71C3488160416A0161002101759FEDC20AC248007826F0F1F99BE00120BC4908704FF47A7048600021B948816024F0A8
:403BC0009AF9B74908610121B5480175D0ED030AB0EE600AB548007826F0D8F90020B04988614FF47A71AE48C16101694162002180F828109FEDAC0AAA48007826F0C6F95F
:403C000070E00220A6490870642048600021A448816024F070F9A24908610121A0480175D0ED030AB0EE600AA048007826F0AEF964209B49886100219948C16101694162CF
:403C4000002180F828109FED980A9648007826F09DF90020924981F87C000121904880F87D10022180F88B10002180F88C1039E002208B4908704FF47A7048600146884876
:403C8000816024F038F986490861012184480175D0ED030AB0EE600A8448007826F076F94FF47A707E49886101467D48C16101694162002180F828109FED7B0A7948007874
:403CC00026F064F90020764981F87C000121744880F87D10022180F88B10002180F88C1000E000BFDDE221F061FD0028FAD0102C75D2DFE804F074083E75ABFA74E7E6E538
:403D0000E47474E3E2E10120654908704FF4FA70C86201466248016324F0EDF86049886301215F4880F83C106148007821F068FD00205B4948604FF47A7159488160816BE5
:403D40000161002101750020554908644FF47A7153484164816BC164002180F850105348007821F04DFD00215248007821F048FD96E201204A4908704FF4FA7008640146AD
:403D80004748416424F0B7F84549C8640121444880F850104748007821F032FD0020404948604FF47A713E488160C16C01610021017500203A49C8624FF47A71384801639A
:403DC000C16C8163002180F83C103848007821F017FD00213648007821F012FD60E25EE201202F4908704FF4FA70486001462C48816024F080F82A49086101212848017585
:403E00002A48007821F0FCFC0020254908644FF47A71234841640169C164002180F8501000201F49C8624FF47A711D48016301698163002180F83C101D48007821F0E0FC29
:403E400000211C48007821F0DBFC29E20120144908704FF4FA70C86201461148016324F04AF80F49886301210D4880F83C101048007821F0C5FC4FF4FA7009490864014659
:403E80000748416424F037F80549C8640121044880F850100748007821F0B2FC002013E070140020BD06002000000000BE060020150700200C070020B5E172E129E1EEE0D7
:403EC000B7E080E049E010E0F74948600021F648816024F010F8F44908610021F2480175F248007821F08CFCDAE10120EE4908703220C8623221EC48016323F0FCFFEA4979
:403F000088630121E84880F83C10E948007821F077FC3220E44908643221E348416423F0EAFFE149C8640121DF4880F85010E148007821F065FC0020DB4948600021DA4890
:403F4000816023F0D8FFD84908610021D6480175D648007821F054FCA2E10120D24908704FF47A70C8620021CF48016323F0C3FFCD4988630121CC4880F83C10CC480078BA
:403F800021F03EFC0020C84948604FF47A71C6488160816B0161002101750020C24908644FF47A71C0484164816BC164002180F85010BE48007821F023FC0021BD48007813
:403FC00021F01EFC6CE10120B74908704FF47A7008640021B448416423F08DFFB249C8640121B14880F85010B248007821F008FC0020AD4948604FF47A71AB488160C16C28
:404000000161002101750020A749C8624FF47A71A5480163C16C8163002180F83C10A348007821F0EDFB0021A148007821F0E8FB36E101209C4908704FF47A70486000217B
:404040009948816023F057FF974908610121964801759648007821F0D3FB0020924908644FF47A71904841640169C164002180F8501000208C49C8624FF47A718A48016304
:4040800001698163002180F83C108948007821F0B7FB00218748007821F0B2FB00E10120814908704FF47A70C86200217E48016323F021FF7C49886301217B4880F83C1029
:4040C0007B48007821F09CFB4FF47A707649086400217548416423F00EFF7349C8640121714880F850107348007821F089FB00206D49486000216C48816023F0FCFE6A498B
:4041000008610021684801756848007821F078FBC6E00220644908704FF47A70486000216148816023F0E7FE5F49086101215E48017500215D48007821F062FB4FF47A7096
:404140005949C86200215848016301698163012180F83C1000215648007821F051FB4FF47A705149086400214F4841640169C164012180F8501000214E48007821F040FBF2
:404180000020494981F87C000221474880F87D10032180F87E1080F88B10002180F88C107EE00220404908706420486000213E48816023F0A0FE3C49086101213A48017541
:4041C0003A48007821F01CFB64203749C86200213548016301698163012180F83C103448007821F00DFB64202F49086400212E4841640169C164012180F850102D48007812
:4042000021F0FEFA0020284981F87C000221264880F87D10032180F87E1080F88B10002180F88C103CE001201F4908704FF47A70486001461C48816023F05DFE1A4908612F
:4042400000211948017501211948007821F0D8FA4FF47A701449C86200211348016323F04AFE1149886301210F4880F83C101048007821F0C5FA00200B4908644FF47A7149
:404280000948416423F037FE0749C8640021064880F850100748007821F0B2FA00E000BF00BF0548047010BD70140020BE060020150700200C0700204E03002001B59DF8DA
:4042C000000000EE100AB8EE400AFE4880ED030A9DF8000000EE100AB8EE400AF94880ED080A00BF01226946F7480068403006F03DF920B99DF80000F44981F8400000BFC2
:404300000120F349087008BD08B506464FF4C8774FF000080121EF4880F8A8119421E94829F001FA307818B94620FFF7C7FF11E0E64890F84050642D03DD6420FFF7BEFF13
:4043400008E00A2D03DA0A20FFF7B8FF02E02846FFF7B4FF0020DB4981F88D0021F00EFAE8B10020FFF78AFBDB48DFEDDC0A9FEDDC0A01230022DB490090DB48007825F0E9
:4043800067FAD548DFEDD50A9FEDD50A01230022D6490090D648007825F05AFA05E021F005FA10B10120FFF769FB0321C94880F8A81100BF012239464FF6FF70DFF834C3FB
:4043C00000DF23F098FD0446BE4890F88D00002874D1012016F0C9FA18BB21F0CFF968B1C548007818B9BA480078012805D10020FFF744FB0020B64908709EE021F0D6F99C
:404400000028FAD0BC480078052803D1B04800780128F2D10520FFF731FB0020AC4908708BE001F0E5FA20BB21F0A8F970B1B2480078092803D1A648007801287DD1092077
:40444000FFF71CFB0020A249087076E021F0AEF9002872D0A8480078022803D19C48007801286AD10220FFF709FB00209849087063E021F083F970B19F480078062803D127
:4044800093480078012858D10620FFF7F7FA00208F49087051E021F089F928B396480078042803D18A480078012846D10420FFF7E5FA0020864908703FE0FFE7814890F8A5
:4044C0008D00012823D121F059F970B18A4800780C2803D17E48007801282ED10C20FFF7CDFA00207A49087027E021F05FF920B3814800780D2803D17548007801281CD1BA
:404500000D20FFF7BBFA00207149087015E06D4890F88D00022810D121F048F968B1764800780F2803D16A480078012805D10F20FFF7A4FA0020664908706248007801285D
:4045400002D002287ED115E15E48007D28BB5D48406810B35B480169204623F003FD5949896888423FD3012156480175046121F005F948B15348D0ED030AB0EE600A5C483B
:40458000007825F003FD2EE021F010F910B301215748007821F034F925E04A48007D012821D148488068A8B146480169204623F0D9FC44494968884215D3002141480175B6
:4045C000046121F0DBF830B19FED4C0A4848007825F0DCFC07E021F0E9F820B100214448007821F00DF9374890F82800C8B935488069B0B13348416A204623F0B3FC314995
:40460000C96988422BD301212E4880F828104462D0ED080AB0EE600A3348007825F0B6FC1DE0284890F82800012818D12548C069A8B12448416A204623F094FC2149896967
:40464000884200E0F6E10AD300211E4880F8281044629FED2A0A2448007825F097FC194890F85000A8B91748006C90B11548C16C204623F077FC1349496C884245D3012182
:40468000104880F85010C4641D48007821F0B8F83BE00C4890F85000012836D10948406C80B30848C16C204623F05CFC0549096C88422AD30021034880F85010C4641048C1
:4046C000007820E070140020B4030020301F00204F03002050410020C8D800200000FA4300247449001C0040BD06002000200040BE060020C10804084E030020000000008E
:404700000C07002001E021F07BF8D84890F83C00A8B9D648C06A90B1D448816B204623F021FCD249096B884223D30121CF4880F83C108463CE48007821F062F819E0CB483D
:4047400090F83C00012814D1C848006B88B1C748816B204623F006FCC449C96A884208D30021C24880F83C108463C148007821F047F85FE1BD4890F88C107C30405C78BBCD
:40478000BA48007D01282CD1B8480169204623F0E9FBB6494968884221D30021B3480175046120F0EBFF30B11FED2C0AB148007825F0ECFB0DE020F0F9FF50B11FED310A61
:4047C000AC48007825F0E2FB0021AA48007821F017F8A6488068002801D14FF00108C1E00BE0A2480169204623F0BCFB9F498968884201D34FF00108B4E09C4890F88C102D
:404800007C30405C01282BD1984890F8280001281AD19648416A204623F0A4FB93498969884210D30021914880F8281044621FED4D0A9148007825F0A9FB8C48C069002869
:4048400001D14FF001088DE08848416A204623F089FB8649C969884201D34FF0010881E0824890F88C107C30405C022836D17F4890F83C00012825D17C48816B204623F0B7
:4048800071FB7A49C96A88426CD30021774880F83C1084637648007820F0B2FF20F086FF50B100217248007820F0AAFF1FED6D0A6F48007825F06AFB6C48006B90BB4FF094
:4048C00001084FE06948816B204623F04BFB6749096B884246D34FF0010843E0634890F88C107C30405C03283CD1604890F8500001282CD15D48C16C204623F033FB5B49A0
:40490000096C88422ED30021584880F85010C46420F034FF38B11FED870A5748007825F035FB0EE01EE020F041FF50B11FED8D0A5248007825F02AFB00215048007820F0E4
:404940005FFF4A48406C68B94FF001080AE04748C16C204623F006FB4449496C884201D34FF00108B8F1010F63D14FF000083F4890F88C00401CC1B23C4880F88C1090F82C
:404980008C1090F88B00814203DB0021374880F88C10364890F88C107C30405C022809D10121324880F83C1084633148007820F027FF3EE02D4890F88C107C30405C01286F
:4049C0000DD10121294880F828104462D0ED080AB0EE600A2848007825F0D8FA29E0234890F88C107C30405C032809D101211F4880F85010C4642148007820F001FF18E0F3
:404A000001211A480175046120F0B8FE48B11748D0ED030AB0EE600A1648007825F0B6FA07E020F0C3FE20B101211248007820F0E7FE00BFBEE42DE9F04106460C46174677
:404A40009846069D2078642803DD6420FFF736FC09E020780A2803DA0A20FFF72FFC02E02078FFF72BFCBDE8F08100007014002015070020BE060020BD0600200C070020A3
:404A800070B541201CE0C41700EBD4646511CD4C54F82540C51700EBD5656D11A0EB45160125B5402C40C51700EBD5656D11A0EB45160125B540AC4200D103E0411EC8B24F
:404AC0000028E0DC00BF70BD30B5C31700EBD3635C11BC4B183353F824300246C41700EBD4646411A0EB44150124AC4023430146C41700EBD4646511B24C183444F82530FC
:404B000030BD13B50C4600BFAF49096801F5B07108190122694605F029FD18B99DF80010AA48015500BF1CBD13B50C4600BFA649096801F25F2108190122694605F016FD24
:404B400020B99DF80010A148FF30015500BF1CBD70B504469E480470E21704EBD2625311984A52F823202146E31704EBD3635B11A4EB43150123AB409A432046E31704EBE5
:404B8000D3635D118F4B43F82520E21704EBD26253118C4A0C3252F82320E31704EBD3635B11A4EB43150123AB409A43E31704EBD3635D11834B0C3343F82520E21704EB76
:404BC000D26253117F4A183252F82320E31704EBD3635B11A4EB43150123AB409A43E31704EBD3635D11774B183343F825200020FFF79AFF70BD30B50146CB1701EBD363F9
:404C00005C11704B53F82430CC1701EBD4646411A1EB44150124AC4023400BB1012030BD0020FCE76B49087070476A480078704770B52DED048B04460025422C70D2DFE893
:404C400004F02122272C2D2E2F37424D586069737F88A3A8BBFEFDFCFBFAF9F8F7F6F5F4F3F2F1F0EFEEEDECEBEAE9E8E7E6E5E4E3E2E1E0DFDEDDDCDBDAD9D8D7D6D5D496
:404C8000D3D2D194F2E20EF0B3FE80F00105EDE220F06CFD80F00105E8E2E7E2E6E2E5E2F8F7DFFA08B1012000E000200546DDE20FF02BFD30B1F8F7CCFA08B1012000E0EE
:404CC00000200546D2E20FF020FD30B1F8F7D9FA08B1012000E000200546C7E20FF015FD30B1F8F7C6FA08B1012000E000200546BCE20CF0ADFA012800D100E000200546BC
:404D0000B4E20CF0A5FA032801D1012000E000200546ABE2304890F83800012801D101E0A3E200200546A1E20FF0EFFC38B12A4890F8380008B9012000E00020054695E21C
:404D4000254890F89000012800D100E0002005468CE20FF0DAFC38B11F4890F8900008B9012000E00020054680E21B4890F83800022804D0184890F89000022801D1012079
:404D800000E00020054671E20AF08BFF80F001056CE21248007D60B90A48001F006900F48030B0F5803F04D002F01EFD08B1012000E00020054659E20948007D08B901204A
:404DC0003FE03DE000170020BC0300203025002058030020590300205427002088290020A02900203DE212E200E2F3E1EAE1DDE1D1E1C5E1BCE1B3E1A7E19EE192E189E1E1
:404E000080E177E16EE165E15CE153E14AE141E138E12FE126E121E115E103E1DAE0CDE0C0E0B3E0A6E099E08CE082E077E06CE054E047E03AE029E01CE00FE006E002E01F
:404E40000020054612E2F74805780FE2F5F762FB08B1012000E00020054607E20EF05CFBB0EE408A9FEDF01ADFEDF00A0EF0D3FA0546FBE10EF050FBB0EE408A9FEDEC1A81
:404E8000DFEDEC0A0EF0C7FA0546EFE102F077FFB0F57B4F07DB02F072FF4FF6FF71884201DA012000E000200546DFE102F028FF28B1E1488078FE2801D0012000E0002089
:404EC0000546D3E1DC488078FE2806D0F8F723F918B101250020D9490872C7E1D6488078FE2805D0D648007810B1F6F706FD20B101251A20FFF796FE06E0FFF796FE1A2878
:404F000002D10020FFF78EFEB0E1CE48007800F0B40008B1012000E000200546A6E1C948007800F0480008B1012000E0002005469CE1C5480088102801D0012000E000206B
:404F4000054693E10EF037FBB0EE408A9FEDB61ADFEDB80A0EF05FFA054687E10EF033FBB0EE408A9FEDB01ADFEDB20A0EF053FA05467BE10EF02FFBB0EE408A9FEDAA1AA2
:404F8000DFEDAC0A0EF047FA05466FE10EF0ECFAB0EE408A9FEDA41ADFEDA60A0EF03BFA054663E10DF055FBB0EE408A9FED9E1ADFEDA00A0EF02FFA054657E10EF0DCFAD4
:404FC000B0EE408A9FED981ADFED9A0A0EF023FA05464BE120F0D2FB18B3F5F7F3FEB0EE408AF5F7C4FE38EE400A10EE106A30462DF01CF941EC190BB0EE490AF0EE690A4B
:4050000029F0EEFCB0EE408AF0EE608A9FED8F0B53EC102B51EC180B2CF010FF00D2012500BF23E1F5F7CEFEDFED8A0AB4EEE00AF1EE10FA04DDF4F7DBFC08B1012000E06D
:405040000020054612E102F0CFFB20B903F017F908B9012000E00020054607E107F0D9FD054603E10FF051FB18B1F6F731FD80F00105FBE0F5F759FA08B1012000E0002090
:405080000546F3E0F5F770FA08B1012000E000200546EBE0F5F712FB08B1012000E000200546E3E0F5F74AFB08B1012000E000200546DBE0F5F77EFB08B1012000E000205B
:4050C0000546D3E0F5F7B2FB08B1012000E000200546CBE0F5F7EAFB08B1012000E000200546C3E0F5F71EFC08B1012000E000200546BBE0F5F752FC08B1012000E00020D6
:405100000546B3E0F5F78AFC08B1012000E000200546ABE0F5F7C4FC08B1012000E000200546A3E00FF0F1FA30B1F5F728FD08B1012000E00020054698E0F5F73EFD08B1C2
:40514000012000E00020054690E00FF0DEFA30B1F5F751FD08B1012000E00020054685E0F5F76BFD08B1012000E0002005467DE0F5F781FD08B1012000E00020054675E01D
:405180000FF0C3FA30B1F5F794FD08B1012000E0002005466AE00FF0B8FA30B1F5F7A7FD08B1012000E0002005465FE00EF09FFA06460EF01FFB06430EB1012000E00020BC
:4051C000054653E00EF04EFB08B1012000E0002005464BE00FF099FA38B107F0B3FF012803D1F6F7E6FB00B901253FE0F5F733F928B9F5F721FE10B9F5F738FE20B1F6F700
:40520000D8FB08B9012000E0002005462EE00EF0CFFB20B91048007820F0F4FEF0B101201DE000009D03002000FF7F4700A0254600007A460000000000C800204431002061
:40524000E8040020B103002052070020000000000070A7400000FA45220700200020054604E003F03BF8054600E000BF00BF05B100BF3DB9FE480078002807DDFC480078E7
:40528000844203D10120BDEC048B70BD0020FAE74FF00008C1464FF0010A4FF0500B0321F44880F8B81000248FE0F348005D04EB840101EBC401F14A02EB81018968087098
:4052C000ED48FF30005D00287DD0E21704EBD2625311EB4A52F82320E31704EBD3635B11A4EB431C012303FA0CF31A43E31704EBD3634FEA631CE24B43F82C20E21704EBCD
:40530000D2625311DE4A0C3252F82320E31704EBD3635B11A4EB431C012303FA0CF31A43E31704EBD3634FEA631CD54B0C3343F82C2004EB840000EBC400D04901EB800088
:40534000007BE0B1E21704EBD2625311CC4A183252F823202146E31704EBD3635B11A4EB431C012303FA0CF31A432046E31704EBD3634FEA631CC24B183343F82C2022F029
:40538000BAFDC04941F8240000BFE21704EBD2625311BB4A243252F823202146E31704EBD3635B11A4EB431C012303FA0CF39A432046E31704EBD3634FEA631CB04B24333D
:4053C00043F82C2000BF601CC4B2422CFFF66DAF4FF47A60DFF8B0C200DFA648D0F8DC100120DFF8A8C200DF4FF47A60DFF898C200DF00BF002259460320DFF894C200DFF2
:405400000646022E21D1DFF88CC200DF074607F00200D0B1002416E0002004EB840101EBC401964A02EB81018968087004EB840101EBC40102EB8101896808782146FFF7BA
:4054400060FB601CC4B2422CE6DB0024AAE22046FFF7EEFB05462046FFF7CDFBA8427DD0002D7CD1A946E31704EBD3634FEA631C834B0C3353F82C304FEAE47C04EBDC6C51
:405480004FEA6C1CA4EB4C1E4FF0010C0CFA0EFC03EA0C034FEAE47C04EBDC6C4FEA6C1CA4EB4C1E4FF0010C0CFA0EFC634501D04FF0010904EB840000EBC4006F4901EB6C
:4054C000800090F8330000F0010008B14FF0010904EB840000EBC400684901EB800090F8330000F0020020B10AF096FA08B14FF0010904EB840000EBC400604901EB8000FE
:4055000090F8330000F0040038B107F08AFB10B920F05FF908B14FF0010904EB840000EBC400564901EB800090F8330000F0080020B1BAF1000F01D04FF0010904EB84002C
:4055400000EBC4004D4901EB800090F8330000F0100038B15048005D012801E010E010E000D18146B9F1010F0AD100204A4908554FF001082046FFF7EBFA3620F7F736FFB8
:4055800003E1E31704EBD3634FEA631C3C4B53F82C304FEAE47C04EBDC6C4FEA6C1CA4EB4C1E4FF0010C0CFA0EFC03EA0C034FEAE47C04EBDC6C4FEA6C1CA4EB4C1E4FF057
:4055C000010C0CFA0EFC6345DAD000203249085500BF02F009F9E8B1E21704EBD2625311274A243252F823202146E31704EBD3635B11A4EB431C012303FA0CF31A43204661
:40560000E31704EBD3634FEA631C1D4B243343F82C201CE0E21704EBD2625311184A243252F823202146E31704EBD3635B11A4EB431C012303FA0CF39A432046E31704EB60
:40564000D3634FEA631C0E4B243343F82C20E21704EBD26253110A4A52F82320E31704EBD3635B11A4EB431C012303FA0CF315E05A0300205041002030250020142404082F
:4056800000170020F41500200108040861080408C108040809080408B21500201A43E31704EBD3634FEA631CFE4B43F82C2022F022FCFD4941F8240004EB840000EBC4002E
:4056C000FA4901EB800080680078401C04EB840101EBC401F54A02EB81018968087004EB840000EBC400114601EB8000806800787E2808DD7E2004EB840101EBC40102EB83
:4057000081018968087000BF00BF02F06DF801281DD1E21704EBD2625311E24A243252F823202146E31704EBD3635B11A4EB431C012303FA0CF31A432046E31704EBD36321
:405740004FEA631CD74B243343F82C201CE0E21704EBD2625311D34A243252F823202146E31704EBD3635B11A4EB431C012303FA0CF39A432046E31704EBD3634FEA631CDB
:40578000C84B243343F82C2000BF002D7DD0E21704EBD2625311C34A0C3252F82320E31704EBD3635B11A4EB431C012303FA0CF31A40002A53D104EB840000EBC400BB4900
:4057C00001EB8000406AE8BBE21704EBD2625311B44A0C3252F82320E31704EBD3635B11A4EB431C012303FA0CF31A43E31704EBD3634FEA631CAB4B0C3343F82C204FF0DF
:40580000010804EB840000EBC40001EB8000806800787E2811DA04EB840000EBC40001EB800080680078401C04EB840101EBC4019E4A02EB81018968087021460120FFF733
:4058400073F900E00CE004EB840101EBC401974A02EB8101896808782146FFF752F95BE004EB840202EBC402904B03EB8202516A8D4A52F8240022F044FBE8B3E21704EBDE
:40588000D2625311874A0C3200E083E052F82320E31704EBD3635B11A4EB431C012303FA0CF31A43E31704EBD3634FEA631C7D4B0C3343F82C204FF0010804EB840000EB70
:4058C000C4007A4901EB8000806800787E2811DA04EB840000EBC40001EB800080680078401C04EB840101EBC401704A02EB810189680870214600E00EE00120FFF714F96A
:4059000004EB840101EBC401684A02EB8101896808782146FFF7F5F804EB840202EBC402624B03EB8202127BA2B3E21704EBD26253115C4A183252F82320E31704EBD36321
:405940005B11A4EB431C012303FA0CF31A400ABB01F04AFF10B901F008FCE0B104EB840000EBC400514901EB8000806A68B104EB840202EBC4020B4603EB8202916A4A4A60
:4059800052F8240022F0BDFA20B12046FFF79CF84FF0010804E02046FFF796F84FF00108601CC4B2422CFFF652ADB8F1010F0BD13F48D0F8DC100120DFF8F8C000DF4FF09F
:4059C00000083620F7F712FD4FF0000AFFF758F804460FE5002107E0324850F8210008B101207047481CC1B20329F5DB0020F8E7002108E02B48183050F8210008B101202A
:405A00007047481CC1B20329F4DB0020F8E770B541201DE0C41700EBD4646511214C183454F82540C51700EBD5656D11A0EB45160125B5402C40C51700EBD5656D11A0EB87
:405A400045160125B540AC4200D103E0411EC8B20028DFDC00BF70BD70B5002401F0C4FEF8B1412437E0E31704EBD3635D110D4B0C3353F82530E51704EBD5656D11A4EB4F
:405A800045160125B5402B40E51704EBD5656D11A4EB45160125B540AB421AD104EB84030AE01BE000170020F415002014240408504100206108040803EBC403294D05EB45
:405AC000830393F83330102B03D1274B1B5D03B903E0601EC4B2002CC5DC00BF204670BD0121214A1154704701460020FF2906DA1D4A525C0AB1012200E00022104670476D
:405B000000B5002304E01846FFF7EAFF581CC3B2422BF8DB00BD0EB5144A07CA8DE807001BF0D1F91CF0A3FF0C226946FF201BF096F90EBD014601EB810000EBC100094A81
:405B400052F820007047014601EB810000EBC100044A02EB8000007970477047044908707047000014240408B21500207C3104085A030020FE48007B7047FD490873704735
:405B800070B52DED068B04460D46284622F0DBF900EE100AB8EE400AB0EE408A9FEDF50AC8EE000AB0EE608A94ED000AD4ED020A00EE880ADFEDF00A68EE200A20EE200A9B
:405BC00010EE101A08462CF031FB41EC1A0BB0EE4A0AF0EE6A0A29F0C3FDB0EE409AF0EE609A51EC190B2BF0E5FC08EE100A94ED040A20EE080AB0EE408AB0EE480ABDEC0B
:405C0000068B70BD10B52DED088BF0EE409AF0EE608A04469FEDD90AF0EE40AA9FEDD50AC0EE290AB0EE608AB1EE000A28EE800AC0EE080AB0EE60AA9FEDD00AB0EE40BAB0
:405C4000204622F080F9BCEEC80A10EE101AB0FBF1F201FB120000EE100AB8EE400AB0EE409AB5EE000A28EE000AB4EEC90AF1EE10FA15D8B6EE080A28EE000AB4EEC90A20
:405C8000F1EE10FA0CDDBFEE000A2AEE000AB0EE40AAB0EE000A28EE800AB0EE40BA0EE0B6EE080A28EE000AB4EEC90AF1EE10FA05D8B9EE000A28EE800AB0EE40BAB0EE4B
:405CC0004B0A0AEE090AF0EE40AAB0EE6A0ABDEC088B10BD2DE9F0412DED028B05460F4690460024002600BF32E0322108FB01F000EE100AB8EEC00ADFED9E0A80EE201A07
:405D000005F1300000EB840090ED000A30EE410A05F1300000EB840080ED000A08FB01F000EE100AB8EEC00ADFED920A80EE201A05F1700000EB840090ED000A30EE410A91
:405D400005F1700000EB840080ED000A601CC4B2082CCADB0024D8E007F1300000EB840090ED000A07F1700000EB8400D0ED000A30EE600AF0EE000A20EE200AB0EE408A64
:405D800005F1300000EB840090ED000A07F1300000EB8400D0ED000A30EE600A05F1900000EB860080ED000A05F1900000EB860090ED000AC0EE080A9FED710A20EE800A96
:405DC00005F1CC0000EB860080ED000A05F1500000EB840090ED000A05F1100000EB8400D0ED000A30EE600A07F1500000EB8400D0ED000A07F1100000EB840090ED001A6D
:405E000070EEC10A80EE201A05F5847000EB860080ED001AB7EE000AC0EE080A05F5A27000EB8600C0ED000A701CC6B20F2E6ADA07F17000611C00EB810090ED000A07F1B3
:405E4000300000EB8400D0ED000A30EE600AF0EE000A20EE200AB0EE408A05F1700000EB810090ED000A07F1700000EB8100D0ED000A30EE600A05F1900000EB860080EDCC
:405E8000000A05F1900000EB860090ED000AC0EE080A9FED3B0A20EE800A05F1CC0000EB860080ED000A05F1500000EB810090ED000A05F1100000EB8400D0ED000A30EEF4
:405EC000600A07F1500000EB8100D0ED000A07F1100000EB840090ED001A70EEC10A80EE201A05F5847000EB860080ED001AB7EE000AC0EE080A05F5A27000EB8600C0ED5F
:405F0000000A701CC6B2601CC4B2082CFFF624AF1C4B0F221C4901F13C0012F06EFC1B4B0F2219493C3901F1780012F066FC154890ED010A0E4880ED1D0A124890ED000AE2
:405F40000B4880ED230A114890ED010ADFED100A30EEC00AD0ED000A80EE201A044880ED261A0F210848783812F02DFC004811E04417002000007A44DB0FC940000000005D
:405F80000000B44360030020F4180020680300200000344380ED200ABDEC028BBDE8F08170B52DED028B0446B0EE408A0D46207800F0100000280AD094ED020A84ED030AE0
:405FC00084ED028AA078082802D10420208086E0207800F00100D8B394ED020AD4ED030AB4EEE00AF1EE10FA20DD94ED020AFE48817804F1500000EB810080ED000AFB4946
:40600000486821F0A0FF00EE100AB8EE400A5FED270A80EE201AF448817804F1700000EB810080ED001A0020E07002E0E078401CE070E0782179884251DD208840F002003C
:406040002080208820F0010020800020E07046E0FFE7207800F00200F0B394ED020AD4ED030AB4EEE00AF1EE10FA1ED294ED020AA17804F1100000EB810080ED000ADB490C
:40608000486821F060FF00EE100AB8EE400A5FED470A80EE201AA17804F1300000EB810080ED001A0020E07002E0E078401CE070E0782179884212DD208840F001002080D8
:4060C000208820F002002080A078401CA0700020E0700DB1207900E001E0401E2071BDEC028B70BD10B52DED028BF0EE408AB0EE608ABE49486821F026FFB0F57A7F0BD9DD
:406100000121B0EE480ABA48FFF74AFF0021B0EE680AB548FFF744FFB548008804280DD1B1480088042809D10222AF49B048FFF7D1FD2020AE490880AB490880BDEC028B46
:4061400010BD70B52DED0C8B0446F5F70DFD60B1F7F7B2F8B0EE408AD4ED098AF1EE009AB1EE00AAB0EE009A57E0F5F736FD40B30FF030F805460FF031F8281A00EE100AB0
:40618000B8EEC00ADFED9B0A20EE200AB0EE40BA0FF096F8DFED980A20EE208A94ED090ADFED950A60EE208AB1EE000A6BEE009AB1EE000A2BEE00AAB0EE000A2BEE009A21
:4061C0002BE00AF063FEB0EE408A8C4991F8280091ED0F0AF0EE400AB0EE480A0AF06DFDDFED870A20EE200AB0EE408A834991F8280091ED0F1AF0EE410A94ED091AB0EEAC
:40620000410A0AF05AFDDFED7E0A60EE208AF0EE009AB0EE00AAB7EE009A4020005D40B994ED0B0A38EEC00A84ED0E0A01214020015519EE900A2BF0F9FF41EC1B0B94ED52
:406240000B0A30EE480A10EE101A08462BF0EEFF41EC1D0BB0EE4D0AF0EE6D0A28F0C0FBB0EE40CAF0EE60CA53EC1B2B51EC1C0B2BF0E4FD0ED24C20005D58B9606821F081
:4062800062FE00EE100AB8EE400A84ED110A01214C2001551AEE100A2BF0C8FF41EC1B0B38EEC80A10EE101A08462BF0BFFF41EC1C0BB0EE4C0AF0EE6C0A28F091FBB0EE9A
:4062C00040DAF0EE60DA53EC1B2B51EC1D0B2BF07BFC0ED25820005D58B9606821F033FE00EE100AB8EE400A84ED140A01215820015519EE100A2BF099FF41EC1B0B38EE5C
:40630000C80A10EE101A08462BF090FF41EC1C0BB0EE4C0AF0EE6C0A28F062FBB0EE40DAF0EE60DA53EC1B2B51EC1D0B2BF086FD0DD8002164200155607B324951F8200063
:4063400000EE100AB8EE400A84ED170A31E019EE100A2BF06BFF41EC1B0B38EEC80A10EE101A08462BF062FF41EC1C0BB0EE4C0AF0EE6C0A28F034FBB0EE40DAF0EE60DAEC
:4063800053EC1B2B51EC1D0B2BF01EFC11D26420005D70B9012164200155606821F0D3FD00EE100AB8EE400A84ED170A21F0A3FDA06078EEC8AA94ED0E0AB5EEC00AF1EE34
:4063C00010FA0BD2B4EEE88AF1EE10FA06D294ED1B0AB4EEEA0AF1EE10FA24D394ED0E0AB5EEC00A10E000006C19002044170020EC17002017B7D1380AD7233C301F002006
:40640000E02E654288310408F1EE10FA25DDB4EEE88AF1EE10FA20DD94ED1B0AB4EEEA0AF1EE10FA19DDC4ED1BAA94ED1B0A10EE101A08462BF0FAFE41EC1C0BB0EE4C0AF5
:40644000F0EE6C0A28F0CCFAB0EE40BAF0EE60BA51EC1B0B2BF0AEF8A066BDEC0C8B70BD00200022002100BF33E0FE4B03EB820393ED000AB5EEC00AF1EE10FA01D14B1CB9
:4064800099B2F84B403303EB820393ED000AB5EEC00AF1EE10FA01D14B1C99B2F24B03EB820393ED000AB5EEC00AF1EE10FA01D14B1C99B2EC4B403303EB820393ED000A49
:4064C000B5EEC00AF1EE10FA01D14B1C99B2531CDAB2082AC9DB00224FE0E44B93ED1D0ADFEDE30AB4EEE00AF1EE10FA06DC93ED1D0AB5EEC00AF1EE10FA01D24B1C99B238
:40650000DA4B93ED230ADFEDDA0AB4EEE00AF1EE10FA08DC93ED230ADFEDD60AB4EEE00AF1EE10FA01D24B1C99B2D04B93ED260ADFEDCF0AB4EEE00AF1EE10FA06DC93EDE6
:40654000260AB5EEC00AF1EE10FA01D24B1C99B2C64B93ED200ADFEDC60AB4EEE00AF1EE10FA06DC93ED200AB5EEC00AF1EE10FA01D24B1C99B2531CDAB20F2AADDB01B967
:4065800001207047B94890F8A4007047B74981F8A4007047B548407B0C2823D0B348407B0B281FD0B148407B07281BD0AF48407B112817D0AD48407B082813D0AB48407B83
:4065C0000A280FD0A948407B04280BD0A748407B052807D0A548407B0F2803D0A348407B102801D1012070470020FCE79F48407B08281BD09D48407B042817D09B48407BDE
:40660000052813D09948407B0A280FD09748407B0B280BD09548407B0F2807D09348407B102803D09148407B112801D1012070470020FCE78D48407B082817D08B48407BFF
:40664000042813D08948407B05280FD08748407B0A280BD08548407B0B2807D08348407B102803D08148407B0F2801D1012070470020FCE77D48407B082803D07B48407B50
:406680000A2801D1012070470020FCE770B5002426F0FCFC002872D101F032FB18B10720FFF774FF80E009F0FCFA30B9FFF7E2FF18B90220FFF76AFF76E018F0A6FCB5EEBE
:4066C000C00AF1EE10FA06D2FFF7B4FF18B90920FFF75CFF68E018F098FCDFED670AB4EEE00AF1EE10FA02D2FFF780FF60B15F48407B0F280CD118F08CFCDFED5F0AB4EE4E
:40670000E00AF1EE10FA03D20420FFF73FFF4BE018F07BFCDFED590AB4EEE00AF1EE10FA06DDFFF763FF18B90520FFF72FFF3BE05348007D18B90120FFF728FF34E0F3F776
:406740008AFE50B1F5F735F938B94848407B0F2803D10D20FFF71AFF26E006F042FB28B106F03FFB0546FFF711FF1DE0F6F791FD30B1F6F78EFD0546FFF708FF14E01AE059
:4067800006F047FA38B13948407B0B2803D02420FFF7FCFE08E0FFF72BF928B1FFF7FAFE10B90A20FFF7F2FEFFF7ECFE18B10120FFF7E3F90124204670BDC9B1DFED310ACC
:4067C000C0ED000ADFED300AC0ED010A2F4AD2ED060AB8EE601ADFED2E1AC1EE210A9FED2D1AC1EE201AC0ED021A80ED040A1CE0DFED290AC0ED000ADFED280AC0ED010A66
:40680000224AD2ED0D0AB8EE601ADFED211AC1EE210ADFED231A81EEA01AF6EE000A61EE200AC0ED020A80ED040A704710B501219FED1C0A0D481030FFF7BFFF4FF4C0713B
:406840000848303826F06FFF4FF4C0710648303826F069FF0A2003493039087102493039087121E01C1800209C1900204417002000409C4500409CC52FDDE43E2FDDE43FEB
:40688000A0290020CDCCCC3D14AE473F8831040800007A447A142E3FCDCC4C3E0000204233331F4235FA0E3D1120FA490880FA49088010BD2DED028B84B04FF47A66A82166
:4068C000F64826F030FF1421F54826F02CFF00BF002231460320DFF8CCC300DF0546022D70D1DFF8C4C300DF0446022C6BD1EC480078002867D0EA480078122863DC0120A7
:40690000EA490870E6480078E449487321F0F3FAE2494860E24890ED010A084680ED090A407BE34908700020DC498860084600218166C1660167C165016641668163C16320
:40694000016441648164C1640165416581650020D24981F8A4000846407BD64951F82000CE4908600846407B122873D2DFE800F0A14C4F5051520943494A489C412C3A4D84
:406980004E44C648002141678167C1678030C160016141618161C1610162016041608160FFF744FF04208DF8040003208DF8050005208DF80600022201A9FF201AF04FFABC
:4069C000042677E0ACE079E000219FEDBB0AB3481030FFF7F2FE9FEDB90AB04880ED090A042667E09FEDB60AAC4880ED090A042660E0C8265EE000BFFCF74DFFC82659E0EB
:406A000000BF00BF042655E000BF00BF00BF00BF00BF00BFF5F7A8F850B1F6F74DFCB0EE408A9E4880ED0B8A012180F834102BE0F5F7D3F878B10EF043FCDFEDA20A20EE60
:406A4000200AB0EE408A954880ED0B8A012180F8341019E02DE00AF019FAB0EE408A9A4991F8280091ED0F0AF0EE400AB0EE480A0AF023F9DFED950A20EE200A874880ED14
:406A80000B0A012180F8341004208DF8040003208DF8050005208DF80600032201A9FF201AF0DDF9042605E04FF4C87606F0B5FA00E000BF00BF042078490873012C2FD1EB
:406AC000002076494873002101209FED7C0AF3F75EFC0020754908709FED780A704880ED010A9FED760A6D4880ED090A012180F864104FF47A665720F6F778FC5820F6F721
:406B000075FCFFF737F8042802D10020FFF735F80C2018F0AFFF002201A9FF201AF09FF95E48407B00287DD05C4A1168506821F0E8F918BBFFF71EF804280FD05748407B2B
:406B400007281BD05548407B112817D05348407B0B2813D05148407B0C280FD0FFF796FD60B94E4890F8640001286DD14B49886840F6C41121F0C5F9002865D04748407B20
:406B8000022807D04548407B012803D04348407B032819D1414890F8640030B93F4890ED000AB8EE400A80ED170A3C4890F8580030B93A4890ED000AB8EE400A80ED140A7A
:406BC0005820F6F713FC1FE03448407B06281BD1FFF746FC80B99FED3E0A304880ED1D0A9FED3B0A80ED230A9FED390A80ED260A9FED370A80ED200A0020264908802649BF
:406C000008805720F6F7F2FB0C2018F033FF002022494873FEF7AEFF042802D10020FEF7ACFF00E010E0002101209FED240AF3F7AEFB00201D4908709FED200A184880ED8E
:406C4000010A4FF47A6643E61448407B122879D2DFE800F0095279F5F3F2F1F0EFEEEDECEBEAE90A0BE81CE200BFF4F7B6FF88B30EF0B0FB00EE100AB8EE400A074880ED75
:406C8000090AD0ED090AB0EE600A0121032007F0C0FD2DE0EC1700206C1900204417002030170020C1080408090804085C03002078030020883104080000A0420000000086
:406CC000000070420AD7233C301F0020E02E6542003C1C46FFE71FED070AFC4880ED090AD0ED090AB0EE600A0121032007F001FCF648FFF726FAD4E1F4F76FFF88B10EF06F
:406D000065FA00EE100AB8EE400AF04880ED090AD0ED090AB0EE600A0121032007F079FD0CE01FED1A0AE94880ED090AD0ED090AB0EE600A0121032007F0DBFBE348FFF7E2
:406D400000FAAEE193E1F4F70FFF68B19FEDE00ADE4880ED090AD0ED090AB0EE600A0121032007F09AFC59E0F4F737FF00B30EF02DFA00EE100AF8EE408A0EF027FA80466F
:406D80000EF02CFAA8EB000000EE100AB8EEC00ADFEDD00A40EEC08ACC48C0ED098AD0ED090AB0EE600A0121032007F032FD35E01EF00FFDD8B1C84890ED640ADFEDC70A9F
:406DC00020EE200A5FED410A20EE200AB0EE408A014691F8280091ED0F0AF0EE400AB0EE480A09F0F9F9B94880ED090A0DE0BA4991F8280091ED0F0AF0EE400A9FEDB80A63
:406E000009F0EAF9B14880ED090AB048D0ED090AB0EE600A0121032007F06BFBAB48FFF790F93EE1F9E0D0E0E5E00BE104E1F7E001E1F6E0F0E08FE07FE06FE0FFE7F4F78E
:406E400093FE68B19FEDA50AA04880ED090AD0ED090AB0EE600A0121032007F01EFC59E0F4F7BBFE00B30EF0B1F900EE100AF8EE408A0EF0AFF980460EF0A8F9A8EB000009
:406E800000EE100AB8EEC00ADFED920A40EE808A8E48C0ED098AD0ED090AB0EE600A0121032007F0B6FC35E01EF093FCD8B18A4890ED650ADFED890A20EE200A5FED7F0A79
:406EC00020EE200AB0EE408A014691F8280091ED0F0AF0EE400AB0EE480A09F07DF97B4880ED090A0DE07C4991F8280091ED0F0AF0EE400A9FED7B0A09F06EF9734880EDDE
:406F0000090A7248D0ED090AB0EE600A0121032007F0EFFA6D48FFF714F9C2E06E4890F84210D03000EB8100D0ED000AB0EE600A01210846F3F72BFAB3E0674890F84210C7
:406F4000D83000EB8100D0ED000AB0EE600A01210846F3F71CFAA4E05C4841681030FEF70FFE5A4880ED090A5B4991F8280091ED0F1AF0EE410A554991ED091AB0EE410ADC
:406F800009F02AF9F0EE408A0121032007F0B1FA4E4890F82900B8B100204C4981F8290009F0F3FFF0EE408A03214F480FF05EF84D4890ED001AF0EE410A444890ED091AFB
:406FC000B0EE410AFFF78EF86BE0404948684749D1ED000A464991ED000AFEF713FE3B4880ED090AD0ED090AB0EE600A01210846F3F7CDF955E0354841681030FEF7C0FDEB
:40700000324880ED090AD0ED090AB0EE600A01210846F3F7BCF944E000BFFCF791FB40E000BF2A48D0ED090AB0EE600A01210846F3F7ADF935E034E005F0EEFE8046FEF71F
:407040009CFD2EE0214A083202F11C0101F18000F9F7D6FB8046FEF790FD1C48D0ED090AB0EE600A01210846F3F791F919E00020164948730873002101201FEDF00AF3F739
:4070800086F900201B4908701FEDF40A1A4880ED010A002201A9FF2019F0E1FE4FF47A6600BF00BFFEF766FD04287FF4CCAD4FF4FA71384620F025FF00283FF4C4AD20F051
:4070C0001AFF07460C2018F0D5FC01E44417002000008CC23333333F301F002000008C42C2B8B2BEC2B8B23E70030020800300207C0300205C0300203017002070B52DED14
:40710000028B0446B0EE408A0025B5EEC08AF1EE10FA0AD04CB1122C07DCAF4890ED010AB4EE480AF1EE10FA0DD1AC48D0F890110120DFF8ACC200DF9FEDAA0AA64880EDA6
:40714000010A00250DE00CB1A3480470A24880ED018AA248D0F890110220DFF884C200DF01252846BDEC028B70BD9F480078704701209E4981F8290070477A2303709B4B1F
:40718000D3ED0E0A9FED9A0AB2EE041A00EE810ABDEEC00A10EE103A1AB24270130A8370924B93ED110ABCEEC00A10EE103A99B2C1700B0A03718D4B93ED140ABCEEC00A22
:4071C00010EE103A99B241710B0A8371874B93ED170ABCEEC00A10EE103A99B2C1710B0A0372824BD3ED1A0A9FED810AB2EE041A00EE810ABDEEC00A10EE103A1AB24272CF
:40720000130A837270477B230370784BD3ED1D0A9FED781A9FED760A00EE810ABDEEC00A10EE103A19B241700B0A83706F4BD3ED230A9FED701A9FED6E0A00EE810ABDEE01
:40724000C00A10EE103A19B2C1700B0A0371674BD3ED260A9FED671A9FED650A00EE810ABDEEC00A10EE103A19B241710B0A83715E4B93ED200ADFED600A20EE200ABCEEA6
:40728000C00A10EE103A9AB2C271130A0372704710B500245548407B122813D2DFE800F013141718191A1B091E1F1D0E121C1215160A00BFFCF73FFB044611E005F0A7FE92
:4072C00004460DE000BF00BF00BF00BF00BF00BF00BF00BF00BF00BF00BF00BF00BF00BF00BF204610BD10B500244048407B122813D2DFE800F013141718191A1B091E1F07
:407300001D0E121C1215160A00BFFCF718FB044611E005F07CFE04460DE000BF00BF00BF00BF00BF00BF00BF00BF00BF00BF00BF00BF00BF00BF00BF204610BD2B48407B75
:4073400070472A4890F86400704710B500242748407B122816D2DFE800F01718191A1B1C1D0920211F16151E150E0F0A00BFF7F7FAFC044613E000BFFFF7E3FF642110FBAA
:4073800001F40CE000BF00BF00BF00BF00BF00BF00BF00BF00BF00BF00BF00BF00BF00BF204610BD002011490873704713480078704710B500F0A5FF044644F6206120F0A3
:4073C000A0FD38B900F09DFF40F2DC51884201D9012010BD0020FCE7301700205041002061080408000000005C03002044170020000000470000C84200007A44780300204E
:4074000070B50023012113E0CC1701EBD4646511F84C54F82540CD1701EBD5656D11A1EB45160125B5402C4004B10B46481CC1B24029E9DB184670BD70B504460D46E21737
:4074400004EBD2625311EB4A52F823202146E31704EBD3635B11A4EB43160123B3401A432046E31704EBD3635E11E24B43F826202846FDF7D7FB002C37D00821DE48DFF846
:407480007CC300DF012813D0DB482038817F807F401CD94A203A907710464454807F1E2802DB002011468877D348DFF854C300DF0821D448DFF844C300DF012815D020F0BA
:4074C0001AFDD14901EBC4014860CF4810F83400FF2806DACC4810F83400401CCA4901F83400C848DFF818C300DF70BDC7490870704710B5C648007905287DD2DFE800F030
:4075000003152581DE00FEF773FA10B90220C0490871C048007838B10120BF490870FFF7E5FF0020BB49087006E1FEF761FA10B90220B7490871B748007828B10120B64955
:4075400008700020B3490870F6E0FEF751FA18B10020AF49087153E0AE48007898B30120AD490870FEF744FA50B1FEF750FA044621460920FFF760FF0120FFF7B7FF3FE086
:4075800005F047FB38B127210320FFF755FF0120FFF7ACFF34E0A148007800F0080038B918213120FFF748FF0120FFF79FFF27E003209749087120F09EFC994908600020C3
:4075C000FDF730FB1CE0FFE7FFF7BBFEC0B907F05BFEA8B1FFF7C9FD90B9FFF7EAFE78B117F017FDDFED8F0AB4EEE00AF1EE10FA06DD9FED8D0A00E09DE00F20FFF77EFDB5
:407600009AE08448007800284DD005F002FB50B127210320FFF710FF0120FFF767FF01207D49087049E0FEF7E3F968B10120FFF75DFF012078490870FEF7E9F904462146A0
:407640000920FFF7F9FE38E04FF47A717448006820F057FC90B17148007800F0020008BB0120FFF743FF18213120FFF7E5FE0120694908700020664908711EE0674800788C
:4076800000F00B0070B1FFF770FD30B16748D0F890110120DFF898C100DF04205C49087108F0DEF909E018210220FFF7C5FE0120594908700220564908713DE0554800786D
:4076C00050B918210220FFF7B7FE01205249087002204F49087123E005F09BFA68B127210320FFF7A9FE0220494908710120FFF7FDFE01204849087012E0FEF779F978B17B
:407700000020434908710120FFF7F0FEFEF77FF9044621460920FFF78FFE01203E4908703B480079042805D020F0E5FB3849086008F095F900E000BF00BF35480079344908
:40774000487110BD2B48001F0021016041608160C160704737490870704710B5364991F83000F4F7F0F830B1002213466421334812F06DFC11E0304991F83000F4F705F9C3
:4077800028B92D4991F83000F4F707F928B1002213463121294812F05AFC10BD10B50024254991F83000F4F7CEF858B9224991F83000F4F7EAF828B91F4991F83000F4F7E2
:4077C000ECF800B10124204610BD1A480078704710B504461A480078844204D018480470112018F047F910BD09490979042929D1012128E08C1D0020781D0020290D040889
:40780000450C0408141B0020581B0020920300208803002093030020940300209C030020980300202FDDE43E0000C842504100206108040890030020301F002040CD002015
:407840008603002000210846704700EE900AB8EE601ADFEDF80AF5EE001A51EE210AB0EE600ADFEDF50A80EE201AB0EE410A7047F2480078704710B52DED028BFFF7F8FF7F
:40788000022807D0FFF7F4FF032803D0FFF7F0FF052812D10CF024FF30B10CF01BFF022802D19FEDE78A0AE00CF01AFF10B19FEDE58A04E01FED258A01E01FED268AB0EE46
:4078C000480ABDEC028B10BD10B52DED028B17F080FBB0EE408AFFF7CEFFB4EEC08AF1EE10FA03DB0120BDEC028B10BD0020FAE710B52DED048BF0EE408AB0EE609A04464A
:40790000F0EE689AFFF7E0FF00EE100AB8EE400AB4EEC90AF1EE10FA07DDFFF7D5FF00EE100AB8EE400AB0EE409A29EE090ADFEDC60A80EE808AECB1F4EEC88AF1EE10FA26
:4079400005DDF0EE489A0120C049087015E0B1EE480AF4EEC08AF1EE10FA07D2B1EE480AF0EE409A0120B949087006E00020B749087002E00020B5490870B0EE690ABDECFB
:40798000048B10BD10B504460020206060606071207120F0B0FA206010BD2DED048B92B04FF05008002405E04FF6FF702DF81400601CC4B2022CF7DB0020FFF7CBFE00202A
:4079C0008DF80400A2490870FFF790FD0020A1490870A148DFF884C200DFA148DFF87CC200DFA048DFF874C200DF00209A49183908759D48FFF7C6FF03219C4880F84411BA
:407A000000BF002241460720DFF864C200DF0746022F7AD1DFF85CC200DF054605F00200002873D010218C48DFF84CC200DF012809D028228849183908A825F020FE8648A9
:407A4000DFF838C200DFBDF82060FFF7CDFE08B1012000E00020814617F0BBFAF0EE408A3046FFF7F2FEB0EE409A4846F0EE680AFFF73EFFB0EE408AFFF7B6FE00B37648F3
:407A80001838007D01280BD1DDED0A0AB0EE600A0121042006F0A4FD8146FFF799FE2FE06D481838007D02280BD1DDED090AB0EE600A0121052006F0F0FD8146FFF788FEF4
:407AC0001EE065481838007D03280BD1DDED0B0AB0EE600A0121062006F09BFE8146FFF777FE0DE05C481838007D042808D101210220B0EE480A06F0FCFC8146FFF768FE6F
:407B00009DF83500012802D102E047E032E000205B4908709DF8350040B95A48007840F00800584908700020FFF7E0FC4FF6FF7086421FD05348007800F00200D0B9514876
:407B4000007800F00800A8B1002410E03DF81410711A08B20EF0EFFC022806DC4948007840F002004749087003E0601CC4B2022CECDB00BF05F0040080B1434801889DF8F6
:407B80000420501CC0B28DF804002DF812109DF80400022802DB00208DF804001AF07FFF68B10BF025FF50B1FFF70FFE38B9FFF7F5FD08B1FFF7D1FD0120FFF7CBFD9DF81C
:407BC000360090B10C9820F0BEF9B0F5C87F0CD301201F4908702548D0F8B4100120DFF8ACC000DF0CF09DFD02E00020184908702748007D01284DD19DF81C0028B9002045
:407C00002049087020F077F9824640F2E241504620F077F968B11DF0DCFD50B901200D4908701248D0F8B4100120DFF860C000DF4FE04EE00000FB4500007A4484030020DA
:407C40000AD7A33C9A99193ED222FB3F95030020910300209D0300203C1B0020350C0408781D0020141B00208803002050410020C108040809080408290D0408450C0408AB
:407C8000930300209C0300204C1B002061080408702900209DF81C0001281AD1F848007DB8B90020F7490870FFF74CFDF648D0F8B4100120DFF8D4C300DFF548007840F073
:407CC0000100F34908700120F249087020F013F982461822EA4902A825F0D1FCFFF709FCEC48007801287FF48CAEFFF789FBEA4908700020E7490870122017F0BBFE80E65C
:407D0000E64800787047E64800787047E5480078704770B50025E448007D012801D1002405E0E148007D08B9012400E002242543DE48C472FDF75CFE08B9012400E00024A8
:407D400045EA8400C5B2D9484472D948007D08B9012406E0D648007D012801D1002400E0022445EA0410C5B2D0488472FFF7CEFF044645EA8415CD480472284670BDCD4800
:407D8000008870472DE9F04105460C4617469846069EB5F52D4F28D12821C6481830DFF818C300DF012820D0A078C249C875A07800F0030048752078617840EA0120BD496F
:407DC000088020F098F8BB4908610120887504200875AD48D0F840110220DFF8B0C200DFB4481830DFF8D4C200DFBDE8F081F0EE400A9FEDB30A30EEC01ADFEDB21A81EEC1
:407E0000210A70472DE9F0412DED028B04460D4616461F462078AD2833D12821A5481830DFF894C200DF01282AD0E078A149C875E07800F0030048756078A17840EA012033
:407E400000EE100AB8EEC00AB0EE408AB0EE480AFFF7CDFF974880ED020A20F04CF8954908610120887508758748D0F840110220DFF818C200DF8F481830DFF840C200DF71
:407E80006BE02078AE2834D128218A481830DFF828C200DF012860D0E0788649C875E07800F0030048756078A17840EA012000EE100AB8EEC00AB0EE408AB0EE480AFFF73A
:407EC00096FF7C4880ED010A20F015F87949086101208875022008756B48D0F840110220DFF8A8C100DF73481830DFF8D0C100DF33E02078AF2830D128216E481830DFF8B4
:407F0000B8C100DF012828D0E0786A49C875E07800F0030048756078A17840EA012000EE100AB8EEC00AB0EE408A624880ED038A1FF0E1FF5F4908610120887503200875FA
:407F40005148D0F840110220DFF840C100DF59481830DFF868C100DF00BFBDEC028BBDE8F0811FEDCB1A5FEDCD0A40EE010AF1EE001AB6EE001A00EEA11AFCEEC10A10EE43
:407F8000901A88B2704710B52DED028B08F07EFFB0EE408A9FED4C0AB4EE408AF1EE10FA06D0B0EE480AFFF7DCFF4049088003E04FF6FF703D4908803348D0F840110420A1
:407FC000DFF8C8C000DF39480088BDEC028B10BD70B58CB006460025002E50D01DF0F9FB002876D040F2B240012102220023CDE90532CDE90710042017210193CDE9023188
:408000000490972013460022114600900AA811F01FFE0AA9304611F011FB044640F292400440844204D11DB9042028490870012540F2B240012102220023CDE90532CDE927
:408040000710042017210193CDE902310490972001230022114600900AA811F0F9FD0AA9304611F0EBFA044640F292400440844205D1002DFCD10520144908700125E0E0D8
:40808000702900209D03002050410020610804089C0300209403002085030020910300208603002092030020A02900204C1B002010280020241B0020290D0408450C04082B
:4080C00000401C460000C84200FF7F4784030020FFE740F2B240012102220023CDE90532CDE9071017210193CDE902319720049300900123002211460AA811F0A9FD0AA9FF
:40810000304611F09BFA044640F292400440844204D11DB903207C490870012540F2B240012102220023CDE90532CDE9071017210193CDE902319720049300901346002255
:4081400011460AA811F084FD0AA9304611F076FA044640F292400440844204D11DB9022069490870012540F2B240012102220023CDE90532CDE9071017210193CDE9023169
:408180009720049300900323002211460AA811F05FFD0AA9304611F051FA044640F292400440844204D11DB9032057490870012540F2B240012102220023CDE90532CDE92A
:4081C000071017210193CDE902319720049300900423002211460AA811F03AFD0AA9304611F02CFA044640F292400440844204D11DB9022044490870012540F2B240012165
:4082000002220023CDE90532CDE9071017210193CDE9023197201A461946049300900AA811F016FD0AA9304611F008FA044640F292400440844204D11DB9012032490870E2
:40824000012515B15520F5F7D1F828460CB070BD10B52E4890F8280007280DD116F0B9FEDFED2B0AB4EEE00AF1EE10FA01DB012000E00020044600E00124204610BD10B522
:4082800016F0A7FEDFED230AB4EEE00AF1EE10FA01D8012010BD0020FCE79FED1F0A70479FED1E0A70471848007803280FD01648007802280BD014480078012807D0124819
:4082C0000078042803D010480078052801D1012070470020FCE712480079704710B5F3F72DFC10B10F48047800E00024204610BDF0EE400A1FED8D1A1FED8F0A00EE810A37
:40830000704707480068704784030020301F00202FDDE43E83C00041B81E4141A245484188030020950300201FB51DF066FA062808D01DF062FA072804D01DF05EFA0828DD
:4083400041F077821DF045FA00287DD0002000900190029003460122FE4903901DF027FB002000900190029003460322FA49039001201DF01CFB0020009001900290034652
:408380000322F649039002201DF011FB002000900190029003460322F149039010461DF006FB002000900190029003460322ED49039004201DF0FBFA002000900190029016
:4083C00003460422E849039005201DF0F0FA002002220123CDE901200093039003460322E24906201DF0E3FA002000900190029003460246DE49039007201DF0D8FA0020DC
:4084000000900190029003460322DA49039008201DF0CDFA002000900190029003460122D549039009201DF0C2FA002000900190029003460122D14903900A201DF0B7FAB3
:4084400000200090019000E0E0E3029003460122CB4903900B201DF0AAFA002001210090CDE9010103460A46C64903900C201DF09EFA002000900190029003460246C24992
:40848000039011201DF093FA002000900190029003460322BD49039012201DF088FA00200222CDE9000202900346B949039016201DF07DFA002001210090CDE901010346CA
:4084C0000A46B449039017201DF071FA002000900190029003460222AF49039019201DF066FA00200222CDE9000202900346AB4903901A201DF05BFA0020009001900290AF
:4085000001230222A64903901B201DF050FA002000900190029001230222A24903901C201DF045FA00200222CDE90002029003469D4903901E201DF03AFA00200222CDE9F5
:408540000002029003460246984903901F201DF02EFA0020009001900290034603229449039021201DF023FA0020009001900290034603228F49039022201DF018FA0020A5
:40858000009001900290034603228B49039023201DF00DFA0020009001900290034603228649039024201DF002FA0020009001900290034603228249039025201DF0F7F90B
:4085C0000020009001900290034603227D49039026201DF0ECF90020009001900290034601227949039027201DF0E1F90020009001900290034601227449039028201DF003
:40860000D6F90020009001900290034601227049039029201DF0CBF90020009001900290034602226B4903902B201DF0C0F9002000900190029003460222674903902C205F
:408640001DF0B5F9002000900190029003460122624903902D201DF0AAF90020009001900290034601225E4903902E201DF09FF900200090019002900346012259490390E5
:408680002F201DF094F90020009001900290034601225549039031201DF089F90020009001900290034601225049039032201DF07EF900200121CDE9000103460A46CDE9F8
:4086C00002104B4936201DF072F9002000900190029003460122474903903B201DF067F9002000900190029003460122424903903C201DF05CF900200122CDE90002029034
:4087000003463E4903903D201DF051F900200122CDE9000202900346394903903E201DF046F9002001210090CDE9010103460A463449039041201DF03AF900200090019078
:408740000290034601223049039042201DF02FF900205BE0CB060020E8060020E70600202B0700202C070020EB060020EC06002037070020E9060020FF060020FE06002073
:40878000FD0600201F070020B4060020F1060020A7060020BE060020A8060020AD0600202D0700202E070020AC060020B1060020A1060020A3060020F4060020F5060020F6
:4087C000F6060020F7060020F9060020F8060020FA060020FB060020FC060020ED060020EF060020EE06002000070020010700200207002004070020050700200607002068
:408800000707002008070020D206002000900190029003460122FE49039043201DF0C7F8002000900190029003460122F949039044201DF0BCF8002001210090CDE90101F8
:4088400003460A46F449039048201DF0B0F8002001210090CDE9010103460A46EF4903904B201DF0A4F8002001210090CDE9010103460A46EA4903904D201DF098F800205D
:4088800000900190029003460322E64903904F201DF08DF8012000220092CDE9012013460246E149039050201DF081F8002001210090CDE9010103460A46DC490390512088
:4088C0001DF075F8002000900190029003460122D749039052201DF06AF8002000900190029003460322D349039054201DF05FF8002000900190029003460322CE49039078
:4089000055201DF054F8002000900190029003460322CA49039056201DF049F8002000900190029003460322C549039057201DF03EF800200222CDE9000202900346024603
:40894000C049039057201DF032F8002000900190029003460322BC49039058201DF027F8002000900190029003460322B749039059201DF01CF800200090019002900346A6
:408980000322B34903905A201DF011F8002000900190029003460322AE4903905B201DF006F8002001210090CDE9010103460A46A94903905C201CF0FAFF002000900190B8
:4089C000029003460122A54903905D201CF0EFFF002000900190029003460122A04903905E201CF0E4FF0020009001900290034601229C4903905F201CF0D9FF00200222FB
:408A0000CDE900020290034601229749039061201CF0CDFF00200222CDE900020290034601229249039062201CF0C1FF0020009001900290034601228D49039064201CF0C6
:408A4000B6FF0020009001900290034601228949039065201CF0ABFF002001210090CDE9010103460A468449039067201CF09FFF002001210090CDE9010103460A467F49C3
:408A8000039069201CF093FF00200222CDE900020290034602467A4903906A201CF087FF01200021009101910B460246CDE9021074496B201CF07BFF00200222CDE90002DB
:408AC00002900346704903906D201CF070FF00200222CDE90002029003466C4903906E201CF065FF00200222CDE9000202900346674903906F201CF05AFF0020012100904A
:408B0000CDE9010103460A466249039073201CF04EFF00200222CDE900020290034602465D49039079201CF042FF002000900190029003460222594903907A201CF037FF2B
:408B4000002000900190029003460122544903907B201CF02CFF002000900190029003460122504903907C201CF021FF0020009001900290034601224B4903907D201CF072
:408B800016FF002001210090CDE9010103460A46464903907E201CF00AFF002000900190029003460122424903907F201CF0FFFE002001210090CDE90101034602223D4926
:408BC000039082201CF0F3FE002001210090CDE90101034602223849039083201CF0E7FE002001210090CDE90101034602223349039084201CF0DBFE0120002100910191B0
:408C00000B460222CDE902102D495BE0DAE00000090700200A0700202F070020300700201E070020EA0600200B0700200C0700200D0700203407002035070020360700207C
:408C400038070020B9060020120700201307002014070020AF06002015070020170700201807002016070020F3060020F2060020190700201A0700201B0700201D07002005
:408C8000DF060020CC060020310700203207002033070020200700202207002023070020C5060020C6060020240700202507002021070020CF060020D0060020D106002040
:408CC0002707002086201CF072FE01200021009101910B460222CDE90210FE4987201CF066FE01200021009101910B460246CDE90210F94988201CF05AFE002000900190AF
:408D0000029003460322F54903908E201CF04FFE002000900190029003460322F04903908F201CF044FE002000900190029003460322EC4903908F201CF039FE01200AF03B
:408D400078FB0021E84800781CF05AFD0021E74800781CF055FD0021E54800781CF050FD0021E44800781CF04BFD01200021009101910B460222CDE90210DF4986201CF07A
:408D800016FE01200021009101910B460222CDE90210DA4987201CF00AFE0121D84800781DF0B3F90121D74800781DF0AEF90121D54800781DF0A9F90121D44800781DF016
:408DC000A4F9E1E3002000900190029003460122CF4903901CF0EBFD002000900190029003460322C649039001201CF0E0FD002000900190029003460322C2490390022046
:408E00001CF0D5FD002000900190029003460322C049039010461CF0CAFD002000900190029003460322BC49039004201CF0BFFD002000900190029003460422B7490390B4
:408E400005201CF0B4FD002002220123CDE901200093039003460322B14906201CF0A7FD002000900190029003460322A749039007201CF09CFD00200090019002900346C1
:408E80000322A149039008201CF091FD002000900190029003460122A249039009201CF086FD0020009001900290034601229E4903900A201CF07BFD00200090019002909F
:408EC00003460122994903900B201CF070FD002001210090CDE9010103460A46944903900C201CF064FD0020009001900290034603229049039011201CF059FD00200090D1
:408F000001900290034603228B49039012201CF04EFD00200222CDE90002029003468749039016201CF043FD002001210090CDE9010103460A466E49039017201CF037FD10
:408F40000020009001900290034602227C49039019201CF02CFD00200222CDE9000202900346784903901A201CF021FD002000900190029001230222734903901B201CF0AB
:408F800016FD0020009001900290012302226F4903901C201CF00BFD00200222CDE90002029003466A4903901E201CF000FD00200222CDE900020290034602466549039024
:408FC0001F201CF0F4FC00200222CDE900020290034602466049039020201CF0E8FC0020009001900290034603225C49039021201CF0DDFC002000900190029003460322CB
:409000005749039022201CF0D2FC0020009001900290034603225349039023201CF0C7FC0020009001900290034603224E49039024201CF0BCFC00200090019002900346D0
:4090400003224A49039025201CF0B1FC0020009001900290034603224549039026201CF0A6FC0020009001900290034601224149039027201CF09BFC002000900190029038
:40908000034601223C49039028201CF090FC0020009001900290034601223849039029201CF085FC002000900190029003460222334903902B201CF07AFC002000900190C6
:4090C0000290034602222F4903902C201CF06FFC002059E02807002029070020D8060020D9060020D7060020150700200C070020BE06002001070020BB060020BA06002075
:40910000E8060020E7060020E9060020E6060020CB0600202B0700202C070020EB060020EC060020FF060020FE060020FD0600201F070020B5060020F1060020A7060020CF
:40914000A8060020AD0600202D0700202E070020AC060020B1060020B8060020A1060020A3060020F4060020F5060020F6060020F7060020F9060020F8060020FA060020C3
:40918000FB060020FC06002000900190029003460122FE4903902D201CF009FC002000900190029003460122F94903902E201CF0FEFB002000900190029003460122F54931
:4091C00003902F201CF0F3FB002000900190029003460122F049039031201CF0E8FB002000900190029003460122EC49039032201CF0DDFB00200121CDE9000103460A4679
:40920000CDE90210E64936201CF0D1FB002000900190029003460122E24903903B201CF0C6FB002000900190029003460122DE4903903C201CF0BBFB00200122CDE90002D2
:4092400002900346D94903903D201CF0B0FB00200122CDE9000202900346D54903903E201CF0A5FB002001210090CDE9010103460A46D049039041201CF099FB0020009039
:409280000190029003460122CB49039042201CF08EFB002000900190029003460122C749039043201CF083FB002000900190029003460122C249039044201CF078FB0020D2
:4092C00001210090CDE9010103460A46BD49039048201CF06CFB002001210090CDE9010103460A46B84903904B201CF060FB002001210090CDE9010103460A46B3490390BC
:409300004D201CF054FB002000900190029003460322AF4903904F201CF049FB012000220092CDE9012013460246AA49039050201CF03DFB002001210090CDE90101034680
:409340000A46A549039051201CF031FB002000900190029003460122A049039052201CF026FB0020009001900290034603229C49039054201CF01BFB0020009001900290F7
:40938000034603229749039055201CF010FB0020009001900290034603229349039056201CF005FB0020009001900290034603228E49039057201CF0FAFA002000900190AB
:4093C0000290034603228A49039058201CF0EFFA0020009001900290034603228549039059201CF0E4FA002000900190029003460322814903905A201CF0D9FA00200090EE
:4094000001900290034603227C4903905B201CF0CEFA002001210090CDE9010103460A46774903905C201CF0C2FA002000900190029003460122734903905D201CF0B7FA72
:409440000020009001900290034601226E4903905E201CF0ACFA0020009001900290034601226A4903905F201CF0A1FA00200222CDE90002029003460122654903906120CC
:409480001CF095FA00200222CDE900020290034601226049039062201CF089FA0020009001900290034601225B49039064201CF07EFA00200090019002900346012257496D
:4094C000039065201CF073FA002001210090CDE9010103460A465249039067201CF067FA002001210090CDE9010103460A464D49039069201CF05BFA00200222CDE9000264
:40950000029003460246484903906A201CF04FFA01200021009101910B460246CDE9021042496B201CF043FA00200222CDE90002029003463E4903906D201CF038FA002004
:409540000222CDE90002029003463A4903906E201CF02DFA00200222CDE9000202900346354903906F201CF022FA002001210090CDE9010103460A463049039073201CF0F0
:4095800016FA002002225BE053E10000ED060020EF060020EE0600200007002001070020020700200407002005070020060700200707002008070020D2060020090700202B
:4095C0000A0700202F070020300700201E070020EA0600200B0700200C0700200D07002034070020350700203607002038070020120700201307002014070020AF060020A9
:4096000015070020170700201807002016070020F3060020F2060020190700201A0700201B0700201D070020DF060020CC06002031070020320700203307002020070020B3
:40964000CDE90002029003460246FE49039079201CF0ADF9002000900190029003460222F94903907A201CF0A2F9002000900190029003460122F54903907B201CF097F94D
:40968000002000900190029003460122F04903907C201CF08CF9002000900190029003460122EC4903907D201CF081F9002001210090CDE9010103460A46E74903907E20C4
:4096C0001CF075F9002000900190029003460122E24903907F201CF06AF9002001210090CDE9010103460222DD49039082201CF05EF9002001210090CDE901010346022239
:40970000D849039083201CF052F9002001210090CDE9010103460222D349039084201CF046F901200021009101910B460222CDE90210CE4986201CF03AF901200021009175
:4097400001910B460222CDE90210C94987201CF02EF901200021009101910B460246CDE90210C44988201CF022F9002000900190029003460322C04903908E201CF017F9E5
:40978000002000900190029003460322BB4903908F201CF00CF9002000900190029003460322B74903908F201CF001F9012009F040FE0021B34800781CF022F80021B2485B
:4097C00000781CF01DF80021B04800781CF018F80021AF4800781CF013F801200021009101910B460222CDE90210AA4986201CF0DEF801200021009101910B460222CDE9CF
:409800000210A54987201CF0D2F80121A34800781CF07BFC0121A24800781CF076FC0121A04800781CF071FC01219F4800781CF06CFC1FBD1FB500200090019002900346E5
:4098400003229A49039001201CF0B1F80020009001900290034603229549039002201CF0A6F80020009001900290034603229149039010461CF09BF8002000900190029083
:40988000034603228C49039004201CF090F80020009001900290034604228849039005201CF085F80020009001900290034603228349039006201CF07AF800200090019041
:4098C0000290034603227F49039007201CF06FF80020009001900290034603227A49039008201CF064F80020009001900290034602225549039009201CF059F800200090A5
:4099000001900290034602227049039017201CF04EF80020009001900290034602466C49039019201CF043F80020009001900290034603226749039021201CF038F8002075
:40994000009001900290034603226349039022201CF02DF80020009001900290034602224D49039027201CF022F80020009001900290034602224749039028201CF017F878
:409980000020009001900290034602465349039029201CF00CF801200021009101910B460A46CDE902104E492A201CF000F80020009001900290034602464A4903902B2033
:4099C0001BF0F5FF002000900190029003460122454903902D201BF0EAFF002000900190029003460246414903902E201BF0DFFF0020009001900290034602463C49039093
:409A00002F201BF0D4FF0020009001900290034602463849039030201BF0C9FF0020009001900290034602463349039046201BF0BEFF0020009001900290034602462F49E1
:409A400003905DE02207002023070020C5060020C6060020240700202507002021070020CF060020D0060020D1060020270700202807002029070020D8060020D906002001
:409A8000D7060020150700200C070020BE06002001070020BB060020BA060020E8060020E7060020E9060020E6060020F4060020A1060020A2060020A3060020A4060020FB
:409AC000F7060020A5060020A6060020D3060020AB060020AE060020AF060020BC060020B5060020B2060020DC060020DD060020DE060020DF060020B0060020E1060020BF
:409B000047201BF054FF002000900190029003460246F649039048201BF049FF002000900190029003460122F149039057201BF03EFF002000900190029003460222ED492E
:409B4000039059201BF033FF002000900190029003460222E84903905A201BF028FF002000900190029003460122E44903905B201BF01DFF0020009001900290034601220C
:409B8000DF4903905C201BF012FF002000900190029003460122DB4903905D201BF007FF002000900190029003460122D64903905E201BF0FCFE002000900190029003463E
:409BC0000122D24903905F201BF0F1FE002000900190029003460122CD49039060201BF0E6FE002000900190029003460122C949039061201BF0DBFE0020009001900290A8
:409C000003460122C449039064201BF0D0FE002000900190029003460122C049039065201BF0C5FE002000900190029003460122BB49039066201BF0BAFE0020009001902D
:409C4000029003460122B749039067201BF0AFFE002000900190029003460122B249039068201BF0A4FE002000900190029003460122AE49039069201BF099FE002000906E
:409C80000190029001231A46A94903906A201BF08EFE002000900190029003460122A54903906C201BF083FE002000900190029003460122A04903906D201BF078FE002096
:409CC000009001900290034601229C4903906E201BF06DFE01200021009101910B460A46CDE9021096497C201BF061FE01200021009101910B460A46CDE9021091497D20D1
:409D00001BF055FE002001210090CDE9010103460A468D49039081201BF049FE0020009001900290034602228849039082201BF03EFE0020009001900290034602228449AC
:409D4000039083201BF033FE0020009001900290034602227F49039084201BF028FE0020009001900290034602227B49039086201BF01DFE0020009001900290034602225E
:409D80007649039087201BF012FE0020009001900290034602467249039088201BF007FE0020009001900290034603226D4903908D201BF0FCFD00200090019002900346CE
:409DC0000322694903908E201BF0F1FD002000900190029003460322644903908F201BF0E6FD0121584800781BF00AFD0121604800781BF005FD01215E4800781BF000FD51
:409E00001FBD1FB500240CE000205B4901EB041189680870584901EB0411C9680870601CC4B2902CF0DB1BF03DFC1CF0DBFA1FF031FE0121022022F0A6F9002000900190D7
:409E40000290034601224D49039016201BF0AFFD002001210090CDE9010103460A46484903901E201BF0A3FD002000900190029003460122434903906B201BF098FD1BF00A
:409E8000BCFCFF2831D00121084622F07CF90121042022F078F90121082022F074F90121102022F070F90121202022F06CF90121402022F068F90121802022F064F901214B
:409EC000080222F060F91BF098FC0A2862D2DFE800F06105060708095B5C5D5E00BF00BF00BF00BFFFF7A6FC55E055E0B1060020E5060020BD060020BE060020BF060020AF
:409F0000C0060020C1060020E2060020E3060020E4060020C20600200507002006070020C5060020C6060020C7060020C8060020C9060020CC060020CD060020CE0600207E
:409F4000B8060020B7060020D2060020CF060020D0060020D1060020E8060020E7060020D4060020D7060020D8060020D9060020D5060020D6060020B0510408A70600206C
:409F8000AC060020CB06002000BF00BF00BFFEF7CBF900E000BF00BF1FBD10B50120FE4908701DF0A8FFFC494860012021F09CFF1CE0612021F03AFF78B145F25550F7498F
:409FC00008600120486040F6B83088604CF6CC4008600220F049087008E0EF4948681DF0B2FF642802D90320EB490870EA4800780128DED010BD10B50020E74908704FF4BF
:40A00000FA701DF051FFFA201DF08FFFFFF7C5FFFFF7F7FE1BF0B2FBC8B1E14800781BF0F1FF40B90121DF4800781BF0E9FB0020DD4908700BE0DD4800781BF0E3FF18B18D
:40A040000220D949087002E00120D74908701AF007FEEEF737F900221146D548DFF854C300DF002010BD10B572B66FF0040000F059FA6FF0010000F055FA4FF0FF3000F085
:40A0800051FA042000F04EFA052000F04BFA062000F048FA072000F045FA082000F042FA092000F03FFA0A2000F03CFA0B2000F039FA0C2000F036FA0D2000F033FA0E20E9
:40A0C00000F030FA0F2000F02DFA102000F02AFA112000F027FA122000F024FA132000F021FA142000F01EFA152000F01BFA162000F018FA172000F015FA182000F012FAE4
:40A10000192000F00FFA1A2000F00CFA1B2000F009FA1C2000F006FA1D2000F003FA1E2000F000FA1F2000F0FDF9202000F0FAF9212000F0F7F9222000F0F4F9232000F056
:40A14000F1F9242000F0EEF9252000F0EBF9262000F0E8F9272000F0E5F9282000F0E2F9292000F0DFF92A2000F0DCF92B2000F0D9F92C2000F0D6F92D2000F0D3F92E20F3
:40A1800000F0D0F92F2000F0CDF9302000F0CAF9312000F0C7F9322000F0C4F9332000F0C1F9342000F0BEF9352000F0BBF9362000F0B8F9372000F0B5F9382000F0B2F90E
:40A1C000392000F0AFF93A2000F0ACF93B2000F0A9F93C2000F0A6F93D2000F0A3F93E2000F0A0F93F2000F09DF9402000F09AF9412000F097F9422000F094F9432000F0FC
:40A2000091F9442000F08EF9452000F08BF9462000F088F9472000F085F9482000F082F9492000F07FF94A2000F07CF94B2000F079F94C2000F076F94D2000F073F94E20F2
:40A2400000F070F94F2000F06DF9502000F06AF9512000F067F96FF0040000F06CF96FF0010000F068F94FF0FF3000F064F9042000F061F9052000F05EF9062000F05BF9D4
:40A28000072000F058F9082000F055F9092000F052F90A2000F04FF90B2000F04CF90C2000F049F90D2000F046F90E2000F043F90F2000F040F9102000F03DF9112000F0C7
:40A2C0003AF9122000F037F9132000F034F9142000F031F9152000F02EF9162000F02BF9172000F028F9182000F025F9192000F022F91A2000F01FF91B2000F01CF91C2015
:40A3000000F019F91D2000F016F91E2000F013F91F2000F010F9202000F00DF9212000F00AF9222000F007F9232000F004F9242000F001F9252000F0FEF8262000F0FBF81F
:40A34000272000F0F8F8282000F0F5F8292000F0F2F82A2000F0EFF82B2000F0ECF82C2000F0E9F82D2000F0E6F82E2000F0E3F82F2000F0E0F8302000F0DDF8312000F070
:40A38000DAF8322000F0D7F8332000F0D4F8342000F0D1F835200FE0A803002000300040B2060020CE060020A4030020DF060020774802087510040800F0BDF8362000F042
:40A3C000BAF8372000F0B7F8382000F0B4F8392000F0B1F83A2000F0AEF83B2000F0ABF83C2000F0A8F83D2000F0A5F83E2000F0A2F83F2000F09FF8402000F09CF8412008
:40A4000000F099F8422000F096F8432000F093F8442000F090F8452000F08DF8462000F08AF8472000F087F8482000F084F8492000F081F84A2000F07EF84B2000F07BF835
:40A440004C2000F078F84D2000F075F84E2000F072F84F2000F06FF8502000F06CF8512000F069F862B610BD38B5044660680090009D206880F3088800BFA84738BD00BF34
:40A48000BFF34F8F3048006800F4E0602F490843001D2D490860BFF34F8F00BF00BFFEE710B500212A4800781BF0AAF90021294800781BF0A5F90021274800781BF0A0F96A
:40A4C00001DF10BD01B500BF04226946234800688C3000F04BF818B921480099C0F87C1400BF08BD01B500BF042269461B480068903000F03BF818B919480099C0F88014F5
:40A5000000BF08BD01B500BF0422694613480068943000F02BF818B911480099C0F8841400BF08BD00F01F02012191400D4A430942F82310704700F01F02012191400A4AF9
:40A54000430942F8231070470CED00E00000FA05060700200407002005070020B8030020301F002080E100E080E200E070B504460D461646324629462046EEF746FC70BD83
:40A580002DE9F34F82B0844600BF00210A460B460E460F46002001908046009063E09CF80000A0F13004E5179CF800002E2838D1B8F1000F0CD1F9494FF00009A2FB010AC4
:40A5C00003FB01A102FB0919861949EB07071FE0B8F1010F0CD1F2494FF00009A2FB010A03FB01A102FB0919861949EB07070FE0B8F1020F0CD14FF47A714FF00009A2FBC2
:40A60000010A03FB01A102FB0919861949EB070708F1010000F0FF0800200090002213461BE09CF80000C0B1009810B922462B460FE0009801280CDB0A214FF0000B914636
:40A64000A9FB010E03FB01E102FB0B19021949EB05030098401CC0B200900CF1010C0198401CC0B2019003990198884297DBB6185F413046394604B0BDE8F08F2DE9F04FD6
:40A6800083468946924600BF00BF51465846FFF777FF05460E4651464846FFF771FF07468846781B78EB060001DA012407E0E81B76EB080002DA4FF0FF3400E000242046BF
:40A6C000BDE8F08FF0B585B00546B6A2B8A101A822F0A0FE1022294601A8FFF7CFFF00283CDDB44890F82464012434E0062C0CD2DFE804F00B0C09070503AF4F08E0AF4F95
:40A7000006E0AF4F04E0AF4F02E000BFAE4F00BF00BF40F6C41000900222694607F56070FFF724FFB44204D1BDF80000A149A1F880034FF47A5000900222694607F2823044
:40A74000FFF714FFB44204D1BDF800009949A1F88203601CC4B2052CC8DD00BF05B0F0BD2DE9F04105460E4617463A4631462846EEF7C1FB044604B103DF2046BDE8F081C1
:40A78000F0B585B0054691A289A101A822F042FE1022294601A8FFF771FF00282FDD854890F82474012427E0062C0CD2DFE804F00B0C09070503804E08E0804E06E0804EED
:40A7C00004E0804E02E000BF7F4E00BF00BF042206F5C6716846FFF7C3FF0422694606F56270FFF7C3FEBC4204D19DED000A714880EDE20A601CC4B2052CD5DD00BF05B0E2
:40A80000F0BDF0B585B0054673A269A101A822F001FE1022294601A8FFF730FF00282BDD644890F82464012423E0062C0CD2DFE804F00B0C090705035F4F08E05F4F06E0C6
:40A840005F4F04E05F4F02E000BF5F4F00BF00BF002000900122694607F19700FFF786FEB44204D19DF80000524981F89700601CC4B2052CD9DD00BF05B0F0BD2DE9F041F4
:40A8800086B0054657A24AA102A822F0C3FD1022294602A8FFF7F2FE002836DD002001900026444890F8247400242BE0062C13D2DFE804F0130F0C090603DFF8FC800FE045
:40A8C000DFF8F8800CE0DFF8F88009E0DFF8F48006E0DFF8F48003E000BFDFF8148100BF00BF042201A908F1B400FFF73FFEBC4206D130490198C1F8B4000846C0F89860DB
:40A90000601CC4B2052CD1DD00BF06B0BDE8F081F0B587B0064637A225A103A822F07AFD1022314603A8FFF7A9FE002869DD214890F82474002483E0062C0ED2DFE804F084
:40A940000E0B090705031C4D0AE01C4D08E01C4D06E01C4D04E01C4D02E000BF244D00BF00BF042205F1300101A8FFF7F9FE13208DF809000198F0F7E6FF18B90198F1F712
:40A980000CF818B190208DF808003EE00198F0F7FCFFA8B313208DF8080036E000CA9A3B40420F00322E342E302E35330000000025730000301F0020581B0068701700683A
:40A9C00088130068A00F0068B80B0068322E342E302E343400000000322E332E302E333000000000322E322E302E343600000000D0070068322E322E302E313800000000BA
:40AA000000E021E0FF208DF8080001220DF1090105F1B300FFF7AAFD012202A905F1B200FFF7A4FDBC4209D19DF80910FE4880F8B3109DF80800FC4981F8B200601CC4B205
:40AA4000052C7FF779AF00BF07B0F0BDF0B585B00546F6A2AFF2A80101A822F0DBFC1022294601A8FFF70AFE00282DDDEE4890F8246401200090002423E0062C0ED2DFE8DA
:40AA800004F00E0B09070503EA4F0AE0EA4F08E0EA4F06E0EA4F04E0EA4F02E000BFEA4F00BF00BF0122694607F14B00FFF75EFDB44204D19DF80000DB4981F84B00601C36
:40AAC000C4B2052CD9DD00BF05B0F0BDF0B587B00546DEA2AFF2281103A822F09BFC1022294603A8FFF7CAFD002839DDCE4890F82474002431E0062C0ED2DFE804F00E0B6B
:40AB000009070503CB4E0AE0CB4E08E0CB4E06E0CB4E04E0CB4E02E000BFCB4E00BF00BF012206F1280102A8FFF71AFE9DF80800042810D0B2EE040A8DED010A042201A905
:40AB400006F5FC70FFF712FDBC4204D19DED010AB54880ED7E0A601CC4B2052CCBDD00BF07B0F0BDF0B585B00646BAA2AFF2C01101A822F04FFC1022314601A8FFF77EFD64
:40AB8000002843DD0727B6A2AFF2DC1101A822F041FC1022314601A8FFF770FD002800DD09270020009000242DE0062C0ED2DFE804F00E0B090705039E4D0AE09E4D08E0D0
:40ABC0009E4D06E09E4D04E09E4D02E000BF9E4D00BF00BF042205F130016846FFF7C0FD009838440090009814280BD30422694605F13000FFF7BAFC9348854202D18A49CD
:40AC000000980863641C062CCFD300BF05B0F0BD2DE9F3410D468449ADEB01040846071988482618AAB239463046FFF79FFC7E48071983482618AAB239463046FFF796FC6F
:40AC4000794807197D482618AAB239463046FFF78DFC7548071978482618AAB239463046FFF784FC7048071972482618AAB239463046FFF77BFCBDE8FC812DE9FE4F8146A4
:40AC80008A46174698460020009000262D2200233846414622F033FB05462D2200233846414622F02CFB934615B9BBF1000F35D0D5B1002416E0C4EB041000EB4000484480
:40ACC0000290C4EB041000EB4000504401902D22DDE90110FFF74AFC0646009931430091601CC4B2AC42E6D3BBF1000F18D0C5EB051000EB400048440290C5EB051000EB69
:40AD00004000504401901FFA8BF2DDE90110FFF72DFC064600993143009101E0402000900098BDE8FE8F01B500BF012269464F4800682D30FFF71AFC20B99DF800103A48EE
:40AD400080F81D1400BF08BD2DE9FE4F81468A46174698460020009000262D2200233846414622F0CCFA05462D2200233846414622F0C5FA934615B9BBF1000F35D0D5B1CC
:40AD8000002416E0C4EB041000EB400048440290C4EB041000EB4000504401902D22DDE90110FFF7DDFC0646009931430091601CC4B2AC42E6D3BBF1000F18D0C5EB05107A
:40ADC00000EB400048440290C5EB051000EB4000504401901FFA8BF2DDE90110FFF7C0FC064600993143009101E0402000900098BDE8FE8F3EB5002002900A2001900020D1
:40AE000000904FF47C71084822F08DFCB021184822F089FC4FF458711548B03022F083FC012201A9114825E0301F0020322E322E302E3200581B006870170068881300680E
:40AE4000A00F0068B80B0068D0070068322E322E302E3100322E312E302E373300000000322E312E302E353400000000B80300202023002000689830FFF778FB0122FB48B8
:40AE80000168983102A8FFF76BFC9DF80800401CC0B20190012201A9F44800689830FFF765FB0122F1480168983102A8FFF758FC9DF808009DF80410884207D0EC480078B9
:40AEC00040F08000EA49087001248CE00122E74801682E316846FFF743FC9DF8000044284CD0FF224FF47C71E248F0F79FFF4FF47C720023DF49E048FFF7BFFE4FF47C72C4
:40AF00000023DC49DD48FFF7B8FE4FF47C720023D849DB48FFF7B1FE4FF47C720023D549D848FFF7AAFE4FF47C720023D149D648FFF7A3FE4FF47C720023CE49D348FFF7EC
:40AF40009CFE4FF47C71CB4822F0EDFBB0220023CF494FF0D040FFF790FE4FF458720023CB49B031CB48FFF788FE4420009001226946BE4800682E30FFF7F8FAB0220023F7
:40AF80004FF0D041C248FFF7DFFE4FF458720023C049BF48B030FFF7D7FE0122B34801682D31BB482D30FFF7DBFBB24890F81D04672810D001246720FFF7B5FE4FF47C71D1
:40AFC000AC4822F0B0FB4FF47C720023A949AA48FFF753FE07E002244FF47C720023A649A448FFF7B1FE20463EBD10B5AA48EDF7BBFE0446204610BD70B58CB00024002069
:40B00000089009900A900B9004900590069007900090019002900390954908709F49087001200870FFF7E1FFFFF7E4FE9C4908709C4AAFF2846108A822F0ECF904A81BF0EA
:40B04000C9F999A104A822F095FB08B1012000E00020054645B196A01BF0A8F992A01BF0A5F997A01BF088F904A81BF097F9102204A908A8FFF702FB044689480078012866
:40B0800006D100208549087008A81BF075F9C3E0002CFCD0002007F015F8002007F065F808A81BF069F9002C39DA0020FFF73BFEFF224FF47C716F48F0F7B8FE4FF47C7276
:40B0C00000236C496C48FFF7D8FD4FF47C72002368496A48FFF7D1FD4FF47C72002365496748FFF7CAFD4FF47C72002361496548FFF7C3FD4FF47C7200235E496248FFF714
:40B10000BCFD4FF47C7200235A496048FFF7B5FD4FF47C71574822F006FB03DF7CE06AA2AFF27471684622F075F9102204A96846FFF7A4FA002838DD0020FFF7F4FDFF22A9
:40B140004FF47C714B48F0F771FE4FF47C72002348494948FFF791FD4FF47C72002345494648FFF78AFD4FF47C72002341494448FFF783FD4FF47C7200233E494148FFF795
:40B180007CFD4FF47C7200233A493F48FFF775FD4FF47C72002337493C48FFF76EFD4FF47C71344822F0BFFA03DF4AA2AFF60001684622F02FF9102204A96846FFF75EFAE9
:40B1C000002811DD012009F0D2F801212948B130FFF71EFD1AF0D2FA30B10320F0F728FF01213F48FFF714FD04A8FFF7BBFC04A8FFF76CFC04A8FFF729FC04A8FFF788FBE9
:40B2000004A8FFF73BFB04A8FFF7FBFA04A8FFF7B7FA04A8FFF756FA0020F0F760F90020F0F770F9F0F705FD0646F0F702FC1B4800780CB070BD19480078704701B500BFA7
:40B2400001226946094800683430FFF78FF920B99DF80010074880F8241400BF2148C16B0220DFF884C000DF08BD0000B8030020B1030020301F0020D0070068B80B006827
:40B28000A00F00688813006870170068581B006820230020F401006800380040B2030020B00300209CBE0008322E302E310000003030303030303030303030300000000039
:40B2C000322E302E302E3100322E302E302E363500000000322E312E302E333900000000E320002050410020610804087CB505460E46FE4C042204F1340101A8FFF730FA75
:40B30000012204F1B1016846FFF72AFA0198854205D19DF80000B04201D101207CBDF44C042204F1340101A8FFF71AFA012204F1B1016846FFF714FA0198854205D19DF808
:40B340000000B04201D10220E8E7EA4C042204F1340101A8FFF704FA012204F1B1016846FFF7FEF90198854205D19DF80000B04201D10320D2E7E04C042204F1340101A800
:40B38000FFF7EEF9012204F1B1016846FFF7E8F90198854205D19DF80000B04201D10420BCE7D64C042204F1340101A8FFF7D8F9012204F1B1016846FFF7D2F90198854290
:40B3C00005D19DF80000B04201D10520A6E70020A4E738B5C54C042204F5EC716846FFF7BFF940F2FD110098884201D0012038BDBF4C042204F5EC716846FFF7B1F940F25B
:40B40000FD110098884201D00220F0E7B94C042204F5EC716846FFF7A3F940F2FD110098884201D00320E2E7B34C042204F5EC716846FFF795F940F2FD110098884201D092
:40B440000420D4E7AD4C042204F5EC716846FFF787F940F2FD110098884201D00520C6E70020C4E710B54FF47C71A54822F05BF94FF47C720023A249A248FFF7FEFB10BD17
:40B4800010B54FF47C719E4822F04DF94FF47C7200239B499B48FFF7F0FB4FF47C72002397499248FFF7E9FB4FF47C72002394498F48FFF7E2FB4FF47C72002390498D4898
:40B4C000FFF7DBFB4FF47C7200238D498A48FFF7D4FB4FF47C72002389498848FFF7CDFB4FF47C71864822F01EF910BD2DE9F0410446884615461F463CB982482E183A4673
:40B5000041463046FFF732F830E0012C07D177482E183A4641463046FFF728F826E0022C07D173482E183A4641463046FFF71EF81CE0032C07D16F482E183A46414630462E
:40B54000FFF714F812E0042C07D16B482E183A4641463046FFF70AF808E0052C06D167482E183A4641463046FFF700F8BDE8F0812DE9F04104460F46154698463CB961483E
:40B580002E18424631463846FFF7EAF830E0012C07D156482E18424631463846FFF7E0F826E0022C07D152482E18424631463846FFF7D6F81CE0032C07D14E482E18424618
:40B5C00031463846FFF7CCF812E0042C07D14A482E18424631463846FFF7C2F808E0052C06D146482E18424631463846FFF7B8F8BDE8F08110B5424890F82444062C2CD231
:40B60000DFE804F02C030B131B234FF47C7200233B493648FFF731FB21E04FF47C72002337493348FFF729FB19E04FF47C72002333493048FFF721FB11E04FF47C7200234A
:40B640002F492D48FFF719FB09E04FF47C7200232B492A48FFF711FB01E000BF00BF00BF10BD70B505460E4631462846FFF73EFE0446062C6CD2DFE804F06C031527475928
:40B680004FF47C72002319491D48FFF75DFB4FF47C7200231A491B48FFF7EFFA0120FFF7CDFD62E04FF47C72002311491448FFF74BFB4FF47C72002311491248FFF7DDFAEA
:40B6C0000220FFF7BBFD50E04FF47C72002309490B48FFF739FB4FF47C72002308490948FFF7CBFA0320FFF7A9FD3EE0B80B0068A00F00688813006870170068581B00688A
:40B70000301F0020D00700684FF47C72002339493948FFF719FB4FF47C72002336493748FFF7ABFA0420FFF789FD1EE04FF47C72002333493048FFF707FB4FF47C720023DB
:40B740002D492E48FFF799FA0520FFF777FD0CE000BFFFF787FE0020FFF770FD002029494860222014F086F900BF00BF04B103DF70BD4FF40050704710B51F4890F82404B5
:40B78000062831D2DFE800F031030C151E271E4C042219493C3104F13C00FEF7E7FE25E01A4C042214493C3104F13C00FEF7DEFE1CE0174C042210493C3104F13C00FEF7CF
:40B7C000D5FE13E00B4C04220B493C3104F13C00FEF7CCFE0AE00A4C042207493C3104F13C00FEF7C3FE01E000BF00BF00BF10BD0848704770170068301F0020D0070068BC
:40B80000581B006844310020B80B0068A00F006888130068FF57F63B10B51CF06CFBFE49086005F0B6FBFC4880ED010A10BD10B5FA4890F84A00022824D1F84890F8BD0138
:40B8400002281FD1F64890ED020ADFEDF60AB4EEE00AF1EE10FA0ADBFBF7C6FFC4B223467D22ED490C3101200DF0FEF82EE0FBF7BBFFC4B223467D22E7490C3100200DF043
:40B88000F3F823E0E648D0ED010AE448B0F8BE0100EE100AB8EE400AF4EEC00AF1EE10FA0ADBFBF7A1FFC4B22346FA22DA490C3101200DF0D9F809E0FBF796FFC4B2234674
:40B8C000FA22D5490C3100200DF0CEF810BD10B52DED048B19F06AFF002867D0FFF7A7FFEEF7C5FD18B10020CB49087261E0CA48007A60B9C84890F82000002859D1012017
:40B90000C54908721CF0F7FAC349086051E0C248007A01280CD1C049C86947F230511CF0F0FAA0B30220BC490872FFF775FF40E0B948007A02283CD105F02BFBB648D0ED63
:40B94000010A30EEC00A10EE104A204626F06EFC41EC190BB0EE490AF0EE690A23F040F8B0EE408AF0EE608A9FEDAF0B53EC102B51EC180B26F062FA0ED2A74890F820007F
:40B98000012805D10020A44948720120087210E00120A14948720CE09F4908684FF4FA611CF0AFFA28B1FFF737FF02E000209A494872BDEC048B10BD994981F8900070478F
:40B9C000974981F838007047F0EE400A9FED980A20EE800A704770B52DED0A8B82B004468E4890F8BD010F287ED2DFE800F07D365EFC37FBFAF97D7D087DF8F7F600EEF735
:40BA000032FD10EE105A284626F010FC41EC1A0BB0EE4A0AF0EE6A0A22F0E2FFB0EE409AF0EE609A51EC190B25F0C4FDA0619FED810A84ED1C0A94ED060A84ED010AEEF72E
:40BA40005AFD18B10020FFF7BBFF02E00320FFF7B7FF0320FFF7B0FF6AE200BF764800781AF0D0FA20B19FED750A84ED060A03E09FED700A84ED060A714800781AF0C2FA8A
:40BA800020B19FED6E0A84ED1C0A03E09FED690A84ED1C0A0320FFF793FF0320FFF78CFF94ED060A84ED010AEAE3634800781AF06DF800EE100AF8EE400A9FED621A9FED1A
:40BAC000620A10EE810A84ED0C0AE16821611CF012FAE060D4E90310091A6161D4ED0C0AB0EE600A0A2100E0BBE304F118000AF0BDFA94ED060ADFED550AB4EEE00AF1EE85
:40BB000010FA03D20020FFF75BFF0FE094ED060AF0EE040AB4EEE00AF1EE10FA03DD0120FFF74EFF02E00320FFF74AFF0320FFF743FF94ED0C0AB5EEC00AF1EE10FA02D231
:40BB40009FED3C8A01E094ED068A94ED0F0A84ED100A84ED0F8A94ED050AB8EE400ADFED370A80EE201A11EE105A284626F05EFB41EC1A0B94ED0F0AD4ED100A30EE600A88
:40BB800010EE101A084626F051FB41EC1C0BB0EE4C0AF0EE6C0A22F023FFB0EE40BAF0EE60BA53EC1A2B51EC1B0B25F0F1FD41EC190B25F0FFFC60639FED1E0A84ED1C0AF4
:40BBC000B0EE480AFFF700FF84ED010AD4ED0D0AB0EE600AFFF7F8FE06E0D5E2A9E1E2E2F7E112E103E069E084ED020A48E31248007819F0CBFF00EE100AB8EE400ADFED25
:40BC0000110A20EE200ADFED120A80EE201A84ED0C1AD4ED0C0A1DE030270020301F00205427002000C0DA44000000401857B63FC0A9064600000000E606002000007A4434
:40BC4000EA0600203333533A9A99193FCDCCCCBE0CAC233FB0EE600A0A2104F118000AF005FA94ED060ADFEDFE0AB4EEE00AF1EE10FA03D20020FFF7A3FE0FE094ED060ADA
:40BC8000DFEDF80AB4EEE00AF1EE10FA03DD0120FFF796FE02E00320FFF792FE0320FFF78BFE1FED1C0A84ED1C0AD4ED060AB0EE600AFFF789FE84ED010AE1E2EA48007881
:40BCC00019F064FF00EE100AF8EE400A1FED231A1FED230A10EE810A84ED0C0AD4ED0C0AB0EE600A0A2104F118000AF0BFF994ED060A5FED2A0AB4EEE00AF1EE10FA03D2EA
:40BD00000020FFF75DFE0FE094ED060AF0EE040AB4EEE00AF1EE10FA03DD0120FFF750FE02E00320FFF74CFE94ED0C0AB5EEC00AF1EE10FA02D21FED418A01E094ED068A9D
:40BD4000CA48007819F022FF00EE100AF8EE400A1FED441A1FED440A10EE810A84ED220AD4ED220AB0EE600A0A2104F170000AF07DF994ED1C0A5FED4B0AB4EEE00AF1EE45
:40BD800010FA03D20020FFF717FE0FE094ED1C0AF0EE040AB4EEE00AF1EE10FA03DD0120FFF70AFE02E00320FFF706FE94ED220AB5EEC00AF1EE10FA02D25FED628A01E094
:40BDC000D4ED1C8AB0EE480AFFF7FEFDB0EE401AB0EE680AFFF7F8FD31EE400A10EE105A284626F023FA41EC1A0BB0EE4A0AF0EE6A0A22F0F5FDB0EE409AF0EE609A51EC6F
:40BE0000190B25F0D7FB60603AE29748007819F0BDFE00EE100AB8EE400A5FED760A20EE200A5FED750A80EE201A84ED0C1AD4ED0C0AB0EE600A0A2104F118000AF016F9DA
:40BE400094ED060ADFED860AB4EEE00AF1EE10FA03D20020FFF7B4FD0FE094ED060ADFED810AB4EEE00AF1EE10FA03DD0120FFF7A7FD02E00320FFF7A3FD7C48007819F0FD
:40BE800085FE00EE100AB8EE400A5FED920A20EE200A5FED910A80EE201A84ED221AD4ED220AB0EE600A0A2104F170000AF0DEF894ED1C0ADFED6A0AB4EEE00AF1EE10FAFA
:40BEC00003D20020FFF778FD0FE094ED1C0ADFED650AB4EEE00AF1EE10FA03DD0120FFF76BFD02E00320FFF767FD94ED060AD4ED1C0A30EE600A10EE101A084626F096F9C3
:40BF000041EC1B0BB0EE4B0AF0EE6B0A22F068FDB0EE40AAF0EE60AA51EC1A0B25F04AFB09EE100AB0EE490AFFF74EFD84ED010AA6E16421E0681BF0E4FFE0B31BF0DBFF4C
:40BF4000E06094ED0F0A84ED100A494800781DF078FF00EE100AB8EEC00A84ED0F0A94ED0F0AD4ED100A30EE600A10EE101A084626F05CF941EC1A0BB0EE4A0AF0EE6A0A59
:40BF800022F02EFDB0EE409AF0EE609A51EC190B25F010FB206394ED0C0ADFED360A80EE201A84ED0C1AD4ED0C0AB0EE600A032104F1180000E00BE00AF058F894ED060A58
:40BFC00084ED010A0320FFF7FBFC0320FFF7F4FC56E16421E0681BF094FF00287DD01BF08AFFE06094ED0F0A84ED100A1E4800781DF027FF00EE100AB8EEC00A84ED0F0A89
:40C0000094ED0F0AD4ED100A30EE600A10EE101A084626F00BF941EC1A0BB0EE4A0AF0EE6A0A22F0DDFCB0EE409AF0EE609A51EC190B25F0BFFA206394ED0C0ADFED0D0A76
:40C0400080EE201A84ED0C1A94ED250A84ED260A094800781DF0F5FE00EE100A0EE00000CDCCCC3C33339F40E6060020E9060020E8060020CDCCCC3DEA060020B8EEC00A40
:40C0800084ED250A94ED250AD4ED260A30EE600A10EE101A084626F0C9F841EC1A0BB0EE4A0AF0EE6A0A22F09BFCB0EE409AF0EE609A51EC190B25F07DFA8821085194ED6B
:40C0C000220A5FED140A80EE201A84ED221AD4ED0C0AB0EE600A032100E054E004F1180009F0C4FFD4ED220AB0EE600A032104F1700009F0BBFF94ED060AD4ED1C0AB4EE2A
:40C10000E00AF1EE10FA04DD94ED060A84ED010A03E094ED1C0A84ED010AEEF7ECF918B10020FFF74DFC13E094ED1C0AD4ED060A30EE600AF3EE090AB4EEE00AF1EE10FAEA
:40C1400003DD0220FFF73CFC02E00320FFF738FCEEF7DEF918B10020FFF72EFC13E094ED060AD4ED1C0A30EE600AF3EE090AB4EEE00AF1EE10FA03DD0220FFF71DFC02E04C
:40C180000320FFF719FC7BE09FEDFB0A84ED0C0A9FEDF90A84ED010A0320FFF711FC0320FFF70AFC6CE0FA21E0681BF0AAFEE8B36A4601A9F14800781DF096FF05461BF08E
:40C1C0009AFEE06094ED0F0A84ED100A9DED000A84ED0F0A94ED0F0AD4ED100A30EE600A84ED0C0A94ED0C0AF5EE000A80EE201A11EE106A304626F019F841EC1A0BB0EE6E
:40C200004A0AF0EE6A0A22F0EBFBB0EE409AF0EE609A51EC190B25F0CDF92063D4ED0C0AB0EE600A022104F1180000E018E009F01DFF94ED060A84ED010A012D06D19DEDB9
:40C24000010AB5EEC00AF1EE10FA03D10020FFF7B7FB02E00320FFF7B3FB0320FFF7ACFB0EE09FEDC50A84ED0C0A9FEDC30A84ED010A0020FFF7A4FB0020FFF79DFB00BF91
:40C2800000BF02B0BDEC0A8B70BD10B519F0A1FAD0B1FBF7A9FAC4B22346FA22B84900200CF0E2FB9FEDB40AB64880ED060A9FEDB20A80ED060A032180F8381080F89010A8
:40C2C0000020B14948722EE0AE48FFF784FBAF48B0F8BE0118B90220A949087521E0A948D0ED010AA948B0F8BE0100EE100AB8EE400AF4EEC00AF1EE10FA09DBFBF774FA4E
:40C30000C4B22346FA229E4901200CF0ADFB08E0FBF76AFAC4B22346FA22994900200CF0A3FBFFF7D4FA10BD97494872704731B50024BDF80000C82803DDC8200090022472
:40C3400006E0BDF80000012802DA01200090032400BF022269468E48006800F5DF70FEF705F920B9BDF800008849A1F8BE0100BF204638BD31B50024BDF80000642803DD42
:40C3800064200090022406E0BDF80000012802DA01200090032400BF022269467C48006800F5DF70FEF7E2F820B9BDF800007749A1F8BE0100BF204638BD31B50024BDF87B
:40C3C0000000B0F5FA7F04DD4FF4FA700090022406E0BDF80000012802DA01200090032400BF022269466A48006800F5DF70FEF7BDF820B9BDF800006449A1F8BE0100BF77
:40C40000204638BD31B50024BDF80000322803DD32200090022406E0BDF80000012802DA01200090032400BF022269465848006800F5DF70FEF79AF820B9BDF80000534999
:40C44000A1F8BE0100BF204638BD31B50024BDF80000C82803DDC8200090022406E0BDF80000012802DA01200090032400BF022269464748006800F5DF70FEF777F820B99B
:40C48000BDF800004149A1F8BE0100BF204638BD31B50024BDF8000040F26351884203DD08460090022406E0BDF80000012802DA01200090032400BF02226946344800688A
:40C4C00000F5DF70FEF752F820B9BDF800002F49A1F8BE0100BF204638BD31B50024BDF8000045F2CC01884203DD08460090022406E0BDF80000012802DA01200090032458
:40C5000000BF022269462248006800F5DF70FEF72DF820B9BDF800001C49A1F8BE0100BF204638BD10B52DED028BB0EE408A0024164890F8BD010E2853D2DFE800F0072BF4
:40C5400008122C091336522D4052493700BF00BFBCEEC80A10EE101A88B2FFF7BEFF044648E000BFBCEEC80A10EE101A88B2FFF78FFF04463EE0000000000000E60600207C
:40C58000102800205427002030270020301F0020B403002000BF00BFBCEEC80A10EE101A88B2FFF752FF044624E000BFBCEEC80A10EE101A88B2FFF725FF04461AE0BCEE35
:40C5C000C80A10EE101A88B2FFF7F7FE044611E0BCEEC80A10EE101A88B2FFF7CBFE044608E0BCEEC80A10EE101A88B2FFF79FFE044600BF00BF4020F0F7F8FE0020FFF786
:40C6000093FE2046BDEC028B10BD10B52DED020B00BF04226946FE48006800F5E670FDF7A5FF20B99DED000AFA4880ED730A00BFF948016D0120DFF8E4C300DF1CBD10B5CC
:40C640002DED020B00BF04226946F148006800F5E470FDF78BFF20B99DED000AED4880ED720A00BFEC48016D0120DFF8B0C300DF1CBD10B52DED020B00BF04226946E448DC
:40C68000006800F5E270FDF771FF20B99DED000AE04880ED710A00BFDF48016D0120DFF87CC300DF1CBD10B52DED020B00BF04226946D748006800F5E070FDF757FF20B938
:40C6C0009DED000AD34880ED700A00BFD248016D0120DFF848C300DF1CBD10B5CD4890F830000A2818D1CB4890F8BD010A2813D19FEDCB0AFFF716FF9FEDCA0AFFF7D3FFF2
:40C700009FEDC90AFFF7B5FF9FEDC80AFFF797FF9FEDC70AFFF779FFBE4890F83000702819D1BC4890F8BD010A2814D19FEDC10AFFF7F8FE9FEDC00AFFF7B5FF9FEDBF0A02
:40C74000FFF797FF9FEDBE0AFFF779FF9FEDBD0AFFF75BFF18E0AF4890F8BD010A2813D19FEDB40AFFF7DEFE9FEDAE0AFFF79BFF9FEDAD0AFFF77DFF9FEDB30AFFF75FFF3B
:40C78000BBEE040AFFF741FFA24890F8BD01012804D1B7EE000AFFF7C5FE53E09D4890F8BD01022804D19FEDA90AFFF7BBFE49E0984890F8BD01032804D1B3EE040AFFF7B7
:40C7C000B1FE3FE0934890F8BD01042804D11FED960AFFF7A7FE35E08E4890F8BD01052804D19FED9B0AFFF79DFE2BE0894890F8BD01062804D19FED970AFFF793FE21E033
:40C80000844890F8BD01072804D0824890F8BD010D2804D1B1EE040AFFF784FE12E07D4890F8BD01092804D19FED8A0AFFF77AFE08E0784890F8BD010C2803D1B2EE040A6F
:40C84000FFF770FE10BD10B5724890F8BD010A280DD1704890F830000A2803D1FA20FFF7ACFD03E04FF49670FFF7A7FD00E000BF00BF10BD00B589B018F098FF002879D094
:40C88000644890F8BD010E2875D2DFE800F074072A2B4E75769974EFEEEDECEB0020009001900290034602466B4903900846007819F07DF800200090019002900346024648
:40C8C000664903900846007819F071F801216248007819F01AFC01216048007819F015FC89E100BF002000900190029003460322594903900846007819F059F80020009090
:40C900000190029003460322544903900846007819F04DF803215048007819F0F6FB03214E48007819F0F1FB65E101200021009101910B460A46CDE9021047490846007863
:40C9400019F035F801200021009101910B460A46CDE9021041490846007819F028F801213D48007819F0D1FB01213C48007819F0CCFB40E140E119E100BF0020009001901C
:40C98000029003460322344903900846007819F00EF80020009001900290034603222F4903900846007819F002F800212A48007819F0ABFB00212948007819F0A6FB1AE114
:40C9C000002000900190029003460222224903900846007818F0EBFF0020009001900290034603221D4903900846007818F0DFFF0020009001900290034602221849039027
:40CA00000846007818F0D3FF0221134800782EE0B4030020301F0020504100206108040800007A43C6DCB53DB8AF833E52B8444114AE4740000096436744293EE5F25F3E36
:40CA400052B862416666E6C133331B41000016430080BB440000C842E6060020E9060020EA060020A1E081E02DE0A1E09FE019F04CFB0221FB48007819F047FB00200090AF
:40CA80000190034614220121029004A81CF0F8FF04A8DFEDF50A9FEDF50A02230022F4490090F44800781CF0D3FE04A8DFEDEE0A9FEDEE0A02230322EF490090E9480078AD
:40CAC0001CF0C6FE97E0002000900190029003460222E84903900846007818F068FF002000900190029003460322E44903900846007818F05CFF0020009001900290034670
:40CB00000222D84903900846007818F050FF0621D848007819F0F9FA0621D248007819F0F4FA002000900190034614220121029004A81CF0A5FF04A8DFEDCB0A9FEDCB0A17
:40CB400002230022CA490090CA4800781CF080FE04A8DFEDC50A9FEDC50A02230322C6490090C04800781CF073FE44E0002000900190029003460222BE490390084600786B
:40CB800018F015FF0121BB48007819F0BEFABC48DFEDB50A9FEDBB0A05230022B4490090B44800781CF054FE25E024E000BF00BF002000900190029003460322AD49039021
:40CBC0000846007818F0F3FE002000900190029003460322A94903900846007818F0E7FE0121A448007819F090FA0121A348007819F08BFA00BF00BFA34890F8BD01A34936
:40CC000008700020FFF790FB0020A149087209B000BDA049097D012900D100E00021084670479C48407D70479A48007D08B9012070470020FCE7984909880143964A1180F7
:40CC40007047F7EE000AB0EE600A7C2202708E4A92F8BD210E2A22D2DFE802F007120809130A0B1721141B211E1800BF00BF00BF00BF01224270DFED890AB0EE600A0FE09A
:40CC800000BF00BF022242700AE000BF0422427006E00522427003E00622427000E000BF00BF7A4AD2ED060A60EE800AFCEEE00A10EE902A91B281700A0AC270734AD2EDD8
:40CCC0001C0A60EE800AFCEEE00A10EE902A91B201710A0A42716C4AB2F8BE1181710A0AC2717047694890ED010A704701B500BF012269466A48006800F2BD10FDF736FCD9
:40CD000020B99DF80000604981F8BD0100BFFFF7E4FC012002F0C3FD1D20F0F767FB08BD01B500BF022269465D48006800F5E870FDF71CFC20B9BDF800005349A1F8D001B0
:40CD400000BF08BD0020504991F8BD110E291AD2DFE801F01A0D0A070E0B0810131B1519171100BF012011E000BF01200EE000BF01200BE000BF012008E0012006E00120FD
:40CD800004E0012002E000BF00BF00BF00BF704700203D4991F8BD110E291DD2DFE801F01D0F0B07100C0812151E171C1A1300BF40F2635013E000BF45F2CC000FE000BFF0
:40CDC000C8200CE000BF322009E0C82007E04FF4FA7004E0642002E000BF00BF00BF00BF70470020294991F8381009B9142012E0264991F83810012901D116200BE02349D8
:40CE000091F8901009B9152005E0204991F89010012900D11720704770B50424214880780A2876D2DFE800F0051399E8E8E8E8E2E4E600201B490870C8808860FFF770FF05
:40CE4000184880781749487001208870D5E0FFF7C8FF144908700846007810B1072088707AE021E0EA060020000000000050434700040040E606002000000140E906002057
:40CE8000C8D8002000247449301F0020542700203027002010280020C0030020C0A90646B403002028280020A848806820B91BF022F8A64988604FE0A44988684FF47A7132
:40CEC0001BF01FF8002847D0FFF70CFFBCEEC00A10EE100A85B22846FFF722FF9C48B0F8AC0068B19A48B0F8AC009949B1F8D011884205DD9648B0F8AC009449C88022E090
:40CF00009348B0F8D001002804DC01208F49C88019E071E08E4890F8BD01032804D08C4890F8BD01062805D18948B0F8D00100F5FA7006E08648B0F8D0018000032190FBCC
:40CF4000F1F08249C8800220804988701AF0D3FF7E498860002008734FE0FFF7C3FE7B48C08800EE900AF8EE600AB4EEE00AF1EE10FA05DB7548007B401C7449087302E0E8
:40CF8000002072490873FFF72CFF704908700846007810B10720887027E06C48007B04280DDB6A48C08800EE900AF8EE600AB0EE600AFFF7B7FA09206449887015E06349E9
:40CFC000886841F288311AF09CFF70B15F48C08800EE900AF8EE600AB0EE600AFFF7A2FA07205A4988701820087006E0012404E0022402E0032400E000BF00BF534800782D
:40D0000018B152490878F9F7C1FA204670BD4F48807870474D480078704700204B498870C870704701B500BF0222694649480068AC30FDF79BFA20B9BDF800004449A1F8CF
:40D04000AC0000BF08BD10B52DED028B404890F8BD0103280ED03E4890F8BD01062809D03B4890F8BD01022804D0394890F8BD0105280CD113F098FF10B1012806D102E095
:40D08000B7EE008A02E09FED348A00BF01E0B7EE008AB0EE480ABDEC028B10BDB7EE000AF0EE400A2A4890F8BD010E2818D2DFE800F007100809110A0B131712141715160D
:40D0C00000BF00BF00BF00BF1FED8C0AF0EE400A07E000BF00BF00BF00BF00BF00BF00E000BF00BF1D4890ED060A20EE200A7047B7EE000AF0EE400A154890F8BD010E281A
:40D1000018D2DFE800F007100809110A0B1317121417151600BF00BF00BF00BF1FEDA10AF0EE400A07E000BF00BF00BF00BF00BF00BF00E000BF00BF084890ED1C0A20EED3
:40D14000200A70470648407A7047000028280020301F0020B4030020D7A3DC405427002030270020B5EEC00AF1EE10FA04DDF4EEE10AF1EE10FA09DAB5EEC00AF1EE10FA8B
:40D1800006D2F4EEC10AF1EE10FA01D8012070470020FCE7FD480078704710B52DED028B0446B0EE408AB7EE000AF0EE408AFFF7F1FF80B3F9F7D9FF68BBF2EE0A0AB4EECA
:40D1C000E08AF1EE10FA03DBDFEDF10AB0EE608AFDEEC80A10EE901A08B200EE900AF8EEE00A38EE600A04F1140101EB8001D1ED000AB7EE001A31EE401A60EE810A04F163
:40D200001401421C01EB820191ED001A41EE000AF0EE608A00BFB0EE680ABDEC028B10BD70B52DED028B04460D46B7EE000AB0EE408AF9F79AFF40B9D64800EBC40000EBE7
:40D24000850090ED000AB0EE408AB0EE480ABDEC028B70BDD0ED000A91ED001A60EE810A90ED011AD1ED011A41EE210A90ED021AD1ED021A41EE210A90ED031A60EE810AA4
:40D28000B0EE600A704710B52DED068B04469FEDC20AF0EE409A94F8C200012804D194ED210A84ED220A87E004F1900104F14C00FFF7D0FFB0EE408AB64A4C3A92F8421093
:40D2C00092F84100FFF7ACFF20EE080AB0EE408A11F07FFEB0EE40AA2046FFF75EFF20EE080AB0EE408AB5EEC08AF1EE10FA06DD94ED1B0A20EE080AB0EE408A05E094EDA6
:40D30000170A20EE080AB0EE408A94F87C0001283AD194ED220A30EE080A84ED220A94ED220AD4ED180AB4EEE00AF1EE10FA43DD94ED220AD4ED1C0AB4EEE00AF1EE10FA60
:40D340003AD2B5EEC08AF1EE10FA0ED294ED220AD4ED1C0A30EE600AB0EE408A94ED180A30EE080AB0EE408A26E094ED220AD4ED180A30EE600AB0EE408A94ED1C0A30EEE1
:40D38000080AB0EE408A17E084ED228AB5EEC08AF1EE10FA08DD94ED220AD4ED1C0A30EE200A84ED220A07E094ED220AD4ED180A30EE200A84ED220A94ED220AD4ED1D0ABA
:40D3C000B4EEE00AF1EE10FA04DD94ED1D0A84ED220A0CE094ED220AD4ED190AB4EEE00AF1EE10FA03D294ED190A84ED220AA0681AF0A9FD00EE100AB8EE409A94ED030ABC
:40D4000060EE098A94ED220AD4ED1C0AB4EEE00AF1EE10FA08DB94ED230AD4ED1C0AB4EEE00AF1EE10FA11D394ED220AD4ED180AB4EEE00AF1EE10FA14D894ED230AD4EDD1
:40D44000180AB4EEE00AF1EE10FA0BDD94ED180AB0EEC00AD4ED1C0A30EE200A30EE280AF0EE408A94ED220AD4ED230A30EE600AB4EEE80AF1EE10FA06DD94ED230A30EEAC
:40D48000280A84ED220A12E094ED220AD4ED230A30EE600AF1EE680AB4EEE00AF1EE10FA05D294ED230A30EE680A84ED220A1AF022FDA06094ED220A84ED230A35484C389B
:40D4C00090F830000A2806D1EEF75CFB18B1B7EE000AF0EE409AFAF7F7F9B8B1F5EEC09AF1EE10FA1ED094ED1E2AF0EE421A94ED1A2AB0EE421A94ED202AF0EE420A94ED69
:40D50000232AB0EE420AFFF72DFE58B1F9F716FF102807D09FED200A84ED220A9FED1E0A84ED230A0120BDEC068B10BD70B52DED088B05460C46B0EE408A94ED010AD4ED85
:40D54000000A30EE600A84ED040A18EE100A24F06DFE41EC190B94ED040A10EE101A084624F064FE41EC1B0BB0EE4B0AF0EE6B0A21F036FAB0EE40AAF0EE60AA53EC192B62
:40D5800051EC1A0B24F020FB0CD207E0DC0300200AD74F417C1F0020000000001FED020A84ED040A94ED040AD5ED040A30EE600A84ED060A94ED070A10EE101A084624F0CF
:40D5C00035FE41EC190B94ED060A10EE101A084624F02CFE41EC1B0BB0EE4B0AF0EE6B0A21F0FEF9B0EE40AAF0EE60AA53EC192B51EC1A0B24F022FC04D21FED190A84EDC4
:40D60000050A12E0FAF760F978B194ED040AD5ED040A30EE200AF0EE000AC0EE208A94ED050A30EE280A84ED050ABDEC088B70BDFD4A92F8281092F83020702A38D19FEDB4
:40D64000FB0A80ED030A9FEDFA0A80ED040A9FEDF90A80ED050A9FEDF80A80ED060A9FEDF70A80ED070A9FEDF60A80ED080A9FEDF50A80ED090A9FEDF40A80ED0A0A9FED52
:40D68000F30A80ED0B0A9FEDF20A80ED0C0A9FEDF10A80ED0D0A9FEDF00A80ED0E0A9FEDEF0A80ED0F0AB7EE000A80ED100A0AE3DD4A92F830200A2A38D19FEDDF0A80ED7C
:40D6C000030A9FEDE70A80ED040A9FEDE60A80ED050AB6EE080A80ED060A9FEDDC0A80ED070A9FEDE10A80ED080A9FEDE00A80ED090A9FEDDF0A80ED0A0AB7EE000A80ED0C
:40D700000B0A9FEDDC0A80ED0C0A9FEDDB0A80ED0D0A9FEDDA0A80ED0E0A9FEDD90A80ED0F0AB7EE040A80ED100ACCE2BE4A92F84A20032A7CD10E297CD2DFE801F07B07E3
:40D740007C7B407F80817B7B7B7B7E7D9FEDBA0A80ED030A9FEDC20A80ED040A9FEDC10A80ED050AB6EE080A80ED060A9FEDB70A80ED070A9FEDBC0A80ED080A9FEDBB0A7B
:40D7800080ED090A9FEDBA0A80ED0A0AB7EE000A80ED0B0A9FEDB70A80ED0C0A9FEDB60A80ED0D0A9FEDB50A80ED0E0A9FEDB40A80ED0F0AB7EE040A80ED100A79E09FED88
:40D7C000B10A80ED030A9FEDB00A80ED040A9FEDAF0A80ED050A9FEDAE0A80ED060A9FEDAD0A80ED070A9FEDAC0A80ED080A9FEDAB0A80ED090A9FEDAA0A80ED0A0A9FED21
:40D80000A90A80ED0B0A9FEDA80A80ED0C0A9FEDA70A80ED0D0A9FEDA60A80ED0E0A9FEDA50A80ED0F0A9FEDA40A80ED100A40E040E0FFE700BF00BF00BF00BF00BF00BF4E
:40D84000B7EE000A80ED030AB7EE000A80ED040AB7EE000A80ED050AB7EE000A80ED060AB7EE000A80ED070AB7EE000A80ED080AB7EE000A80ED090AB7EE000A80ED0A0A44
:40D88000B7EE000A80ED0B0AB7EE000A80ED0C0AB7EE000A80ED0D0AB7EE000A80ED0E0AB7EE000A80ED0F0AB7EE000A80ED100A00BF08E20E297AD2DFE801F079077A4015
:40D8C000B4B3B2B179797979B0AFB6EE000A80ED030A9FED660A80ED040AB7EE040A80ED050A9FED760A80ED060AB0EE000A80ED070AB0EE020A80ED080A9FED710A80ED01
:40D90000090A9FED700A80ED0A0A9FED6F0A80ED0B0A9FED6D0A80ED0C0A9FED6B0A80ED0D0A9FED690A80ED0E0A9FED670A80ED0F0A9FED650A80ED100AC3E19FED630A95
:40D9400080ED030A9FED620A80ED040A9FED610A80ED050A9FED600A80ED060A9FED5F0A80ED070A9FED390A80ED080A9FED5C0A80ED090A9FED400A80ED0A0AB7EE040A97
:40D9800080ED0B0A9FED570A80ED0C0AB7EE080A80ED0D0A9FED490A80ED0E0A9FED520A80ED0F0AB0EE000A80ED100A8AE14DE19FED480A80ED030A9FED460A80ED040AF1
:40D9C0009FED440A80ED050A9FED430A80ED060A9FED420A80ED070A9FED1C0A80ED080A9FED3F0A80ED090A9FED230A80ED0A0AB7EE040A80ED0B0A9FED3A0A80ED0C0ADD
:40DA0000B7EE080A80ED0D0A9FED2C0A80ED0E0A9FED2A0A80ED0F0A68E06CE0A4E018E116E114E1D9E00000301F00208FC2F53EB81E053F295C0F3F9A99193F0AD7233FBA
:40DA40007B142E3FEC51383F5C8F423FCDCC4C3F3D0A573FAE47613F1F856B3F8FC2753F6666263F3333333F9A99593F6666663F3333733F6666863FCDCC8C3F3333933F17
:40DA80009A99993FA69B443D6F12833D6F12033EF4FD543E6F12833E96438B3EBC74933EE3A59B3E0AD7A33E3108AC3E5839B43E7F6ABC3EA69BC43ECDCCCC3E3333D33F24
:40DAC000CDCC1C400AD7234066662640CDCCCC3DCDCC4C3E9A99993E7B14EE3EAE47213F48E17A3F3333B33F6666E63F1FED0D0A80ED100AE6E01FED2B0A80ED030A1FED7A
:40DB00002D0A80ED040A1FED2F0A80ED050A9FEDFC0A80ED060A1FED330A80ED070A1FED350A80ED080A1FED370A80ED090A1FED310A80ED0A0AB7EE000A80ED0B0A1FED00
:40DB4000320A80ED0C0A1FED330A80ED0D0A1FED340A80ED0E0A1FED360A80ED0F0A1FED380A80ED100AADE01FED4D0A80ED030A9FEDE40A80ED040A9FEDE30A80ED050A4F
:40DB80009FEDE20A80ED060A9FEDE10A80ED070A9FEDE00A80ED080A9FEDDF0A80ED090A9FEDDE0A80ED0A0A9FEDDD0A80ED0B0A9FEDDC0A80ED0C0A9FEDDB0A80ED0D0ABD
:40DBC0009FEDDA0A80ED0E0A9FEDD90A80ED0F0A9FEDD80A80ED100A74E09FEDD70A80ED030A1FED6E0A80ED040A9FEDD40A80ED050A1FED620A80ED060A1FED610A80ED4D
:40DC0000070AB7EE040A80ED080A9FEDCD0A80ED090A9FEDCB0A80ED0A0A9FEDC90A80ED0B0A9FEDC70A80ED0C0A9FEDC50A80ED0D0A9FEDC30A80ED0E0A9FEDC10A80ED9A
:40DC40000F0A9FEDBF0A80ED100A3BE000BF00BF00BFB7EE000A80ED030AB7EE000A80ED040AB7EE000A80ED050AB7EE000A80ED060AB7EE000A80ED070AB7EE000A80ED64
:40DC8000080AB7EE000A80ED090AB7EE000A80ED0A0AB7EE000A80ED0B0AB7EE000A80ED0C0AB7EE000A80ED0D0AB7EE000A80ED0E0AB7EE000A80ED0F0AB7EE000A80EDD8
:40DCC000100A00BF00BF70479E490870704710B504469D4890F842106830405C00EE100AB8EE400ADFED990A80EE201A84ED151A954890F842106C3000EB810090ED000AC8
:40DD000084ED160A904890F842107C3000EB810090ED000A84ED170AEDF726FF20B19FED8C0A84ED180A13E017F028FD40B103F0D2F85FEDB30A20EE200A84ED180A07E058
:40DD400003F0C9F85FEDB60A20EE200A84ED180A7D4890F842106A30405C00EE100AB8EE400ADFED7A0A80EE201A84ED191A764890F84210743000EB810090ED000A84ED0F
:40DD80001A0A714890F84210843000EB810090ED000A84ED1B0AEDF7E7FE20B19FED6B0A84ED1C0A13E017F0E9FC40B103F0D3F85FEDD30A20EE200A84ED1C0A07E003F0DD
:40DDC000CAF85FEDD50A20EE200A84ED1C0A5E4890F841105C3000EB41005B4991F84210405C00EE100AB8EE400ADFED580A80EE201A84ED111A544890F84110603000EBBB
:40DE00004100514991F84210405C00EE100AB8EE400ADFED4E0A80EE201A84ED121A4A4890F84110643000EB4100474991F84210405C00EE100AB8EE400ADFED440A80EE7D
:40DE4000201A84ED131AEDF779FE50B13E4890F830000A2800D004E09FED3E0A84ED140A19E0EDF781FE38B117F0B3FC20B1B1EE040A84ED140A0EE0EDF7AFFE38B117F070
:40DE8000A8FC20B11FEDEF0A84ED140A03E09FED320A84ED140A2C4890ED7E0A84ED010A9FED2E0A84ED020A0120FFF70DFF264890F82800072806D117F078FC18B101203D
:40DEC00084F8740002E0002084F874002046FFF7AFFB0A20EFF78AFA0B20EFF787FA0C20EFF784FA0E20EFF781FA0D20EFF77EFA1120EFF77BFA1020EFF778FA012010BD68
:40DF00007B144E3F3789213F4C37293FE926313F8716393F2506413F39B4483FD7A3503F7593583F8941603F2731683FC520703FD9CE773F77BE7F3F3333B33ED7A3303FD3
:40DF40006666A63FDC030020301F00200000C8420000C8C20000FA4300C05A45000000002DED028B3026FE48FE490860001DFE490860001DFD4908600C38FD490860343073
:40DF8000FC490860401CFC490860B938FB490860FFF79DFEFA4890F82800F14990390870F74890ED0F0A084680ED010A9FEDF50A80ED270A90ED1E0AF34880ED1B0A08468C
:40DFC00090ED1A0AF04880ED1C0ADFF8C0C300DFDFF8BCC300DF8046302201211AF095F8DFF8ACC300DF804601211AF0BDF80321E84880F8401000BF002231464CF20300F5
:40E00000DFF894C300DF0446012C17D100BFE14890F8410040F00101DE4880F84110B0F84C004FF6FF71884207DADA48B0F84C00401C81B2D748A0F84C10DDE7022CDBD1F8
:40E04000DFF858C300DF054605F0020038B3C4488838FFF73CFECA4890F82800C04990390870C74890ED0F0A084680ED010A1021C548DFF82CC300DF012810D0B84890387B
:40E0800090ED1E0AC04880ED1B0AB548903890ED1A0ABD4880ED1C0ADFF808C300DF05F001000028A8D01021B748DFF8F4C200DF01287DD02022AA49103901F120001FF05B
:40E0C000DEFA19F018FF0746A548903890F8C00007286ED2DFE800F0049EA4B5CCE1F300A94890F84100012812D1A748816B384619F038FFFA280BD203209949903981F878
:40E10000C000012081F8C100002081F8C20080E005F06EFCD0B1F9F767FBB8B19A4890F85900012812D19848016D384619F01AFFFA280BD205208A49903981F8C000012097
:40E1400081F8C100002081F8C20062E005F050FCD0B1F9F749FBB8B18B4890F86500012812D18948C16D384619F0FCFEFA280BD206207B49903981F8C000012081F8C100D7
:40E18000002081F8C20044E005F032FCE0B1F9F72BFBC8B17C4890F84D00012814D17A48416C384619F0DEFEFA280DD2042001E0BDE095E06A49903981F8C000012081F8BD
:40E1C000C10081F8C20024E005F012FCD0B1F9F70BFBB8B16C4890F83500012812D16A48C16A384619F0BEFEFA280BD202205C49903981F8C000012081F8C100002081F8E3
:40E20000C20006E000205649903981F8C10081F8C2006BE000205249903981F8C00065E0F9F7E2FA28B101204D49903981F8C10006E000204A49903981F8C10081F8C000B8
:40E2400054E0514890F8410030B14F48816B384619F088FEFA2805D900204149903981F8C00004E001203E49903981F8C1003DE0F9F7BAFA38B101203949903981F8C1000C
:40E2800081F8C20008E000203549903981F8C10081F8C20081F8C00028E0F9F7A5FA28B101202F49903981F8C10006E000202C49903981F8C10081F8C00017E0FFE7F9F796
:40E2C00093FA28B101202649903981F8C10006E000202349903981F8C10081F8C00005E000201F49903981F8C10000BF00BF1C48903890F8C10080B11948903890F8C00072
:40E3000000EB40012048143000EB810090ED010A1348903880ED210A05E01FEDF00A1048903880ED210A1848DFF878C000DF0C48903890F8C10001287ED1EDF7FFFB98B35F
:40E3400002F0A4FD104880ED040A05499039087891ED011AF0EE410A0B4991ED041A24E03C290020C4030020C8030020CC030020D0030020D4030020D8030020E0030020BC
:40E38000301F002099A0063C38280020350C0408A114040850410020C108040809080408290D0408450C040816E0B0EE410A02F084FCFE4880ED200A0146087891ED011A15
:40E3C000F0EE410A91ED211AB0EE410A02F075FCF64880ED210A3BE0EDF7C6FB28B1ECF72FFFF24880ED200A32E0EDF7B4FB38B302F04CFDEE4880ED040A10F0E6FDB0EEA1
:40E40000408AEB48D0ED040AB0EE600AF0EE480A02F011FDE54880ED200A10F0D6FDB0EE408AE248D0ED210AB0EE600AF0EE480A02F001FDDD4800E031E080ED210A07E00E
